:020000040800F2
:100000006005002015A0010855710108577101080D
:100010005F710108677101086F710108000000003D
:1000200000000000000000000000000077710108DF
:1000300079710108000000007B7101087D710108E1
:10004000F9A70108FDA7010801A8010805A80108F2
:1000500009A801080DA801084B72010841720108A6
:10006000377201082D7201082372010811A80108D6
:1000700015A8010819A801081DA8010821A8010850
:1000800025A8010829A801082DA8010831A8010800
:100090009D71010835A8010839A80108F57101080A
:1000A000000000003DA8010841A8010845A801087A
:1000B00049A801084DA8010851A80108A771010825
:1000C00055A8010859A801085DA8010861A8010800
:1000D00065A8010869A801086DA8010871A80108B0
:1000E000C171010875A8010879A801087DA8010857
:1000F00081A80108C0B23A2801D1012000E0002007
:10010000C0B270470100C9B2212904DAC0B20A287E
:1001100001D0012000E00020C0B27047C0B22C28FE
:1001200001D1012000E00020C0B27047C0B23B28DE
:1001300001D1012000E00020C0B27047C0B20A28FF
:1001400001D1012000E00020C0B27047C0B23F28BA
:1001500001D1012000E00020C0B27047C0B22A28BF
:1001600001D1012000E00020C0B2704738B5040082
:100170000D00002C08D1CD22DFF84819DFF848091E
:1001800001F0F6FDAFF30080002D07D1CE22DFF89D
:1001900034197FA001F0ECFDAFF30080E0686860E7
:1001A0002069A860A068286031BD38B504000D0042
:1001B000002C07D1DB22DFF80C1975A001F0D8FD67
:1001C000AFF30080E56031BD38B505000C00002CB0
:1001D00008D1E922DFF8EC18DFF8F00801F0C8FDDB
:1001E000AFF300806068E860A06828612068A860BC
:1001F0000020687531BD38B504000D00002C08D111
:10020000FB22DFF8C018DFF8C40801F0B1FDAFF33E
:100210000080002D08D1FC22DFF8A818DFF8100CB0
:1002200001F0A6FDAFF30080E068286031BD10B595
:1002300004002000C0B201F0ADFD002801D0012073
:1002400000E00020C0B210BD10B504002000C0B214
:1002500001F0ACFD002801D0012000E00020C0B278
:1002600010BD10B504002000C0B201F0A9FD0028A7
:1002700001D0012000E00020C0B210BD10B5040084
:100280002000C0B201F09CFD00280ED12000C0B2B9
:10029000612803DB2000C0B2672806DB2000C0B263
:1002A000412804DBE4B2472C01DA012000E0002001
:1002B000C0B210BD2DE9F14F0C00150098460A9F01
:1002C000009E002E28D0002C26D0002D24D03800EF
:1002D000C0B200280CD15FF03C0B5FF00009B246C1
:1002E0004A465946504601F0AFFD0020707501E0C6
:1002F00001207075F460F06828443061F068B060E7
:1003000086F814800020B075DFF8F40B00683060C8
:1003100000207060012000E00020BDE8F28F2DE990
:10032000F04104000D0016001F005FF00008002CD3
:1003300011D0002D03D0E068286001208046002EF7
:1003400003D02069306001208046002F03D0A07DBB
:100350003870012080464046C0B2002809D14FF4D1
:10036000CF72DFF86017DFF89C0B01F001FDAFF3EF
:1003700000804046C0B2BDE8F0810200002A05D0EE
:10038000002901D010680860506800E00020704724
:10039000746F00002DE9F041804644467FF001056E
:1003A000002C00F0B580A068002800F0B180206922
:1003B000E168401A002800F0AB802169A068091AA2
:1003C0000129C0F2A5805FF0FF363500607D00286E
:1003D00009D1002084F83000002084F8310000208A
:1003E000A0620020E062A1682069814200F0908054
:1003F000A168481CA0600F7894F83000002810D144
:100400003800C0B2232803D1012084F83000EAE785
:10041000DFF8F40A00682060DFF8F00A6060350059
:1004200076E094F8310000285CD1A06A002828D139
:100430003800C0B2FFF715FF002808D1DFF8C80A5E
:1004400000682060DFF8C40A6060350060E03800B2
:10045000C0B23038A062A06A0028C4D1207D002834
:1004600004D00220A0750020050003E0E0682061B0
:1004700001200500DFF8880A006820600020606025
:1004800046E03800C0B2FFF7ECFE002808D1DFF8E4
:10049000780A00682060DFF8740A60603500A2E71F
:1004A000A06A401EA062E26A0A203900C9B230394F
:1004B00000FB0212E262A06A002894D1E06A0028E0
:1004C00003D0012084F831008DE70220A075A068D8
:1004D000206100200500DFF8280A00682060002065
:1004E000606015E0E06A002802D0E06A401EE06229
:1004F000E06A00287FF477AF0220A075A068206131
:1005000000200500DFF8F809006820600020606026
:100510002800BDE8F08170B4040021007FF00102E2
:10052000002971D0886800286ED00869CB68C01A8D
:10053000002869D00B6988681B1A012B64DB5FF007
:10054000FF331A00487D002805D1002081F82800DB
:10055000002081F82A008D680869854242D08868A9
:10056000451C8D60057891F82800002816D12800D8
:10057000C0B2222803D02800C0B2272805D181F8B4
:100580002950012081F82800E5E7DFF8C80B006852
:100590000860DFF8C40B48601A0023E091F82900D6
:1005A00091F82A60B0421AD191F829602800C0B2AF
:1005B000864210D001208875002081F828008868C4
:1005C000401E086100200200DFF83409006808605E
:1005D0000020486006E0002081F82A00BBE781F88F
:1005E0002A50B8E791F8280000280DD0087D00288F
:1005F00008D0DFF8600B00680860DFF85C0B48602B
:100600001A0001E001200200100070BC70472DE9C3
:10061000F04107003C007FF00100002C00F08780D3
:10062000A168002900F083802169E268891A002905
:100630007DD02269A168521A012A78DB5FF0FF356C
:100640002E00617D002904D1002084F82C000020B8
:10065000A062A068216988423FD0A168481CA060C0
:1006600091F8008094F82C00002819D14046C0B2BF
:10067000FFF7EAFD002805D0012084F82C000120B6
:10068000A062E6E7DFF8000C00682060DFF8FC0BF2
:100690006060A068401EE060A0682061280046E01D
:1006A000A06A0C2808D3DFF8E80B00682060DFF8A8
:1006B000E40B606028003AE04046C0B2FFF7B7FDA7
:1006C000002803D14046C0B25F2803D1A06A401C75
:1006D000A062BEE7A068401EA060A16820698142B8
:1006E0000DD3207D002808D0DFF8AC0B0068206017
:1006F000DFF8A80B6060280019E0012017E094F8EB
:100700002C0000280BD00320A075A06820610020D9
:10071000DFF8EC17096821600021616007E0DFF86D
:10072000780B00682060DFF8740B60602800BDE87B
:10073000F08138B5040025002000FFF768FF00288D
:1007400001D10421A97532BDF8B507003D007FF045
:100750000104002D00F0B281A868002800F0AE81ED
:100760002869E968401A002800F0A8812969A8686A
:10077000091A0129C0F2A28101200400687D002825
:100780000DD100206863002085F82D00002085F839
:100790002E00002085F82F00202085F83800A96859
:1007A0002869814200F05F81A86806783000C0B2F5
:1007B000FFF7A8FC00281BD095F83800FFF7A2FC33
:1007C000002807D085F83860A868401CA860A86891
:1007D000E860E4E795F83800FFF7A8FC002807D0A8
:1007E00085F83860A868401CA860A868E860D6E76B
:1007F0003000C0B2FFF79AFC002813D095F83800FB
:10080000FFF794FC002805D195F83800FFF77AFC33
:10081000002807D085F83860A868401CA860A86840
:10082000E860BCE728696863E868286395F82D00EC
:1008300068753800FFF7EBFE0400012C01D10120A0
:1008400000E00020C0B200280ED0A86810F8010C0B
:1008500085F83800012085F82D00DFF8A40600682F
:10086000286000206860FEE0002C18D1002085F888
:100870002D00012085F82E00A868696B884206D3F8
:10088000DFF87C060068286000206860EBE0686B99
:100890002861A86810F8010C85F838007FE7686BBC
:1008A0002861286BE8603000C0B2FFF723FC002805
:1008B0002AD095F82F0000281BD195F83800FFF7B3
:1008C00019FC00280AD05FF0FF300400DFF8940B19
:1008D00000682860DFF8900B6860C4E0DFF820064D
:1008E000006828600020686085F8386001200400F6
:1008F00055E75FF0FF300400DFF8700B00682860F8
:10090000DFF86C0B6860AEE03000C0B2FFF726FC89
:10091000002824D095F83800FFF7F4FB002805D113
:1009200095F83800FFF702FC00280DD0DFF8D0055D
:10093000006828600020686085F83860012085F82C
:100940002F00012004002AE75FF0FF300400DFF8E9
:100950001C0B00682860DFF8180B686083E030002B
:10096000C0B2FFF7F3FB00282ED095F8380000281E
:100970001AD095F83800FFF7E9FB002814D195F854
:100980003800FFF7B7FB00280ED195F82E0000289D
:100990000AD0DFF86C05006828600020686001203C
:1009A000040085F83860FAE65FF0FF300400A868BC
:1009B000401EE860A8682861DFF8CC08006828605D
:1009C000DFF8C80868604EE03000C0B2FFF7B6FB41
:1009D00000280BD13000C0B2FFF794FB002805D1EE
:1009E0003000C0B2FFF7A2FB002823D095F82E00FC
:1009F000002811D095F83800FFF77CFB00280BD1B8
:100A0000A868401E286100200400DFF8F404006894
:100A10002860002068600CE0A868401E2861DFF8AC
:100A2000380B00682860DFF8280C68605FF0FF3042
:100A3000040018E0A868286195F82E0000280FD05F
:100A40002868DFF8BC140968884209D0A868401EED
:100A5000E860DFF8340800682860DFF83008686074
:100A60005FF0FF300400002C19D195F83800FFF733
:100A70006DFB002809D095F82F00002802D0062031
:100A8000A8751BE00820A87518E095F82F0000282D
:100A900002D00520A87511E00720A8750EE0012CF2
:100AA0000CD1287D002809D0DFF8AC0A0068286046
:100AB000DFF89C0B68605FF0FF3004002000F2BD9F
:100AC00000000000E8880108C8A60108D0A60108B7
:100AD000F8B507003C007FF00105002C00F0A6816E
:100AE000A068002800F0A2812069E168401A00286F
:100AF00000F09C812169A068091A0129C0F2968141
:100B000001200500607D00281DD1002084F83100FF
:100B1000012084F82900012084F82800012084F8AD
:100B20002A00002084F82B00002084F82C000020EC
:100B300084F82D00002084F83000002084F82E0076
:100B4000002084F82F00A1682069814200F03481E0
:100B5000A168481CA0600E7894F82900002831D0C4
:100B60003000C0B22D2803D03000C0B22B2829D1CC
:100B700094F83100002812D1002084F829000020C8
:100B800084F82B00012084F82800002084F82C0031
:100B9000012084F82A00002084F82D0011E00020B4
:100BA00084F82900002084F82B00002084F8280015
:100BB000002084F82C00012084F82A00002084F80A
:100BC0002D00C0E794F8280000281DD03000C0B2E6
:100BD0002E2819D1012084F8300094F83100002823
:100BE00011D1002084F82800002084F82900012079
:100BF00084F82B00012084F82A00012084F82C00BE
:100C0000002084F82D009EE794F82A0000282CD0BC
:100C10003000C0B2FFF725FB002826D094F8310041
:100C200000280FD1002084F82900012084F82B002F
:100C3000012084F82C00012084F82D00012084F884
:100C40002E0011E0002084F82900002084F82800FC
:100C5000002084F82B00002084F82900012084F86B
:100C60002D00012084F82F006DE794F82D00002856
:100C70003ED03000C0B2FFF751FA002815D1300045
:100C8000C0B2FFF753FA00280FD13000C0B2FFF70F
:100C900055FA002809D13000C0B2FFF733FA002816
:100CA00026D094F82F00002822D094F83100002894
:100CB00003D1A068401EA0607EE094F82F000028B9
:100CC00002D1002084F83100A068401EA060A06816
:100CD000401EA060A0680078FFF714FA002803D037
:100CE000A068401EA060F5E7A068401CA06063E01B
:100CF00094F82B0000281DD03000C0B2FFF702FA94
:100D0000002817D094F8310000280FD1012084F872
:100D10003100012084F82C00002084F828000020F5
:100D200084F82900002084F82A0002E0002084F8DA
:100D3000280008E794F82C0000282ED03000C0B21C
:100D4000452803D03000C0B2652826D194F8310080
:100D5000002812D1012084F83100002084F82C00F2
:100D6000012084F82900002084F82800012084F85C
:100D70002B00012084F82A000BE0002084F82C00CE
:100D8000002084F82800012084F82A00012084F83B
:100D90002900002084F82D00D5E6DFF8B8080068A7
:100DA0002060DFF8B4086060A068401EE060A068C2
:100DB00020615FF0FF30050015F1010F04D0012D17
:100DC00034D1207D002831D015F1010F02D1A06867
:100DD000401EA06094F82E00002827D094F831001F
:100DE000002810D094F82F0000281FD0A0682061A0
:100DF0000A20A07500200500DFF86003006820606D
:100E00000020606012E0A068206194F830000028A3
:100E100002D00920A07501E00E20A075DFF83C0388
:100E20000068206000206060002005002800F2BDFE
:100E3000D8A60108F8B504005FF0FF3526000020B1
:100E40000090707D00280AD116F118013000FFF7DC
:100E50008DF9009916F11800FFF7A7F904E069462B
:100E600016F11800FFF7C7F9DFF8687B200000993A
:100E700057F82110884705002900002930D00129A2
:100E800007D07FF0010081422BD0B1F1FF3F06D0A7
:100E900028E0009916F11800FFF787F92EE0009876
:100EA00057F820100FF26900814203D196F8300004
:100EB000002823D10098401C022810D20098401C22
:100EC0000090009916F11800FFF76FF916F118015C
:100ED0003000FFF779F90A4800683060C4E70DE098
:100EE0000CE00BE07FF00100050040F2DF72DFF85C
:100EF000E81A97A000F03CFFAFF300802800F2BD95
:100F000090A70108E0A60108C8A701083C9D0108B8
:100F1000F8B507003C007FF00105002C00F01581BA
:100F2000A068002800F011812069E168401A0028BB
:100F300000F00B812169A068091A0129C0F205811E
:100F400001200500607D002810D1002084F82C00CD
:100F5000002084F82D00002084F82E00002084F862
:100F60002F00002084F830000020A062A1682069D2
:100F7000814200F0B880A0680078FFF7D7F8002819
:100F800040F0B180A068411CA160067894F82C0064
:100F900000280BD03000C0B2302803D03000C0B2DF
:100FA000312803D1A06A401CA062DFE794F82D002D
:100FB00000280BD03000C0B2302807DB3000C0B2B0
:100FC000382803DAA06A401CA062CFE794F82E000C
:100FD000002809D03000C0B2FFF750F9002803D034
:100FE000A06A401CA062C1E794F82F0000281AD123
:100FF0003000C0B2232806D1012084F82F00012040
:1010000084F83000B2E75FF0FF300500DFF84406F7
:1010100000682060DFF840066060A068401EE06065
:10102000A06820615FE094F82C00002832D194F889
:101030002D0000282ED194F82E0000282AD130004F
:10104000C0B242280AD0482810D051280AD06228BD
:1010500004D068280AD0712804D00BE0012084F85D
:101060002C0083E7012084F82D007FE7012084F81D
:101070002E007BE75FF0FF300500DFF860090068B5
:101080002060DFF85C096060A068401EE060A06836
:10109000206128E0A06A00280BD03000C0B200F028
:1010A0008FFE002805D13000C0B200F07FFE00287E
:1010B0000FD05FF0FF300500DFF898050068206072
:1010C000DFF894056060A068401EE060A0682061C1
:1010D00009E00020050021480068206000206060D1
:1010E000A068401EA060012D02D1207D002801D102
:1010F000002D2AD1A06A00281DD0A068206194F894
:101100002C00002805D00D20A075E068801CE06050
:101110000EE094F82D00002805D00C20A075E068A2
:10112000801CE06004E00B20A075E068801CE0609B
:101130000020050009E05FF0FF300500DFF89C08A3
:1011400000682060DFF8980860602800F2BD0000A9
:1011500030000000C4A70108289D010890A70108DD
:10116000F8B5060034007FF00105002C00F08980FE
:10117000A068002800F085802069E168401A0028F6
:1011800000F07F802169A068091A012979DB01201C
:101190000500607D002802D1002084F82800A068A6
:1011A000216988424CD0A068411CA16007783800B2
:1011B000C0B2FEF7A7FF0028F1D13800C0B2FEF799
:1011C000BDFF002812D0012084F828008120A075DE
:1011D00000200500A068401EE060A0682061DFF8E4
:1011E000400B006820600020606029E094F828002F
:1011F000002818D13800C0B2FEF790FF002812D0A6
:10120000012084F828008420A075A068401EE060BA
:10121000A068206100200500DFF8040B0068206052
:10122000002060600CE0A068401EE060A0682061C3
:101230005FF0FF3005008B48006820608A486060DE
:10124000012D0DD1207D00281BD00020050081201C
:10125000A075DFF8CC0A006820600020606010E014
:1012600015F1010F0DD194F82800002809D00020B5
:1012700005008120A075DFF8A80A00682060002022
:1012800060602800F2BD000098A70108C49C010816
:10129000B4A701086098010894A70108649F010899
:1012A000F8B5060034007FF00105002C77D0A06867
:1012B000002874D02069E168401A00286FD02169A5
:1012C000A068091A01296ADB01200500607D002859
:1012D00002D1002084F82800A168206981424DD005
:1012E000A06807783800C0B2FEF70CFF00280ED0C7
:1012F00094F82800002801D1A068E060012084F85B
:1013000028008320A075A068401CA060E4E7380096
:10131000C0B2FEF713FF002812D0012084F8280085
:101320008120A075A068401EE060A06820610020B8
:101330000500DFF8EC0900682060002060601DE017
:1013400094F8280000280CD0002005008320A07508
:10135000A0682061DFF8C809006820600020606094
:101360000CE0A068401EE060A06820615FF0FF30E4
:1013700005003C48006820603B486060012D0ED1AC
:10138000207D00280BD0002005008120A075A068DA
:101390002061DFF88C090068206000206060280070
:1013A000F2BDF8B5060034007FF00105002C57D0DF
:1013B000A068002854D02069E168401A00284FD066
:1013C0002169A068091A01294ADB01200500607D16
:1013D000002802D1002084F82800A16820698142F9
:1013E0002ED0A068411CA160077894F8280000283E
:1013F00019D13800C0B2FEF785FE002802D0A068DF
:101400002061EAE73800C0B2FEF790FE00280AD05B
:10141000012084F828008220A075A068401EE060AA
:10142000A06820610CE0A068401EE060A068206118
:101430005FF0FF3005000B48006820600A486060DC
:10144000012D0DD194F82800002809D000200500B6
:101450008120A075DFF8C808006820600020606067
:101460002800F2BDA0A70108D89C0108B0A7010878
:10147000389A0108F8B5060034007FF00105002C09
:1014800067D0A068002864D02069E168401A00286D
:101490005FD02169A068091A01295ADB01200500E3
:1014A000607D002802D1002084F82800A16820690E
:1014B00081423ED0A068411CA160077894F82800C2
:1014C000002827D13800C0B2FEF71CFE0028EDD15D
:1014D0003800C0B2FEF72AFE00280AD0012084F8A6
:1014E0002800A068401EE060A06820618220A075EE
:1014F0001FE03800C0B2FEF721FE00280AD001200C
:1015000084F82800A068401EE060A0682061812067
:10151000A0750EE0A068401EE060A06820615FF04A
:10152000FF300500DFF8FC0700682060DFF8F807EF
:101530006060012D0DD194F82800002809D000200A
:1015400005008120A075DFF8D80700682060002022
:1015500060602800F2BD0000ACA70108F8B50600E5
:1015600034007FF00105002C70D0A06800286DD0F9
:101570002069E168401A002868D02169A068091A2A
:10158000012963DB01200500607D002805D10020D2
:1015900084F82800002084F82900A0682169884286
:1015A0002ED0A06807783800C0B2FEF7ABFD002847
:1015B00006D0012084F82800A068401CA060ECE759
:1015C0003800C0B2FEF7BAFD002806D0012084F82A
:1015D0002900A068401CA06012E094F828000028B0
:1015E0000ED1A068401EE060A06820615FF0FF306F
:1015F0000500DFF8380700682060DFF83407606016
:10160000012D23D194F8280000280FD0207D002838
:101610001CD0DFF80C070068206000206060A06824
:1016200020618520A075002005000FE094F82900B6
:1016300000280BD0DFF8E80600682060002060601A
:10164000A06820618120A075002005002800F2BD5F
:1016500080950108C0A701087C98010810B4040017
:1016600021007FF0010000291CD08A68002A19D0CF
:101670000B69CA689B1A002B14D48B68CA689B1A22
:10168000002B0FD40B698A689B1A012B02DB002206
:10169000100007E00A698B68D21A002A02D15FF0B5
:1016A000FF32100010BC70472DE9FF4F81B00600DB
:1016B0000E9D002E08D140F62832C749DFF8740687
:1016C00000F056FBAFF300800298002808D140F6E6
:1016D0002932C149DFF8600600F04AFBAFF3008011
:1016E0001098002808D140F62A32BB49DFF84C0692
:1016F00000F03EFBAFF300800F98854208D240F621
:101700002B32B549DFF8380600F032FBAFF300802A
:10171000039800280AD1002D08D040F62C32AE499B
:10172000DFF8200600F024FBAFF30080B3467FF023
:1017300001000400DFF810160968CBF80010DFF88C
:101740001016CBF80410002E0ED1029900290BD1EF
:101750000399002908D1002D06D01099002903D142
:101760000F998D42C0F03281002D0ED13000FFF76D
:1017700081FE0400002C08D0DFF8D0050068CBF80B
:101780000000DFF8D005CBF8040000208DF8000041
:1017900000208DF8010000275FF00008A84580F0C8
:1017A00014819DF80000002840F00F81109880F807
:1017B00000805FF000090020072813D2DFF8981599
:1017C000052202FB00F20A441279039B13F8083049
:1017D0009A4205D1052202FB00F28958894601E0B0
:1017E000401CE9E74846002803D15FF0FF300400C1
:1017F000EBE0DBF810A03000FFF7B0FE0400002C97
:1018000003D19BF8160081286DD0CBF810A0DBF82F
:101810000800CBF80C003000FFF720FF00282BD188
:101820003000C8470400002C14D0DFF80005016820
:10183000DBF8000081420CD1DBF80C000078FEF7E9
:1018400075FC002805D081208BF8160000200400CC
:1018500049E0BAE000208DF80100DBF80C10029896
:1018600040F83710DBF81000029901EBC70148601F
:101870000498002808D003E081208BF8160032E09D
:101880009BF816000499C8557F1CCBF810A0DBF814
:101890000800CBF80C003000FFF7E0FE00281FD155
:1018A0003000FFF75DFC0400002C1CD0DFF874044E
:1018B0000168DBF80000814211D1DBF80C000078F0
:1018C000FEF734FC00280AD081208BF81600DFF8E0
:1018D00050040068CBF800000020040003E074E02E
:1018E00081208BF816009BF816108139012902D946
:1018F000C91E33D04EE00F98281A874213D25FF0EA
:10190000FF3004005046CBF80800CBF81000CBF8AD
:101910000C00DFF848040068CBF80000DFF8400452
:10192000CBF8040016E09DF80100002812D05FF00B
:10193000FF300400DFF8EC030068CBF80000DFF8AC
:10194000E803CBF804005046CBF80800CBF81000B1
:10195000CBF80C0001208DF8000027E0AF4215D332
:101960005FF0FF300400DFF8E4030068CBF800000C
:10197000DFF8E003CBF804005046CBF80800CBF8C2
:101980001000CBF80C0001208DF8000001208DF82C
:1019900001000BE05FF0FF300400DFF8AC030068EB
:1019A000CBF80000DFF8A803CBF804009DF8000096
:1019B000002805D1DBF80800CBF80C00CBF810A00C
:1019C0001098077018F10108E8E6200005B0BDE89E
:1019D000F08F0000F0A60108E8880108BCA7010804
:1019E000149D01082DE9FE4F9EB00500002D09D180
:1019F00040F61942DFF86C13DFF8380300F0B8F94D
:101A0000AFF300801E98002809D140F61A42DFF893
:101A10005413DFF8240300F0ABF9AFF300802D98E6
:101A2000002809D140F61B42DFF83813DFF80C0319
:101A300000F09EF9AFF300802B992C98814209D2D7
:101A400040F61C42DFF81C13DFF8F40200F090F9B6
:101A5000AFF30080209800280CD12B98002809D0E3
:101A600040F61D42DFF8FC12DFF8D80200F080F9E2
:101A7000AFF300801F98002809D140F61E42DFF81E
:101A8000E412DFF8E40200F073F9AFF30080A94636
:101A90007FF001000400DFF8B0120968C9F80010F7
:101AA000DFF8AC12C9F80410002D10D11E990029DE
:101AB0000DD1209900290AD12B99002907D02D9901
:101AC000002904D12B9A2C998A42C0F026812B98A8
:101AD00000280ED12800FFF7CDFC0400002C08D010
:101AE000DFF868020068C9F80000DFF86802C9F88A
:101AF00004005FF0000A00208DF800000026002797
:101B00005046C0B2002840F007812D9807705FF062
:101B100000080020072812D2DFF83C12052202FB41
:101B200000F20A441279209B1B789A4205D10522C3
:101B300002FB00F28958884601E0401CEAE7404673
:101B4000002803D15FF0FF300400E5E0D9F810B0C1
:101B50002800FFF703FD0400002C04D199F81600BB
:101B6000812800F08280C9F810B0D9F80800C9F8BF
:101B70000C002800FFF772FD002832D12800C04772
:101B80000400002C14D0DFF8A4010168D9F800008B
:101B900081420CD1D9F80C000078FEF7C7FA002872
:101BA00005D0812089F81600002004005DE0B3E034
:101BB00000208DF80000D9F80C000190D9F8100031
:101BC000029004A8DFF8A411182200F08DF904ABEC
:101BD00099F8162001A90AA800F0CAF9002804D132
:101BE0000FE0812089F816003FE01F9800688642C8
:101BF00007D2DDE90A011E9988552A98002807D0E6
:101C000002E00120824630E099F816002A998855B2
:101C1000761CC9F810B0D9F80800C9F80C002800E3
:101C2000FFF71CFD00281DD12800FFF799FA0400DA
:101C3000002C1AD03B480068D9F80010884210D117
:101C4000D9F80C000078FEF771FA002809D081203D
:101C500089F8160032480068C9F800000020040026
:101C600003E059E0812089F8160099F816108139AF
:101C7000012902D9C91E31D034E02B992C98091AB8
:101C80008E4213D25FF0FF3004005846C9F80800B6
:101C9000C9F81000C9F80C00DFF8C0000068C9F8E6
:101CA0000000DFF8BC00C9F8040014E09DF8000053
:101CB000002810D05FF0FF3004001A480068C9F80F
:101CC00000001948C9F804005846C9F80800C9F8C6
:101CD0001000C9F80C00012082460FE001208DF8A9
:101CE00000000BE05FF0FF300400DFF85C000068EC
:101CF000C9F80000DFF85800C9F804005046C0B227
:101D0000002805D1D9F80800C9F80C00C9F810B0AE
:101D10002D9806707F1CF3E6200021B0BDE8F08FFF
:101D200090A70108A0A70108D89C010898A701085E
:101D3000C49C0108E8A6010834A2010840A20108D9
:101D4000989A0108B09A01089CA70108A4A7010865
:101D5000089A0108209A0108C8950108A8A7010857
:101D6000EC9C0108E88801084CA20108C89A010807
:101D700000B583B00091019202906A460449182090
:101D8000ABBE002801D100F005FA03B000BD00BFD2
:101D90001010020010B5044600F008F820B9303CDD
:101DA0000A2C8041C00F10BD012010BD10B50446A3
:101DB00000F018FA014620460969BDE810400847BE
:101DC00030380A288041C00F7047F0B402461068CE
:101DD00095681318506803EB5004C00748BF4D4482
:101DE000A3422DD013F8016B16F0030004BF13F8C3
:101DF000010BC01C31090F2907D113F8011B0F314A
:101E000003E013F8017B05F8017B401EF9D100299E
:101E1000E6D013F8010BC6F38107032F08BF13F8B0
:101E2000017B00EB0720404228440026B71E8F426A
:101E30001EBF10F8017B05F8017B761CF6D1CFE7B9
:101E4000F0BC02F10C00704762F30F2262F31F42F4
:101E5000401810F0030308D0C91A1FD3DB0748BF8E
:101E600000F8012D28BF20F8022D130030B41446CD
:101E70001546103928BF20E93C00FAD8490728BF89
:101E800020E90C0048BF40F8042D890028BF20F845
:101E9000022D48BF00F8012D30BC7047C91818BF8B
:101EA00000F8012DCB0728BF00F8012D704782688C
:101EB000521C8260426832B103685A1C0260197079
:101EC0004168491E4160704762B38B0708D0521EBB
:101ED00011F8013B00F8013B00F024808B07F6D19C
:101EE000830740F0208000BF103A07D330B4B1E838
:101EF0003810103AA0E83810F9D230BC530724BF8C
:101F0000B1E80810A0E8081044BF51F8043B40F8BD
:101F1000043BD20724BF31F8022B20F8022B44BF28
:101F20000B7803707047121F17D35B0009D151F86B
:101F3000043B20F8023B1B0C121F20F8023BF6D298
:101F40000BE051F8043B00F8013B1B0A20F8023B70
:101F50001B0C121F00F8013BF3D238BF121D521E9A
:101F600024BF11F8013B00F8013BF8D87047040486
:101F70002DE9F84F0600884691461D000027002EE7
:101F800006D1282280498148FFF7F2FEAFF3008096
:101F9000B8F1000F06D129227B497D48FFF7E8FE02
:101FA000AFF30080D8F80410D8F80000091A4029CF
:101FB00003DB032070720020E3E0022070725FF008
:101FC000400B5FF0000A16F11004524659462000FB
:101FD000FFF73AFFD8F80420D8F80000121AD8F812
:101FE000001016F1100000F005F986F808900024A2
:101FF000002000904846C0B209280AD0C0F0B9803D
:102000000B2840D005D30D2845D040D30E2846D00C
:10201000AFE0287C052802DB287C072802DB0520AE
:1020200070722FE0694616F1100000F09BFAC6E9C5
:10203000000100F0A2FA0068002802D003207072AC
:1020400020E0002D1AD0D6E90001D5E9002300F0E8
:102050009FFA08D8D5E90201D6E9002300F098FAE2
:1020600001D8012700E000273800C0B2002802D1C3
:102070000420707206E00020707203E00120070067
:102080000020707275E0002C01D110200400002C9B
:1020900001D108200400002C01D102200400002CF2
:1020A00001D10A2004002200694616F1100000F058
:1020B000D9FAC6E9000100F060FA0068002802D0F1
:1020C0000320707254E0002D4ED0287C052825DBBB
:1020D000287C072822DAD6E9000100F0C7FAC6E911
:1020E00000010A203072D6E90001D5E9002300F092
:1020F0004FFA08D8D5E90201D6E9002300F048FAE2
:1021000001D8012700E000273800C0B2002802D122
:10211000042070722CE00020707229E0287C0028D6
:1021200021D0287C05281EDAD6E90001D5E9002354
:1021300099420DDB01DC90420AD3D5E90201D6E9D0
:102140000023994204DB01DC904201D3012700E027
:1021500000273800C0B2002802D10420707207E0C6
:102160000020707204E003E001200700002070727C
:10217000FFE73800C0B2002801D00020707238009C
:10218000C0B2BDE8F28F00BFA0880108C0A6010858
:1021900028A20108012000F093BA2F00613807E05F
:1021A00005E0A0F161011A2901D2012070474138F0
:1021B0001A288041C00F7047A0F10901052901D3F9
:1021C000202801D10120704700207047A0F1410173
:1021D0001A2938BF20307047A0F161011A2938BF91
:1021E0002038704701487047014870472409002093
:1021F000EC08002001B58B071AD1830724D1121FE8
:1022000021D351F8043BA3F1013C2CEA030C1CF050
:10221000803C04BF40F8043BF1E79CFA8CFCBCFA1C
:102220008CF1C1F118018B40CB4040F8043B13E026
:10223000042A09D311F8013B521E00F8013B5BB19F
:102240008B07F7D1D9E7121D5AB111F8013B521E85
:1022500000F8013B03B1F8D111001CBF0022FFF7C9
:10226000F7FD01BD2DE9FC4D160082468B461F4649
:1022700000F0D5803BF0004108BF002800F0CF807F
:102280004FEA4B02521512F1010F08BF5FEA0B3003
:1022900000F0C5800020002EA94954D57642624D39
:1022A0007D4405F5C275082408E0F20744BFD5E96E
:1022B000002300F00FFA76080835641E002E18BFC0
:1022C000002CF2D104460D466A465046594600F0AD
:1022D000D7FADDF8008022462B4600F009FB424683
:1022E00000F02AFC82468B462AF000023BF00043B5
:1022F00008BF002A7CD04FEA4B01491511F1010FAC
:102300000CBF5FEA0B30002E72D0504659466A4629
:1023100000F0B6FA009C8B4A8B4B00F0DBF92246AA
:1023200000F00AFC20F0000431F0004508BF002C4A
:102330005CD04B005B1513F1010F01D10A0355D09E
:10234000761EE4D152E053DD374D7D4405F1DA05C8
:102350000824F20744BFD5E9002300F0BBF976104A
:102360000835641E002E01DD002CF2D104460D4616
:102370006A465046594600F083FADDF8008022464E
:102380002B4600F0A7F9424600F0D6FB8B4682466A
:102390003BF0004108BF00282AD04FEA4B025215FB
:1023A00012F1010F08BF5FEA0B3021D0002E1FDDB4
:1023B000504659466A4600F063FA009C634A644BF3
:1023C00000F088F9224600F0B7FB20F0000431F05D
:1023D000004508BF002C09D04B005B1513F1010F1D
:1023E00001D10A0302D0761E002EE3DC82468B4622
:1023F0002AF000003BF0004108BF002808D04FEA57
:102400004B02521512F1010F08BF5FEA0B3006D1E3
:1024100000F0AAF81FB1386840F00100386050465B
:102420005946BDE8FC8D00BFE06501002DE9F84983
:1024300009B486B00D4614460BB100211960294637
:10244000069E06A800F015FCC71020F00800012821
:1024500007F0010704942FD10220009001AB0699E8
:102460002A46304600F096FC040002D100200021EC
:102470001DE0029800F068FD022C18DB0DF10C083D
:10248000661EDFF8D0B002460B460020594600F029
:1024900021F9044658F8040B0D4600F055FD22467C
:1024A0002B4600F063FD761E02460B46EDD1049AE2
:1024B000019C079BA2182CE002282DD1009001ABB3
:1024C00006992A46304600F081FE040002D1002021
:1024D000002119E0029800F037FD022C14DB0DF109
:1024E0000C08661EDFF870B000225B4600F0F2F8C0
:1024F000044658F8040B0D4600F026FD22462B46F4
:1025000000F034FD761EEFD1019A00F015FB079B19
:10251000049AFFF7A7FE0CE0032802D100200F4920
:1025200007E0042807BF4FF0FF306FF000410020A4
:1025300000210FB181F0004109B0BDE8F089000031
:102540000000F03F436FAC642806C80A3CBF737FAD
:10255000DD4F157565CDCD410000B0410000F07F25
:10256000002363E70022FBE70FB581B000F038FFDE
:10257000054A2221815001B00FBD80B500F030FF27
:102580000249084402BD0000283B0020283B0020EF
:1025900041EA030C50EA4C0C52EA0C0C4FF4001CBC
:1025A00009D307D01CEB410F9CBF1CEB430F994292
:1025B00008BF904270471CEB410FFBD88B4208BF0D
:1025C000824270472DE9F8430C0091461D4608BF32
:1025D0006C468046464600E0761C307800F002FFEC
:1025E0000028F9D137782D2F18BF2B2F05D116F8D9
:1025F000010F00F0F7FE08B109E02B272B464A46F1
:102600002146304600F0F8FE2268964205D1C4F813
:10261000008000200021BDE8F4832B2F05D14FF06E
:102620000043994209D2BDE8F4832D2FFBD1B1F1CB
:10263000004F12D301D801280FD3FFF795FF0DB13A
:10264000012028602D2F19BF4FF0FF306FF000419F
:1026500000204FF00041BDE8F483404261EB4101AE
:10266000BDE8F48300BF0023ACE7270011F000436E
:1026700003D54942404261F10001A1B1B1FA81F2B2
:1026800041409040C2F12002D141414002F21D423E
:1026900043EA025CC30A420572F1004253EB415027
:1026A0004CEBD121704750B1B0FA80F29040C4F2A7
:1026B000D011A1EB025202EBD02119434005704723
:1026C00080B5AFF30080024A11001820ABBEFBE7D3
:1026D0002600020030B540F2FF7C1CEA11541DBFF9
:1026E0001CEA1355644565453FE0641981EA030C13
:1026F0006FF35F530CF0004C43F48013C90241F0B8
:10270000004141EA505EC5021100A5FB020200280B
:102710004FF00000EEFB01204FF00001E3FB05212C
:1027200018BF42F00102401800214941E3FB0E01AD
:10273000A4F580640D0302D292184041494154F13E
:10274000010470DD450872F1004250F1000051EBC8
:102750000451A1F5801102D441EA0C0130BD40F2D0
:10276000FF7E4CEA0E51002030BD0CEA1355644543
:1027700018BF654581EA030C0CF0004C41D050EACB
:10278000410E1CBF52EA430E02E06146002030BDFC
:1027900024422C441BD15FEA050EF6D0090302BF88
:1027A00001460020AEF1140EB1FA81F5AEEB05043E
:1027B00001FA05FE0C35C5F1200100FA05F5C84007
:1027C0004EEA000E6FF35F5343F480139CE733F03F
:1027D0000043B3FA83F504BFB2FA82FE75440B3DA1
:1027E000641BB5F1200E2FBF02FA0EF3AB40C5F10A
:1027F000200E22FA0EFE38BF43EA0E03AA40641CE4
:102800007CE750EA410E14BF52EA430E6FF000011C
:102810004FF4001515EB430F8EBF194615EB410F12
:102820009DE7B4D830BDD4F10104B4F120050FDA2E
:10283000C4F12005520828BF42F0010210FA05FE3B
:1028400001FA05F57244E2BFE0402843E1400FE0A1
:10285000352C9ADCC5F1200452EA400220FA05F238
:1028600018BF42F0010231FA05F0A1400A430021ED
:1028700072F1004250F1000051EB0C0130BD270015
:1028800010B5144600F002F8226010BDC1F30A53DF
:1028900043B14A0012F5001F28D2A3F2FE32A1EB89
:1028A0000251704750EA410C20D001F0004C31EA4F
:1028B0000C01B1FA81F204BFB0FA80F3D2180B3ADE
:1028C000B2F120032CBF00FA03F1914041EA0C0160
:1028D0003EBFC2F1200C20FA0CF319439040524243
:1028E00040F2FD33D21A01EB0351704700227047CA
:1028F000F0B540F2FF7581EA030C0CF0004C15EACC
:1029000011541DBF15EA1357AC42AF42E5E0BC417C
:10291000C1F31301C3F31303801A994143F48013E5
:1029200004D2641E0018494180185941C90241EA85
:102930005051B1FBF3F603FB1611A2FB0675D7EB62
:10294000C020A94102D2761E80185941C90241EA2D
:102950005051B1FBF3FE03FB1E11A2FB0E75D7EB2A
:10296000C020A94103D2AEF1010E8018594189025D
:1029700041EA9051760546EA8E2EB1FBF3F603FB51
:102980001611A2FB0675D7EB8020A94102D2761E54
:1029900080185941C90241EA50514EEA060EB1FB76
:1029A000F3F603FB1611A2FB0675D7EBC020A94175
:1029B00002D2761E80185941C90241EA5051B1FB3A
:1029C000F3F703FB1711A2FB0735D3EBC020A94196
:1029D00067F100070CBF004247F0010766F3D527F7
:1029E0004FEA1E31B80814F5806412DDBD0775F199
:1029F000004250EB0E5051EB045111F5801F5CBFAB
:102A000041EA0C01F0BD4CF07F6141F0E041002053
:102A1000F0BDBD076D0840EA0E5041F48011D4F1BD
:102A20000104B4F120060ADAC4F120060200E040F5
:102A300001FA06F3E1401843B24015430EE0342C8E
:102A400013DCC6F1200445EA40056D0820FA06F2C1
:102A5000154321FA06F0A1400D43002175F1004213
:102A600050F1000051EB0C01F0BD00205FEA0C01B9
:102A7000F0BDCFB992185B41B3FA83F704BFB2FA45
:102A800082F6BF190B3FB7F120062FBF02FA06F3FB
:102A9000BB40C7F1200622FA06F638BF3343BA40DE
:102AA0001CB1E419641E33E77F4231F00041B1FAF2
:102AB00081F404BFB0FA80F6A4190B3CB4F12006EF
:102AC0002FBF00FA06F1A140C4F1200620FA06F655
:102AD00038BF3143A0403C1B1AE7AC421ABF05EA9D
:102AE0001357AF4212E050EA41061CBF52EA4306B8
:102AF000BFE750EA4107304661461CBF41EA055135
:102B0000F0BD52EA430C08BFC143F0BD00204FF4B2
:102B1000001616EB410F98BF16EB430F08BF16EBDC
:102B2000410F24BFC14305E016EB430F0CBF6146C4
:102B30004CEA0551F0BD2E00124254D440F2FF7C05
:102B40001CEA11530FD0634531D09B1863453CBF3D
:102B500001EB0251704701F0004141EA0C510020A5
:102B6000FFF702BD704750EA410320D001F0004C4E
:102B700091EA0C011CD0B1FA81F30B3B9A420DD9BA
:102B8000D21A994051EA0C01C3F1200C20FA0CFC36
:102B900061449840531C40F2FF7CD7E7914041EAE2
:102BA0000C01C2F1200C20FA0CF31943904070473D
:102BB000B0FA80F31533202BE0D3202AEED3203A4D
:102BC000203B9A4209D9D21A00FA03F141EA0C01DA
:102BD0000020531C40F2FF7CB8E700FA02F141EA02
:102BE0000C0100207047524240F2FF7C1CEA115356
:102BF0000DD06345DBD0B2EB030C3CBFA1EB02511F
:102C000070470CF1010221EA035141F4801150EAAE
:102C1000410CCCD001F0004C352A27DC30B481EADD
:102C20000C01B2F1200309DAC2F12003044601FAD3
:102C300003F5D0402843D1409C400CE0C3F1200272
:102C4000450020FA03F418BF44F0010421FA03F010
:102C500091400C43002174F1004550F1000051EB0C
:102C60000C01244230BC7FF47BAF704761460020EA
:102C700076E72DE9F84305460C462E68002700E06C
:102C8000761C307800F0AEFB0028F9D130782D2882
:102C90000CBF08272B2800D1761C327842F0200088
:102CA0006E2827D1707840F02000612802BFB078EC
:102CB00040F020006E2802D02E68002746E0F61C67
:102CC000B046042798F8000028283FD118F8019F43
:102CD0004846FFF76BF80028F8D1A9F130000A2820
:102CE000F4D398F800005F28F0D029282ED108F1FD
:102CF00001062BE069282CD1707840F020006E2866
:102D000002BFB07840F02000662802D02E6800276D
:102D10001CE016F8030F40F0200047F00307692875
:102D200002BF707840F020006E280FD1B07840F0DC
:102D30002000692802BFF07840F02000742805D1F7
:102D4000307940F02000792808BF761DF4B1266064
:102D50001CE0302A02BF707840F02000782813D1A0
:102D6000B11C08782E2808BF491C0878A0F1610220
:102D7000062A21BFA0F14101062930380A2803D2D2
:102D8000B61C47F0020701E047F001072E60384605
:102D9000BDE8F2832DE9F14F8CB04FF00008169892
:102DA00000EBC0099246C346B9F12D0FC8BF4FF0E2
:102DB0002D09C3F800B0C3F804B0002501E0491C98
:102DC000012508783028FAD000240FE01A68521C38
:102DD0001A600878302807D04FF0010804E04C450D
:102DE000F4DA0DF80400641C491C01250A78A2F1EC
:102DF00030000A28F3D30F461E46FFF7F5F9426A62
:102E000039781078814208BF7F1C002C28460ED1EB
:102E1000397830290BD13068401E30607F1C01208A
:102E2000F6E7302A18BF4FF001087F1C01203A78DE
:102E3000A2F130010A290AD24C45F2DAA2F130009F
:102E40000DF80400641C3268521E3260EDE7B8F1E0
:102E5000000F0FD00DF1FF3212F80910491C02F8D3
:102E6000091007E00DF1FF33195D49B93268521CB2
:102E70003260641E002CF5DC04BF8DF800B0012424
:102E8000002853D0092394FBF3F3C4F1090503EBA5
:102E9000C3035B19092193FBF1F1002201EBC1018E
:102EA000591A17D04FF0010B14E0092193FBF1F1EF
:102EB0001DF8025001EBC101591A1DBF56F82BC075
:102EC0000CEB8C0105EB41050BF1010B46F82B5087
:102ED0005B1C521CA242E8DB397841F020016529D5
:102EE00024D1394617F8012F2B2A16BF2D2A17F89F
:102EF000013B2B2300220025124C08E0A54204DAF6
:102F000005EB85020CEB4205303D7F1C012297F852
:102F100000C0ACF1300EBEF10A0FEFD32D2B08BF6D
:102F20006D423368ED18356002B90F46BAF1000FF3
:102F300003D000B90C9FCAF8007058460DB0BDE828
:102F4000F08F00BF00E1F50510F0004160B148BF0F
:102F50004042B0FA80F29040D21CC2F5846241EA4D
:102F6000025202EBD02140057047430070B491EA51
:102F7000030F4FF0004540F1BF806B40841A71EBA6
:102F8000030604D26E40001BB141121973414FF485
:102F9000001C1CEB410F34BF7CEB430683E00C0D9F
:102FA000A4EB1356362E00F37C80012E45EAC32392
:102FB00041DC43EA525312BFD20292025B0824055D
:102FC00045EAC12141EA5051D2EBC020994125D4B4
:102FD00007D1B0FA80F610FA06F162D00020203650
:102FE00008E0B1FA81F6B140C6F1200220FA02F2FF
:102FF0001143B0404FEAF474B4EB465434F0010688
:103000004FEA74040AD8D6F50016760D04F0004491
:10301000F04061FA06F25040F1404840C00A40EAF0
:10302000415021F0004128BF5FEA500550F10000F7
:1030300044EBD12135E0DB0A45EAC121C90AB6F1EA
:1030400020050EDD42EA0242120CC5F1200603FA09
:1030500006F6EB4042EA06056D42984161F1000137
:103060000DE062FA06F5F240554063FA06FC82EA8A
:103070000C02F3405A406D42904161EB030111F4A0
:10308000801F05D1641E620502D06D004041494198
:1030900021F48011430875F1004350F1000041EB29
:1030A000045170BC70471CEB410F15D223F0004354
:1030B00052EA43060BD04FEA4C0CBCEB410F04D84C
:1030C0000C0D661E342EB7DDEBE7801A994150EAED
:1030D000410608BF0021E4E708BF1CEB430F28BFEF
:1030E0006FF00001DDE7000070B491EA030F4FF0CC
:1030F00000457FF543AF6B40841A71EB030603D2A2
:10310000001BB141121973414FF4001C1CEB410F1D
:1031100034BF7CEB430442E00C0DA4EB1356352E78
:103120004FDC45EAC323DB0A45EAC121C912B6F1E7
:1031300020050DDD63FA05F6EB4086EA0305124231
:1031400018BF45F00105C01851F100010CD213E081
:1031500062FA06F5F2405540F3415A40B340F3405D
:103160005A408018594107D349085FEA30005FEAA6
:10317000350528BF45F0010501F58011420875F1BC
:10318000004250F1000041EB04514E0016F5001FC3
:1031900070BC38BF70470020090D090570471CEB53
:1031A000410F10D252EA43060BD0BCEB410F05D8B9
:1031B0000C0DAB43661E342EB6DD02E0AB43801827
:1031C000594170BC704770BC704701022DE9F14F46
:1031D0008CB09346169CC4EBC4044FF00008232C1B
:1031E000C8BF2324C3F80080C3F80480002501E091
:1031F000491C012508783028FAD000BF0FF2B01022
:1032000071A2C246019000920DF108090E461F46B8
:103210000FE03968491C396009E05445F9DB019A2F
:103220000099801A085C09F80A000AF1010A761C64
:10323000012531785EA0162200F0B4F90028ECD107
:10324000FEF7D2FF406A31780278914208BF761CBF
:10325000BAF1000F17D13078302814D13968491EDF
:103260003960761C0125F6E754450ADB019A00997E
:10327000801A085C09F80A000AF1010A3968491E37
:103280003960761C012531785FF0160248A000F005
:1032900089F90028E8D151468C4215DA19F8041052
:1032A000072904DD0DF10702115D491C1155214666
:1032B0003B685B1C3B6007E00DF107035A5C4AB9B1
:1032C0003B685B1C3B60491E0029F5DC04BF8DF8A0
:1032D000088001213A689200002D3A605AD04FF0E0
:1032E000070991FBF9F9C1F1070CC9EBC909E144E0
:1032F000072299FBF2F20023C2EBC202B9EB0202F1
:103300001AD04FF0010817E057F8282004EB0210FC
:1033100047F828000DE0072202A899FBF2F2C2EB61
:10332000C202C45CB9EB0202EED108F1010847F811
:10333000284009F101095B1C8B42ECDB317841F03C
:103340002001702926D1314616F8012F2B2A16BFED
:103350002D2A16F8013B2B2300229446134809E03E
:10336000844505DA0CEB8C020EEB4202A2F1300C24
:10337000761C012296F800E0AEF130040A2CEFD35F
:103380002D2B08BFCCF1000C3B689C44C7F800C053
:1033900002B90E46BBF1000F03D005B90C9ECBF865
:1033A000006040460DB0BDE8F08F000000E1F5057B
:1033B00030313233343536373839616263646566AB
:1033C000414243444546000000010203040506074C
:1033D00008090A0B0C0D0E0F0A0B0C0D0E0F000046
:1033E0000020704710B50446FEF7FCFE014620465B
:1033F000096ABDE8104008472DE9FC4F85B00C462E
:1034000093460BB100221A600290824601E00AF155
:10341000010A9AF80000FFF7E5FF0028F7D19AF8B3
:1034200000002D2818BF2B2807BF1AF8010B8DF8B4
:1034300000002B218DF80010BBF1000F019405D482
:10344000BBF1010F02D0BBF1250F04DB002C72D0C1
:10345000029820606FE0BBF1000F0DDDBBF1100F93
:1034600004BF9AF80000302802BF9AF8010040F02B
:103470002000782814D10EE09AF80000302818BFF8
:103480004FF00A0B0CD19AF8010040F02000782888
:1034900004D14FF0100B0AF1020A01E04FF0080BC3
:1034A000CDF810A001E00AF1010A9AF800003028D6
:1034B000F9D0094878442030002428300025CDF880
:1034C0000CA000260027A1468DF80100DFF8088037
:1034D000F84408F1040819E04850010001469DF83D
:1034E0000100081A5FFA80F95846A0FB04234FEA4E
:1034F000EB7100FB053301FB0433264600212F4608
:1035000012EB090443EB01050AF1010A9AF80000E5
:1035100000F074F801465A4608F1280000F042F81D
:103520000028DBD1049951455A4607D1019810B1C2
:103530000199029808600020002130E0039B18F8F0
:103540000210AAEB03035B1A002B1BD410DC002132
:10355000B4EB090065EB01018D4209D301D8844227
:1035600006D3D31700F054F8B94208BFB04209D0CF
:10357000FEF7FAFF069808B1012101604FF0FF3411
:10358000254606E09DF800002D2802D1644265EB37
:103590004505019808B1C0F800A02046294607B0AB
:1035A000BDE8F08FC9B2830706D0521E22D310F8AF
:1035B000013B9942F7D11FE0083A13D302F104020C
:1035C00041EA012141EA014150F8043B121F21BFA9
:1035D0004B40A3F1013C2CEA030C1CF0803FF3D0DC
:1035E000C9B2001F083210F8013B521E28BF91EAF1
:1035F000030FF8D818BF0120401E704710B50446CD
:10360000FEF7F0FD01462046896ABDE810400847F4
:10361000BBBBE1B1B2F5803F80F07E80022A1ED9AB
:103620008C46B1FBF2F102FB11C31B0443EA1043C9
:10363000B3FBF2FC02FB1C3380B240EA0343B3FB52
:10364000F2F002FB103240EA0C4000237047022ADD
:1036500005D98446B0FBF2F002FB10C270474AB1B4
:1036600005D100F0010249085FEA300070470022EE
:103670000023704700F0E4B80B0002000021002096
:103680007047904271EB030CF6D3B3F5803F2FD215
:10369000F0B5B3FA83F7B1FA81F4A7F10F0E3D1B31
:1036A0005340CEF1200602FA0EF2F3415340B5F139
:1036B0000F0746D80F3C2C444140C4F12006A040DF
:1036C000F1414140B1FBF3F603FB1611A2FB0645A5
:1036D000001BA94102D2761E8018594180EA0102DE
:1036E00021FA0EF362FA0EF200215A403046F0BD84
:1036F00030B4B1FBF3FC03FB1C11A2FB0C45001B17
:10370000A94103D2ACF1010C8018594130BC0246EA
:103710000B46604600217047B2F1807F65D3F0B55B
:10372000B2FA82F7B1FA81F4C7F10F063D1B22FA13
:1037300006F307F1110EF24120355A40B5F10F079B
:10374000B8D94140C4F12006A040F1414140B1FB4D
:10375000F3FC03FB1C11A2FB0C45001BA94103D287
:10376000BCF1010C801859410F2F12D30F3FC90330
:1037700041EA5041B1FBF3F603FB1611A2FB0645EB
:10378000D4EBC030A94102D2761E8018594146EAD6
:10379000CC3C07B34140C7F12006B840F14141405D
:1037A000B1FBF3F603FB1611A2FB0645001BA94172
:1037B00002D2761E8018594180EA010221FA0EF3E6
:1037C000C7F1200462FA0EF20CFA07F05A402CFA04
:1037D00004F13043F0BD80EA010221FA0EF300212A
:1037E00062FA0EF260465A40F0BD8C46B1FBF2F12F
:1037F00002FB11C31B0243EA1063B3FBF2FC02FBA2
:103800001C331B024CEA002043EA1063B3FBF2FCBA
:1038100002FB1C331B024CEA002043EA1063B3FB9B
:10382000F2FC02FB1C331B024CEA002043EA10634B
:10383000B3FBF2FC02FB1C324CEA00200023704771
:10384000704770B5040000250026002C01D101202E
:1038500079E094F8E901002805D1002084F8E80116
:10386000200001F05DFA032084F8E901002061687E
:10387000884222D21C21012201FB00F3234483F859
:10388000292001FB00F2224482F82800002201FBDB
:1038900000F3234483F82B20002201FB00F3234490
:1038A0005A63002201FB00F323449A63002201FBC8
:1038B00000F12144CA63401CD9E7002160688142BD
:1038C00025D21C20002200FB01F3234483F80921A8
:1038D00000FB01F2224482F80811002200FB01F3F0
:1038E000234483F80B21002200FB01F32344C3F897
:1038F0001421002200FB01F32344C3F81821002205
:1039000000FB01F02044C0F81C21491CD6E701202F
:103910002268A2F8400000202268A2F8400000229D
:103920002068A0F8442000222068A0F850204FF41E
:103930003F422068A0F84020002084F824000120A5
:1039400084F8E901002070BD10B50400002C01D1FD
:1039500001200CE0032084F8E901200000F010F8B9
:10396000200001F00EFA002084F8E901002010BDCB
:1039700010B504000121200001F0ADFC002010BDB5
:10398000010091F8E801012801D1022012E0012094
:1039900081F8E80101220868A0F8402000220868A8
:1039A000A0F8442003220868A0F84020002081F8F5
:1039B000E801002070472DE9FC41040000260020AA
:1039C000ADF800002068B0F84400ADF80200000433
:1039D00040F11C82BDF8020010F00F000700380013
:1039E000C0B2002840F0C280BDF80200C00633D447
:1039F0002068018848F60F7001402068018014F1AA
:103A0000280005002068B0F85000297810EBC100AC
:103A1000216811EB400101F20441088880B2800561
:103A2000800DA8612869A969084428610021200047
:103A300001F0D3F994F824000028C3D06869002865
:103A4000C0D194F8241051F080012068A0F84C10E7
:103A5000002084F82400B5E714F584700500206880
:103A60000088ADF80000BDF80000000522D52068F0
:103A7000B0F85000297810EBC100216811EB40012B
:103A800001F20C41088880B28005800DA861AB6905
:103A90009BB2AA8814F5F671206800F0E0F920685E
:103AA000018840F68F70014020680180200001F0FD
:103AB00079F987E7BDF80000000483D52068018804
:103AC00040F68F700140206801802068B0F85000F7
:103AD000297810EBC100216811EB400101F20C4183
:103AE000088880B28005800DA861A86900280AD0E6
:103AF000AB699BB2AA882969206800F0B0F92969EE
:103B0000A869084428610021200001F054F92068C8
:103B1000B0F85010206810EB410000F20C40E9684A
:103B20003F290BD3EA685209297B11F01F0F00D1FE
:103B3000521E920252F40042028007E0E9684908EE
:103B40002A7BD20700D5491C8902018020680188A0
:103B50004BF68F70084090F4805090F4005040F481
:103B6000004050F08000216808802BE72168380071
:103B7000C0B231F82000ADF80000BDF8000000042C
:103B800040F19F8021683800C0B231F8201040F623
:103B90008F70014020683A00D2B220F8221039001C
:103BA000C9B21C20414304EB010010F584700500EC
:103BB000A87A00281AD12068B0F85000297810EBB4
:103BC000C100216811EB400101F20C410888800519
:103BD000800D0600300080B2002851D033009BB227
:103BE000AA882969206800F03AF949E02168287814
:103BF00031F8200040041AD52068B0F85000297828
:103C000010EBC100216811EB400101F2044108886A
:103C10008005800D0600300080B2002821D03300DE
:103C20009BB2EA882969206800F019F919E0206838
:103C3000B0F85000297810EBC100216811EB400169
:103C400001F20C4108888005800D0600300080B22A
:103C5000002806D033009BB22A892969206800F029
:103C6000FEF82168287831F8201048F68F7001405E
:103C700041F4004151F0C00120682A7820F8221058
:103C8000A969300080B24118A9612969300080B269
:103C9000084428616869002804D0310089B2E868C6
:103CA000814204D22978200001F085F809E0D5F896
:103CB00018806B692A692978200000F014FDC5F886
:103CC0001880BDF8000000067FF57CAE3900C9B24F
:103CD0001C20414304EB0100283005002168380016
:103CE000C0B231F8201048F60F70014020683A0049
:103CF000D2B220F82210A87A00281AD12068B0F891
:103D00005000297810EBC100216811EB400101F24D
:103D10000441088880B28005800DA861A869002848
:103D200051D0AB699BB2AA882969206800F071F86C
:103D300049E02168287811F8200040061AD520684B
:103D4000B0F85000297810EBC100216811EB400158
:103D500001F20441088880B28005800DA861A8693D
:103D6000002821D0AB699BB2EA882969206800F05D
:103D700050F819E02068B0F85000297810EBC10025
:103D8000216811EB400101F20C41088880B28005E6
:103D9000800DA861A869002806D0AB699BB22A896A
:103DA0002969206800F035F82168287831F820105A
:103DB00048F68F70014041F4404151F08001226883
:103DC000287822F820102068B0F85000297810EBED
:103DD000C100216811EB400101F20441088880B262
:103DE0008005800DA8612969A8690844286168696F
:103DF000002804D12978200000F0EFFFE2E56B698C
:103E00002A692978200000F036FDDBE50020BDE8B6
:103E1000F681F0B504001F00BFB27F1C7F081000C0
:103E200080B214EB400C1CF5806C3800002815D0D3
:103E300091F800E07546491C91F800E05FEA0E2E0B
:103E40001FFA8EFE5EEA050E7646ACF800601CF1A5
:103E5000020C1CF1020C491C401EE7E7F0BD2DE9E5
:103E6000F04104001E00B6B2760827008C46100010
:103E700080B217EB400E1EF5806E3000002813D084
:103E8000BEF8008045461EF1020E8CF800501CF171
:103E90000108AC465FEA1C2C88F800C018F1010C40
:103EA0001EF1020E401EE9E75FEAC37804D5BEF8B2
:103EB000008045468CF80050BDE8F08138B505001B
:103EC00000242868B0F84400000402D52800FFF759
:103ED00072FD2868B0F8440040050FD52868B0F896
:103EE00044104FF6FF3001402868A0F84410280025
:103EF00000F08BFF0021280000F082F82868B0F85D
:103F00004400400408D52868B0F844104BF6FF7010
:103F100001402868A0F844102868B0F844008004E4
:103F200008D52868B0F844104DF6FF7001402868A5
:103F3000A0F844102868B0F84400C0041AD52868D6
:103F4000B0F840104FF6FB7001402868A0F8401010
:103F50004FF43D4004002868A0F84040280000F0DD
:103F600070FF2868B0F844104EF6FF7001402868D2
:103F7000A0F844102868B0F84400000520D528684F
:103F8000B0F844104FF2FF7001402868A0F84410C8
:103F90002868B0F8401051F008012868A0F84010D7
:103FA0002868B0F8401051F004012868A0F84010CB
:103FB0002868B0F84400C00402D4280000F031FFA3
:103FC0002868B0F8440080050BD52868B0F8441084
:103FD0004FF6FF5001402868A0F84410280000F078
:103FE0000DFF2868B0F84400C00508D52868B0F86F
:103FF00044104FF6FF6001402868A0F8441031BD1E
:10400000020092F8E801012801D1022011E001200C
:1040100082F8E8010800C0B2002804D180231068AB
:10402000A0F84C3001E082F82410002082F8E8016A
:10403000002070472DE9F0410400002508060AD54C
:104040000E00F6B216F07F061C20464304EB060075
:1040500010F1280609E00E00F6B216F07F061C20CB
:10406000464304EB060010F5847611F07F003070B3
:104070000800C0B2C0097070100080B2F060F37028
:1040800094F8E801012801D1022001E2012084F81E
:10409000E801F078002805D0022812D02DD303289B
:1040A0001CD039E02768307837F8207048F68F1038
:1040B000074057F40077D4F800C030782CF820700F
:1040C0002AE02768307837F8207048F68F100740CC
:1040D000D4F800C030782CF820701DE027683078C4
:1040E00037F8207048F68F10074057F4C067D4F8AF
:1040F00000C030782CF820700EE02768307837F850
:10410000207048F68F10074057F48067D4F800C03D
:1041100030782CF82070FFE748F2800C48F68F7753
:10412000D4F800E030783EF820E017EA0E0E307840
:1041300050EA0E0E5CEA0E0ED4F80080307828F8B3
:1041400020E0B07A002840F0AC80707800283AD0A7
:104150002068B0F8500096F800E010EBCE00D4F8DC
:1041600000E01EEB400E1EF5806EB6F804804FF6A0
:10417000FE7010EA0808AEF80080D4F800E030784D
:104180001EF8200040060ED5D4F800E030783EF846
:104190002000074047F4004757F0C007D4F800E07C
:1041A00030782EF820702768307837F8200048F6ED
:1041B000BF77074097F020075CEA070C2768307844
:1041C00027F820C05FE12068B0F8500096F800E0C2
:1041D00010EBCE00D4F800E01EEB400E1EF5816E11
:1041E000B6F804804FF6FE7010EA0808AEF80080BA
:1041F0002068B0F850E030781EEBC00E206810EB5D
:104200004E0000F20C40D6F80CE0BEF13F0F11D387
:10421000D6F80C805FEA581896F80CE01EF01F0FD5
:1042200001D1B8F101085FEA882858F40048A0F8E5
:1042300000800EE0D6F80CE05FEA5E0E96F80C8087
:104240005FEAC87801D51EF1010E5FEA8E2EA0F854
:1042500000E0D4F800E030783EF8200040040ED5AD
:10426000206896F800E030F82E00074047F44047F9
:1042700057F08007206896F800E020F82E70276835
:10428000307837F820004BF68F77074097F4805747
:1042900097F400575CEA070C2768307827F820C0AD
:1042A000F1E0D4F800E030783EF8208017EA080802
:1042B00048F4014858F08008D4F800E030782EF82F
:1042C00020802068B0F8500096F800E010EBCE0097
:1042D000D4F800E01EEB400E1EF5806EB6F80680A6
:1042E0004FF6FE7010EA0808AEF800802068B0F8BB
:1042F000500096F800E010EBCE00D4F800E01EEB82
:10430000400E1EF5816EB6F808804FF6FE7010EA7A
:104310000808AEF80080707800285CD1D4F800E07E
:1043200030783EF8200040040FD5D4F800E0307813
:104330003EF8208017EA080848F4404858F0800802
:10434000D4F800E030782EF82080D4F800E03078FF
:104350001EF8200040060FD5206896F800E030F8DF
:104360002E00384040F4004050F0C000D4F800E087
:1043700096F800802EF82800D4F800E030783EF857
:104380002000074047F4004757F0C007D4F800E08A
:1043900030782EF820702768307837F820704BF688
:1043A0008F70384090F4805090F400505CEA000028
:1043B000D4F800E037782EF827002768307837F8EF
:1043C000200048F6BF7707405CEA070C2768307882
:1043D00027F820C057E0D4F800E030783EF82000FD
:1043E00040040FD5D4F800E030783EF82000384083
:1043F00040F4404050F08000D4F8008096F800E08F
:1044000028F82E00206896F800E010F82E004006EC
:104410000FD5D4F800E030783EF8208017EA08087D
:1044200048F4004858F0C008D4F800E030782EF87E
:104430002080D4F800E030783EF82000074047F4B0
:10444000404757F08007D4F800E030782EF820700D
:104450002768307837F8207048F6BF7038405CEA3B
:104460000000D4F800E037782EF82700276830786D
:1044700037F820004BF68F7707405CEA070C276877
:10448000307827F820C0002084F8E8012800C0B266
:10449000BDE8F08170B4020008060AD50B00DBB25B
:1044A00013F07F031C20434302EB030010F12803A9
:1044B00009E00B00DBB213F07F031C20434302EB47
:1044C000030010F5847311F07F0018700800C0B26B
:1044D000C009587092F8E801012801D1022000E1DA
:1044E000012082F8E801987A00284CD158780028F9
:1044F00024D01468187814F8200040060ED51468EB
:10450000187834F8204048F68F70044044F4004492
:1045100054F0C00410681D7820F8254014681878FD
:1045200034F8204048F6BF70204040F4004050F07E
:10453000800015681C7825F82400CEE014681878EF
:1045400034F8200040040ED51468187834F8204060
:1045500048F68F70044044F4404454F080041568D9
:10456000187825F820401468187834F820404BF665
:104570008F70204040F4004050F0800014681D7897
:1045800024F82500A9E05878002853D11468187839
:1045900034F8200040040ED51468187834F8204010
:1045A00048F68F70044044F4404454F0800410688E
:1045B0001D7820F8254010681C7810F8240040066B
:1045C0000ED51468187834F8204048F68F700440EF
:1045D00044F4004454F0C00410681D7820F82540CD
:1045E0001468187834F8204048F68F70044044F47A
:1045F000004454F0C00410681D7820F82540146869
:10460000187834F820004BF68F74044048F280008C
:10461000044316681D7826F8254015681C7835F87F
:10462000244048F6BF752540284315681C7825F8B6
:10463000240052E01468187834F8200040040ED5A5
:104640001468187834F8204048F68F70044044F419
:10465000404454F080041568187825F82040146808
:10466000187814F8200040060ED51468187834F82D
:10467000204048F68F70044044F4004454F0C004D5
:1046800010681D7820F8254010681C7830F8244008
:1046900048F68F70044044F4404454F0800410689D
:1046A0001D7820F825401468187834F8200048F662
:1046B000BF74044048F28000044315681E7825F852
:1046C000264015681C7835F824404BF68F75254038
:1046D000284315681C7825F82400002082F8E8019A
:1046E000002070BC7047F0B404000D00EDB215F06E
:1046F0007F051C20454304EB050010F584752A61F5
:104700006B610020A8610020687011F07F002870A4
:10471000EE686869864204D2EE686869801B686149
:1047200002E06E6900206861A87A00281FD1206825
:10473000B0F85030287813EBC003206810EB43002A
:1047400000F20C403F2E0AD333005B0916F01F0F16
:1047500000D15B1E9B0253F4004303806BE03700E3
:104760007F08F30700D57F1CBF02078063E06878ED
:1047700000281FD12068B0F85030287813EBC00310
:10478000206810EB430000F204403F2E0AD33300B0
:104790005B0916F01F0F00D15B1E9B0253F4004310
:1047A000038016E037007F08F30700D57F1CBF02A7
:1047B00007800EE0687801280BD12068B0F850001F
:1047C0002B7810EBC300236813EB400303F2044380
:1047D0001E80687800281FD12068B0F850302878F3
:1047E00013EBC003206810EB430000F20C403F2E97
:1047F0000AD333005B0916F01F0F00D15B1E9B022A
:1048000053F40043038016E037007F08F30700D518
:104810007F1CBF0207800EE0687801280BD120685A
:10482000B0F850002B7810EBC300236813EB400363
:1048300003F20C431E802368287833F820304BF6AF
:104840008F70184090F4805090F4005040F4004075
:1048500050F0800027682B7827F823000020F0BC58
:104860007047C9B211F07F011C2251430844D0F8AF
:10487000200180B270472DE9F84381460C001500F5
:1048800000262100C9B211F07F011C20414309EB31
:10489000010010F128073D617B610020B861012013
:1048A000787014F07F003870F8687969884206D211
:1048B000D7F80C807869B0EB0800786103E0D7F88E
:1048C000148000207861B87A002817D143469BB243
:1048D000BA883969D9F80000FFF79BFAD9F80000C7
:1048E000B0F85000397810EBC100D9F8001011EB86
:1048F000400101F20441A1F80080AFE0D9F80010B6
:10490000387811F8200040063BD57878002823D16C
:10491000D9F80000B0F85010387811EBC001D9F880
:10492000000010EB410000F20C40B8F13F0F0AD339
:104930004146490918F01F0F00D1491E890251F460
:10494000004101801AE0414649085FEAC87200D57B
:10495000491C8902018011E0787801280ED1D9F82C
:104960000000B0F85000397810EBC100D9F8001001
:1049700011EB400101F20C41A1F8008038890600DA
:104980003AE07878002823D1D9F80000B0F8501028
:10499000387811EBC001D9F8000010EB410000F2AB
:1049A0000440B8F13F0F0AD34146490918F01F0FE0
:1049B00000D1491E890251F4004101801AE04146AC
:1049C00049085FEAC87200D5491C8902018011E0DC
:1049D000787801280ED1D9F80000B0F85000397865
:1049E00010EBC100D9F8001011EB400101F20441B5
:1049F000A1F80080F888060043469BB2320092B2CC
:104A00003969D9F80000FFF704FA7878002811D145
:104A1000D9F80010387831F8201048F68F7001402E
:104A200041F4004151F0C001D9F80020387822F853
:104A3000201013E07878012810D1D9F800103878C8
:104A400031F8201048F68F70014041F4404151F098
:104A50008001D9F80020387822F82010D9F8001009
:104A6000387831F8201048F6BF70084090F01000F8
:104A700090F0200040F4004050F08000D9F8001081
:104A80003A7821F822000020BDE8F28330B4020019
:104A900092F8E801012801D1022061E0012082F8AA
:104AA000E80108060AD50B00DBB213F07F031C20D7
:104AB000434302EB030010F1280307E00B00DBB2D5
:104AC0001C20434302EB030010F58473012098700F
:104AD00011F07F0018700800C0B2C0095870187833
:104AE000002813D11468187834F820404BF6BF70B2
:104AF000204090F4805090F0100040F4004050F0BE
:104B0000800015681C7825F8240025E058780028D6
:104B100011D010681C7830F8244048F6BF7020404F
:104B200090F0100040F4004050F0800015681C78B0
:104B300025F8240010E01468187834F820404BF66B
:104B40008F70204090F4805040F4004050F080007E
:104B500015681C7825F82400002082F8E801002060
:104B600030BC704730B4020008060AD50B00DBB237
:104B700013F07F031C20434302EB030010F12803D2
:104B800007E00B00DBB21C20434302EB030010F5EF
:104B900084730020987011F07F0018700800C0B274
:104BA000C009587092F8E801012801D102205BE0A9
:104BB000012082F8E8015878002829D01468187874
:104BC00014F8200040060ED51468187834F82040F8
:104BD00048F68F70044044F4004454F0C004156853
:104BE000187825F82040D878012839D0146818782A
:104BF00034F8204048F6BF70204090F0200040F488
:104C0000004050F0800015681C7825F8240027E04B
:104C10001468187834F8200040040ED51468187809
:104C200034F8204048F68F70044044F4404454F077
:104C300080041568187825F8204010681C7830F832
:104C400024404BF68F70204090F4805090F4005038
:104C500040F4004050F0800015681C7825F82400CE
:104C6000002082F8E801002030BC704730B4020018
:104C700092F8E801012801D102204FE0012082F8DA
:104C8000E80108060AD50B00DBB213F07F031C20F5
:104C9000434302EB030010F1280307E00B00DBB2F3
:104CA0001C20434302EB030010F58473002098702E
:104CB00011F07F0018700800C0B2C0095870187851
:104CC000002801D1012029E05878002811D014686B
:104CD000187834F8204048F6BF70204090F020004B
:104CE00040F4004050F0800015681C7825F824003E
:104CF00010E01468187834F820404BF68F7020408C
:104D000090F4005040F4004050F0800015681C788A
:104D100025F82400002082F8E801002030BC70470C
:104D200030B585B004002168DFF8CC05814226D17A
:104D3000DFF8C815086850F400000860086810F42F
:104D400000000090009800220221142000F07DFB5A
:104D5000142000F08FFB142100226D462800FDF77F
:104D600073F84FF4C0500090002001900020029092
:104D7000032003906946DFF8880500F0A7FB05B023
:104D800030BD10B504002168DFF86C05814208D100
:104D9000DFF86815086830F400000860142000F09F
:104DA00070FB10BD10B5040014F5F671D4F81C02A8
:104DB00000F02DFD10BD38B504000D002900C9B26A
:104DC0001C20414304EB0100D0F818212900C9B28E
:104DD000D4F81C0200F07FFD31BD38B504000D0091
:104DE0002900C9B21C20414304EB0100826B290059
:104DF000C9B2D4F81C0200F034FE31BD10B5040075
:104E0000D4F81C0200F037FF10BD10B504000121DA
:104E1000D4F81C0200F01AFFD4F81C0200F0F0FED7
:104E200010BD10B50400D4F81C0200F013FFA069F7
:104E3000002805D0DFF8CC14086850F006000860A0
:104E400010BD10B50400D4F81C0200F00DFF10BD19
:104E500010B50400DFF8B004C0F81C42C4F81C020E
:104E6000DFF8941401600821416002218160032170
:104E7000C160022101610021816100210162FEF710
:104E8000E0FC002801D001F023F84FF4C0730022A9
:104E90000021D4F81C0201F076F84FF4E0730022F0
:104EA0008021D4F81C0201F06EF8002010BD70B50E
:104EB000040000250026D4F81C02FEF745FD010081
:104EC0000800C0B2002805D0022807D004D3032868
:104ED00006D007E0002006E0022004E0012002E006
:104EE000022000E00220C0B270BD70B504000025B1
:104EF0000026D4F81C02FEF73BFD01000800C0B2FA
:104F0000002805D0022807D004D3032806D007E0E4
:104F1000002006E0022004E0012002E0022000E080
:104F20000220C0B270BD70B5040000250026D4F880
:104F30001C02FEF725FD01000800C0B2002805D0C4
:104F4000022807D004D3032806D007E0002006E09B
:104F5000022004E0012002E0022000E00220C0B2B2
:104F600070BD2DE9F84304000D0016001F005FF02E
:104F700000095FF000083300DBB23A0092B229006A
:104F8000C9B2D4F81C02FFF755F801000800C0B2FE
:104F9000002805D0022856D053D3032855D056E018
:104FA000280624D52800C0B210F07F00000104EBD1
:104FB0000002380080B210622800C0B210F07F00FA
:104FC000000104EB00020020D0612800C0B210F004
:104FD0007F0000012044002282612800C0B210F04E
:104FE0007F00000104EB00020020506127E0280050
:104FF000C0B210F07F00000104EB0002380080B264
:10500000C2F810012800C0B210F07F00000104EBCC
:1050100000020020C2F80C012800C0B210F07F008E
:10502000000104EB00020020C2F808012800C0B211
:1050300010F07F00000120440022C0F8042100206D
:1050400006E0022004E0012002E0022000E002204D
:10505000C0B2BDE8F283F8B504000D0000260027B9
:105060002900C9B2D4F81C02FFF714FA01000800A5
:10507000C0B2002805D0022807D004D3032806D0E8
:1050800007E0002006E0022004E0012002E0022008
:1050900000E00220C0B2F2BDF8B504000D00002609
:1050A00000272900C9B2D4F81C02FFF7EFFC010069
:1050B0000800C0B2002805D0022807D004D3032876
:1050C00006D007E0002006E0022004E0012002E014
:1050D000022000E00220C0B2F2BDF8B504000D00CD
:1050E000002600272900C9B2D4F81C02FFF73AFDB8
:1050F00001000800C0B2002805D0022807D004D360
:10510000032806D007E0002006E0022004E001208A
:1051100002E0022000E00220C0B2F2BDF8B50400B7
:105120000D00002600272900C9B2D4F81C02FFF7A1
:105130009DFD01000800C0B2002805D0022807D05C
:1051400004D3032806D007E0002006E0022004E094
:10515000012002E0022000E00220C0B2F2BD020005
:10516000D2F81C32080609D5C9B211F07F011C2003
:10517000414303EB010090F82A0008E0C9B211F0A6
:105180007F011C20414303EB010090F80A017047A6
:10519000F8B504000D00002600272900C9B2D4F894
:1051A0001C02FEF72DFF01000800C0B2002805D048
:1051B000022807D004D3032806D007E0002006E029
:1051C000022004E0012002E0022000E00220C0B240
:1051D000F2BD2DE9F84304000D0016001F005FF03A
:1051E00000095FF000083B009BB232002900C9B201
:1051F000D4F81C02FFF73FFB01000800C0B20028F2
:1052000005D0022807D004D3032806D007E00020E9
:1052100006E0022004E0012002E0022000E002207B
:10522000C0B2BDE8F2832DE9F84304000D0016007A
:105230001F005FF000095FF000083B009BB23200E6
:105240002900C9B2D4F81C02FFF74DFA010008008A
:10525000C0B2002805D0022807D004D3032806D006
:1052600007E0002006E0022004E0012002E0022026
:1052700000E00220C0B2BDE8F28338B505000C00A2
:105280002100C9B2D5F81C02FFF7EBFA32BD38B5E0
:1052900004000D000020ADF800006A462900C9B2E4
:1052A000D4F81C0200F0BAFF002802D1BDF80000BB
:1052B00001E05FF0FF3032BD0100144A1078002891
:1052C00001D0002002E00120107011487047002238
:1052D0000E490A7070470A00D2B2012A05D10D4B5F
:1052E0001A6852F001021A6004E00A4B1A68520868
:1052F00052001A6070470000005C004024380240F1
:105300000000024010ED00E074340020393B002022
:10531000700900200400014038B50500D5F81C4292
:10532000200000F058FE002801D1002000E00220FB
:1053300032BD040110B410F007025A4B1C684FF63E
:10534000FF010C4054EA022457490C431C6010BC76
:10535000704754480068C0F302207047012210F0E3
:105360001F018A40514B010049B2490943F82120ED
:105370007047012210F01F018A404D4B010049B2D5
:10538000490943F82120704710B4020052B2002AA4
:1053900009D50A01474C03005BB213F00F03234405
:1053A00003F8042C04E00C01434B020052B29C545D
:1053B00010BC704770B4030013F00704D4F1070069
:1053C000052801D3042001E0D4F10700251D072D95
:1053D00001D2002600E0E61E012515FA00F0401E6D
:1053E0000140B14015FA06F6761E3240114308001E
:1053F00070BC7047BFF34F8F2A4A116811F4E06107
:105400002E4801431160BFF34F8F00BFFDE710B579
:105410000400601EB0F1807F01D301200EE0611E08
:10542000274801600F215FF0FF30FFF7ADFF00213B
:1054300024480160072124480160002010BD10B5F8
:1054400004002000FFF776FF10BD2DE9F0418046F3
:105450000C0015000026FFF77CFF07002A00210042
:105460003800FFF7A7FF0100404640B2FFF78CFF6E
:10547000BDE8F08110B50400200040B2FFF76EFFD8
:1054800010BD10B50400200040B2FFF772FF10BD40
:1054900080B5FFF7AFFF01BD10B504002000FFF796
:1054A000B6FF10BD0CED00E00000FA0500E100E0E1
:1054B00080E100E018ED00E000E400E00400FA05FF
:1054C00014E000E018E000E010E000E0F8B50200B1
:1054D0000B000024002000251968E140002900F09D
:1054E000DB8001261F6816FA04F10F4038000028FF
:1054F00000F0D0805968022902D0596812291ED1C3
:105500002100C90802EB81010F6A5FF00F0C14F053
:105510000701C9B289001CFA01FC37EA0C07D3F86D
:1055200010C014F00701C9B289001CFA01FC5CEA42
:1055300007073D002100C90802EB81010D621768D1
:105540005FF0030C2100C9B249001CFA01F18F433E
:1055500093F804E01EF0030E2100C9B249001EFAC0
:1055600001FE5EEA070717605968012908D05968EB
:10557000022905D05968112902D0596812291AD177
:1055800095682100C9B249001CFA01F18D43D3F896
:105590000CE02100C9B249001EFA01FE5EEA0505D1
:1055A00095605168A640B1435E68C6F30016A640F8
:1055B00031430F005760D6682100C9B249001CFA78
:1055C00001FC36EA0C069D682100C9B249008D40F5
:1055D0003543D5605968C9005CD544490E6856F01A
:1055E00001060E60096811F0010100910099404E1A
:1055F0002100890856F821705FF00F0C14F00301A8
:10560000C9B289001CFA01FC37EA0C0739498A4201
:1056100001D1002514E038498A4201D101250FE06B
:1056200036498A4201D102250AE035498A4201D130
:10563000032505E033498A4201D1042500E0052510
:1056400014F00301C9B289008D402F43210089085D
:1056500046F821702C4D296881435E68F60300D519
:1056600001432960294E356885435F68BF0300D533
:105670000543356026490E6886435F68FF0200D502
:1056800006430E6023490D6885435F68BF0200D55D
:1056900005430D60641C1FE7F1BD0200136908009B
:1056A00080B2034201D0012000E00020C0B2704768
:1056B0001300DBB2002B03D00B009BB2836103E02D
:1056C0000B009BB21B048361704710B504001248A5
:1056D0000268210089B20A4206D0210089B2016025
:1056E000200080B200F0C4FD10BD00002038024050
:1056F000080001400000024000040240000802408F
:10570000000C02400010024000040140040401406B
:10571000080401400C0401401404014070B5040069
:105720000D001600002C01D102200EE0D4F810026A
:10573000002802D00020C4F81002012084F8FC01E7
:1057400026702000FFF784FB002070BD10B5040018
:10575000012084F8FC016168C9B22000D4F810224D
:10576000526890472000FFF7DEFB2000FFF79FFB09
:10577000002010BD03000022002903D0C3F810123E
:10578000002000E00220C0B2704710B504002000E5
:10579000FFF7ABFB002010BD10B504006168C9B273
:1057A0002000D4F81022526890472000FFF7BBFB7E
:1057B000002010BD01000020704770B504000D00EE
:1057C0000226D4F81002002812D02900C9B2200005
:1057D000D4F8102212689047002802D10020060059
:1057E00006E02900C9B22000D4F810225268904780
:1057F0003000C0B270BD38B504000D002900C9B238
:105800002000D4F8102252689047002032BDF8B52D
:1058100004000D00290014F5027001F0CDF80027F6
:105820000120C4F8F401B4F80E02C4F8F80194F8A9
:10583000080210F01F00002803D0022821D010D346
:105840002FE014F50271200000F01CFD060030006E
:10585000C0B2002804D014F50271200001F0C0F895
:1058600027E014F50271200000F05EFD0600300014
:10587000C0B2002804D014F50271200001F0B0F885
:1058800017E014F50271200000F074FD06003000EE
:10589000C0B2002804D014F50271200001F0A0F875
:1058A00007E0022694F8081211F080012000FFF7AB
:1058B000F3FB3000C0B200280AD0D4F81002806890
:1058C000002805D000212000D4F8102292689047CB
:1058D0003000C0B2F2BD2DE9F84F81460C00150032
:1058E00000275FF000082000C0B200286FD119F532
:1058F00082700600D9F8F401032840F09880F1681E
:10590000B068814242D200200090D9F8100240696C
:1059100000280AD099F8FC01032806D169464846B8
:10592000D9F8102252699047804699F8080210F081
:10593000600F14D04046C0B200280AD10098002859
:1059400003D1F0684042054409E000984042054414
:1059500005E04046C0B2032801D100208046B1686E
:10596000F068091AB1604046C0B200285FD1B16842
:10597000F068814201D2B26800E0F26892B2290078
:10598000484601F0D7F80020070050E099F80802D7
:1059900010F0600F0FD0D9F81002406900280AD02B
:1059A00099F8FC01032806D100214846D9F81022B5
:1059B0005269904780460020B0604046C0B200283F
:1059C00035D1484601F0ECF8002007002FE0D9F867
:1059D0001002C06900282AD099F8FC01032826D1BA
:1059E0002000C0B210F07F000001484410F5827022
:1059F00006002100C9B24846FFF73FFC83465FF02E
:105A0000000A7068834506D27068B0EB0B00B06086
:105A10000120824601E00020B0605246D2B221004F
:105A2000C9B24846D9F81032DB6998478046380039
:105A3000C0B2002803D14046C0B2002806D02100E1
:105A4000C9B24846D9F81022926890474046C0B281
:105A5000002802D04046C0B201E03800C0B2BDE824
:105A6000F28F2DE9F84381460C00150000275FF006
:105A700000082000C0B2002840F0978019F11400FF
:105A80000600D9F8F401022840F08480F168B0687B
:105A900081423FD2B168F068091AB16099F80802F2
:105AA00010F0600F2BD0D9F810020069002822D026
:105AB00099F8FC0103281ED1002000906946484651
:105AC000D9F810221269904780464046C0B200289B
:105AD0000AD10098002803D1F068404205440EE046
:105AE0000098404205440AE04046C0B2032806D16F
:105AF0000020804603E00220070002208046404646
:105B0000C0B2002846D1B26892B22900484600F0DF
:105B1000B0FF3FE07068F268B0FBF2F102FB1100E9
:105B2000002819D17068F168884215D37168D9F8D6
:105B3000F801814210D200220021484600F099FF6E
:105B40000020C9F8F8010023002200214846FFF791
:105B50006AFB002007001DE00020B06099F80802F1
:105B600010F0600F0FD0D9F81002006900280AD099
:105B700099F8FC01032806D100214846D9F81022E3
:105B80001269904780464046C0B2002802D148467C
:105B900001F012F899F80002012817D14846FFF7E2
:105BA00009FE002089F8000210E0D9F8100280698F
:105BB00000280BD099F8FC01032807D12100C9B2B5
:105BC0004846D9F810229269904780463800C0B202
:105BD000002803D14046C0B2002806D02100C9B237
:105BE0004846D9F81022926890474046C0B2002833
:105BF00002D04046C0B201E03800C0B2BDE8F28336
:105C000010B504004023002200212000FFF7A9F96D
:105C10004020C4F810014023002280212000FFF71B
:105C2000A0F9402020622000FFF776FB012084F8D5
:105C3000FC01D4F81402002806D06168C9B2200023
:105C4000D4F8102252689047002010BD0200117451
:105C500000207047010091F8FC0181F8FD0104204B
:105C600081F8FC0100207047010091F8FD0181F8E6
:105C7000FC010020704710B5040094F8FC010328D3
:105C800009D1D4F81002006A002804D02000D4F80A
:105C90001012096A8847002010BD020080B500F08C
:105CA000C9FF01217A48017000F0C8FF01BD08B4A6
:105CB0002DE9F84180460C00150000F0BBFF07AE4F
:105CC00033002A002100404600F0BCFF070000F02E
:105CD000B5FF3800BDE8F2015DF808FB2DE9F041A1
:105CE0006C48202807D04FF4B2726B496B48FCF720
:105CF0003FF8AFF300806A48016851F480210160E9
:105D0000016851F400310160016851F48031016093
:105D100000F0B6FF00F0C0FF624C206880474FF4EF
:105D2000FA7000F0DEF860480068804700202169C2
:105D300088475E4E30688047022001F070F800F01E
:105D400079FF00F061F85A4C012020705948006832
:105D50004FF47A71B0FBF1F00121B0FBF1F0FFF7E5
:105D60009BFB002200215FF0FF30FFF76EFB00F08D
:105D700065FF514D2868804701F044FA4F4F0120DC
:105D8000387038784E490968496A8847387802F08F
:105D900097FC2078316988470120B169884700263F
:105DA0000027012208214748FFF782FC20780028BD
:105DB00001D002F049FE00F03DFFDFF8D48098F8F2
:105DC0000000002807D00120070002F079FE06003D
:105DD000002088F8000000F031FF3800C0B2002831
:105DE000E4D002F06DFE801B40F2E9318842DDD341
:105DF00000F020FF0120E969884702F08BFCFFF7E3
:105E000047FB00F01BFFFEE710B592B034210022E3
:105E100005AC2000FCF718F8142100226C46200085
:105E2000FCF712F8284A0120116860F3CC211160B8
:105E3000012005900120069002200E905FF4803032
:105E40000F905FF4002010905FF40000119005A8FF
:105E500002F03CFE002801D000F03AF80F2000903C
:105E60000320019000200290002003900020049065
:105E70001649086830F0020008600121684603F006
:105E800019FA002801D000F023F812B010BD00006C
:105E9000353B0020200000002C8D0108588E0108A1
:105EA00024ED00E018990108F49601083C910108DE
:105EB000343B0020E0070020600500206C09002032
:105EC000280700200000024000700040003C024013
:105ED000704710B504000A2000FB04F000F009F838
:105EE00010BD10B50400642000FB04F000F001F8C0
:105EF00010BD38B5050003F06DFB0400240D641CD3
:105F0000052C04DA2100280000F016F811E0092C15
:105F100004DA2100280000F018F80AE0112C04DA55
:105F20002100280000F01BF803E02100280000F009
:105F300020F831BD0000000000FB01F34A189A422E
:105F400002DA00BF521CFAE7704700FB01F39B1016
:105F5000020052109A4201DA5B1EF9E7704700FB1B
:105F600001F39B10020052109A4201DA5B1EF9E71E
:105F7000704700FB01F39B10020052109A4201DAB5
:105F80005B1EF9E7704730B4040008060AD50D001F
:105F9000ADB215F07F051C20454304EB050010F160
:105FA000280507E00D00ADB21C20454304EB0500B9
:105FB00010F58475100080B2002803D10020A8726B
:105FC000AB8005E00120A872EB801800000C28814E
:105FD000002030BC70472DE9F047020000234FF449
:105FE00000740825082600271068B0F85000002823
:105FF00001D0012010E101200100C9B2A94216D24E
:10600000D2F800C00100C9B21CF8211011F0300F05
:1060100001D07F1C09E0D2F800C00100C9B23CF8F1
:10602000211011F4405F00D07F1C401CE4E7B8460B
:106030005FFA88F818F1010808FB06F8A2F80C814D
:10604000A2F80E41A2F81041002082F81201106857
:10605000B0F85000116811EB400111F58161B2F800
:106060000CC14FF6FE7010EA0C0CA1F800C0D2F87B
:10607000140110EB0808A2F82C80D48514860020A7
:1060800082F832001068B0F85000116811EB40013E
:1060900011F58061B2F82CC04FF6FE7010EA0C0CBE
:1060A000A1F800C0506B10EB08085FF001094846EA
:1060B000C0B2082880F2AE803800C0B2002800F0DC
:1060C000A9805FF0000E5FF0000C6046C0B20228AD
:1060D00080F2988000206146C9B2002913D1D2F81D
:1060E00000A04946C9B23AF8211011F4405F0AD025
:1060F000CA465FFA8AFA1C2101FB0AFA02EB0A017E
:1061000011F5847108006146C9B2002912D01168E6
:10611000CA465FFA8AFA11F82A1011F0300F09D036
:10612000CA465FFA8AFA1C2101FB0AFA02EB0A014D
:1061300028310800002862D001218E46817A00298A
:1061400016D1C2461FFA8AFAC16811EB0A0AA245A3
:1061500006D3A0F80480C480048101210B0022E052
:10616000A0F80480C4800481C16811EB08081AE01B
:10617000C2461FFA8AFAC1681AEB410AA24506D341
:10618000A0F80480C480048101210B000BE084800E
:10619000A0F80680C16811EB080841460181D0F8DB
:1061A0000C8018EB01084178002914D01168B1F86F
:1061B00050A04946C9B21AEBC10A116811EB4A0155
:1061C00011F58061B0F804A04FF6FE7010EA0A0ADB
:1061D000A1F800A013E01168B1F850A04946C9B277
:1061E0001AEBC10A116811EB4A0111F58161B0F88F
:1061F00004A04FF6FE7010EA0A0AA1F800A01CF1F4
:10620000010C62E77046C0B2002800D07F1E19F171
:1062100001094CE71800C0B2BDE8F08710B40300D4
:10622000080601D4012021E01C680800C0B210F06B
:106230007F0014F8200010F03000302815D1002A1B
:1062400011D01868B0F850000C00E4B214F07F04CC
:1062500010EBC4001C6814EB400404F204442088D2
:106260008005800D1080002000E0022010BC7047E7
:1062700010B50400200080B2B0F5005F01D103F03A
:1062800013FA10BD70B504000D00002668782128AF
:1062900005D12900200000F034F9C0B243E028788D
:1062A00010F06000402805D12900200000F062F8BD
:1062B000C0B238E06878002824D001282CD0032808
:1062C00025D005280DD0062806D0082813D0092887
:1062D0000CD00A2814D024E02900200000F062F934
:1062E00020E02900200000F058FA1BE029002000DF
:1062F00000F083FA16E02900200000F0DFFA11E038
:1063000002200FE02900200000F0FDFA0AE0290039
:10631000200000F017FB05E02900200000F02BFB17
:1063200000E00220C0B270BDF8B504000D000027E7
:1063300094F8FC01032819D12879022814DA2900DD
:106340002000D4F81022D268904706003000C0B276
:10635000002806D1E888002807D1200000F020FCA2
:1063600003E00220060000E0022600E002263000E2
:10637000C0B2F2BD2DE9F04104000D000026AF8847
:10638000287810F06000C0B2202801D0402807D142
:1063900029002000D4F81022D2689047C0B2AEE0A5
:1063A000687800286DD0012839D0032840F0A380F8
:1063B00094F8FC01022802D003280ED02CE038000B
:1063C000C0B2002808D03800C0B2802804D03900FC
:1063D000C9B22000FEF760FE20E0688800280CD1DA
:1063E0003800C0B2002808D03800C0B2802804D0DD
:1063F0003900C9B22000FEF74FFE29002000D4F872
:106400001022D268904706003000C0B2002802D1A6
:10641000200000F0C5FB01E0022006006DE094F8CA
:10642000FC01022802D003280ED027E03800C0B2B9
:10643000002808D03800C0B2802804D03900C9B282
:106440002000FEF729FE1BE06888002815D117F010
:106450007F0F0BD03900C9B22000FEF73EFE2900A5
:106460002000D4F81022D268904706003000C0B255
:10647000002802D1200000F093FB01E0022006007A
:106480003BE094F8FC01022802D0032809D02FE059
:1064900017F07F0F04D03900C9B22000FEF7FCFDD1
:1064A00028E0380608D53800C0B210F07F0000019F
:1064B000204410F1140807E03800C0B210F07F004B
:1064C0000001204410F582783900C9B22000FEF79F
:1064D00046FE002803D00120C8F8000002E000209A
:1064E000C8F8000002224146200000F085FA01E0D1
:1064F0000220060001E0022006003000C0B2BDE824
:10650000F081F8B507000C0000250026A0880428BB
:1065100002D0052814D026E0D7F81002406A406A5D
:1065200000280AD06946387CD7F81022526A526A8D
:10653000904705000020060001E00220060012E05E
:10654000D7F81002406A806A00280AD06946387C71
:10655000D7F81022526A926A904705000020060080
:1065600001E0022006003000C0B2022817D0BDF8BA
:106570000000002811D0E08800280ED0BDF80010DF
:10658000E088814202D3E088ADF80000BDF8002029
:106590002900380000F030FA01E002200600300047
:1065A000C0B2F2BD2DE9FC4107000C000025002619
:1065B000608880B2000AC0B2012805D0C0F0CB804C
:1065C000032829D014D3C6E0D7F81002406A006827
:1065D00000280AD06946387CD7F81022526A12681F
:1065E000904705005FF0000801E05FF00208B4E0AA
:1065F000D7F81002406AC06900280AD06946387C82
:10660000D7F81022526AD269904705005FF000085F
:1066100001E05FF00208A0E0A07800280CD001287B
:106620001ED0022830D0032842D0042854D0052898
:1066300066D0EE2878D08BE0D7F81002406A406828
:1066400000280AD06946387CD7F81022526A52686E
:10665000904705005FF0000801E05FF0020879E074
:10666000D7F81002406A806800280AD06946387C52
:10667000D7F81022526A9268904705005FF0000830
:1066800001E05FF0020865E0D7F81002406AC068D8
:1066900000280AD06946387CD7F81022526AD2689E
:1066A000904705005FF0000801E05FF0020851E04C
:1066B000D7F81002406A006900280AD06946387C81
:1066C000D7F81022526A1269904705005FF000085F
:1066D00001E05FF002083DE0D7F81002406A40692F
:1066E00000280AD06946387CD7F81022526A5269CD
:1066F000904705005FF0000801E05FF0020829E024
:10670000D7F81002406A806900280AD06946387CB0
:10671000D7F81022526A9269904705005FF000088E
:1067200001E05FF0020815E0D7F81002406A006A45
:1067300000280AD06946387CD7F81022526A126ABB
:10674000904705005FF0000801E05FF0020801E0FB
:106750005FF0020801E05FF002084046C0B2022884
:1067600017D0BDF80000002811D0E08800280ED016
:10677000BDF80010E088814202D3E088ADF8000047
:10678000BDF800202900380000F036F901E00220B1
:1067900080464046C0B2BDE8F681F8B504000D0061
:1067A0000027A888002823D1E888002820D1A878CD
:1067B00010F07F00060094F8FC01032802D10220AB
:1067C000070017E084F8FE613100C9B22000FEF72F
:1067D000DFFC200000F0E4F93000C0B2002803D054
:1067E000022084F8FC0105E0012084F8FC0101E0AE
:1067F000022007003800C0B2F2BDF8B504000D0059
:1068000000262D4F688838703878022802DB022075
:1068100006004DE094F8FC01022802D0032819D0AC
:1068200044E03878002811D038786060032084F87C
:10683000FC0139782000FEF7C0FF06003000C0B22E
:10684000002806D1200000F0ABF902E0200000F0A3
:10685000A7F92DE0387800280CD1022084F8FC013B
:106860003878606039782000FEF7C5FF200000F01E
:1068700097F91AE039786068814213D06168C9B22B
:106880002000FEF7B8FF3878606039782000FEF706
:1068900094FF06003000C0B2002806D1200000F0AE
:1068A0007FF902E0200000F07BF901E00220060001
:1068B0003000C0B2F2BD00003A3B002070B50400C9
:1068C0000D000026E888012802D00220060017E00B
:1068D00094F8FC01022802D0032809D00EE0002021
:1068E000A060012214F10801200000F085F807E003
:1068F0000122211D200000F07FF801E002200600A7
:106900003000C0B270BD70B504000D00002694F8D0
:10691000FC11891E012910D80120E060D4F804027E
:10692000002803D0E06850F00200E060022214F179
:106930000C01200000F060F801E0022006003000A9
:10694000C0B270BD70B504000D0000266888012833
:106950000CD10120C4F8040229002000D4F8102230
:10696000D2689047200000F01BF901E002200600E9
:106970003000C0B270BD70B504000D00002694F860
:10698000FC11891E012912D8688801280CD1002029
:10699000C4F8040229002000D4F81022D2689047DD
:1069A000200000F0FDF801E00220060001E00220D6
:1069B00006003000C0B270BD0A7802704A7842709A
:1069C0008B78CA7813EB022343800B794A7913EB57
:1069D000022383808B79CA7913EB0223C38070472B
:1069E00038B505000C0080212800FEF755FB00217A
:1069F0002800FEF751FB31BD70B504000D001600F4
:106A00000220C4F8F401300080B2A061300080B2EE
:106A1000E06133009BB22A0000212000FEF7D9FB81
:106A200070BDF8B504000D0017001E003000C0B2A4
:106A3000002801D102201BE03000C0B210F07F001E
:106A4000000104EB0001380080B288613000C0B260
:106A500010F07F00000104EB0001380080B2C86133
:106A60003B009BB22A003100C9B22000FEF7B1FB07
:106A7000F2BD70B506000C0015002B009BB2220081
:106A800000213000FEF7A5FB70BDF8B504000D0035
:106A900016001F003800C0B2002801D1022007E014
:106AA00033009BB22A003900C9B22000FEF791FBE7
:106AB000F2BD70B504000D0016000320C4F8F40107
:106AC000300080B2C4F80801300080B2C4F80C0174
:106AD00033009BB22A0000212000FEF7A4FB70BD0A
:106AE000F8B504000D0017001E003000C0B20028E9
:106AF00001D102201DE03000C0B210F07F00000183
:106B000004EB0001380080B2C1F808013000C0B2C7
:106B100010F07F00000104EB0001380080B2C1F8E2
:106B20000C013B009BB22A003100C9B22000FEF7E5
:106B30007AFBF2BD70B506000C0015002B009BB26D
:106B4000220000213000FEF76EFB70BDF8B5040096
:106B50000D0017001E003000C0B2002801D1022035
:106B60001DE03000C0B210F07F00000104EB000116
:106B7000380080B2C1F808013000C0B210F07F00C8
:106B8000000104EB0001380080B2C1F80C013B00A9
:106B90009BB22A003100C9B22000FEF744FBF2BDCF
:106BA00010B504000420C4F8F401002300220021E1
:106BB0002000FEF70EFB10BD10B504000520C4F840
:106BC000F4010023002200212000FEF72CFB10BD61
:106BD00038B505000C002100C9B22800FEF757FBAC
:106BE00032BD010212490879002807D1EFF3108065
:106BF000086072B60879401C087105E00879FF2822
:106C000002D00879401C08717047094801790229AF
:106C100003DB0179491E017108E00179012905D1E1
:106C20000179491E0171016881F3108870470000E5
:106C3000DC3A002080B5FFF7D5FF01BD80B5FFF736
:106C4000E4FF01BD1CB584B00023039300290EBFEF
:106C500001930190491E02910024009405AB01A903
:106C600006487844163002F02AFD019901B10C70F3
:106C7000002858BF039806B010BD00BF33B2FFFF15
:106C800080B50320FEF7DBFB002003F07BFC03F064
:106C90008DFC002002BD030410B586B01421002233
:106CA0006846FBF7D1F82448016851F004010160FF
:106CB000016811F0040105910599016851F0200166
:106CC0000160016811F0200105910599016851F0FA
:106CD00001010160016811F0010105910599016848
:106CE00051F002010160006810F002000590059863
:106CF0004FF460400090032001900020029069460C
:106D00000E48FEF7E3FB4FF4C050009003200190C3
:106D1000002002900A4C69462000FEF7D7FB40F2A3
:106D20000E70009003200190002002906946200020
:106D3000FEF7CCFB06B010BD1C3802400008024034
:106D40000000024010B50400FFF774FF012010BDE1
:106D500010B50400FFF772FF012010BD10B5DFF879
:106D600034440120207001F0ABFEDFF82C140860E1
:106D70002078002801D1012000E00020C0B2DFF817
:106D80001C148969884710BD10B5DFF808442078C5
:106D9000002815D001F094FEDFF8FC130968401AB2
:106DA0004FF47A71B0FBF1F0002809D00020207078
:106DB000207890F00100C0B2DFF8E01389698847BD
:106DC00010BD80B5DFF8CC1300200870087890F073
:106DD0000100C0B2DFF8C4138969884701BD10B54E
:106DE00004002000C0B2002801D0012200E00022EF
:106DF000D2B20221DFF8A803FEF75AFC10BD10B58D
:106E000004002000C0B2002801D0012200E00022CE
:106E1000D2B20421DFF88803FEF74AFC10BD10B59A
:106E200004002000C0B2002805D0022811D009D3E8
:106E3000032815D01AE00020FFF7E1FF0020FFF73C
:106E4000CEFF13E00120FFF7DAFF0020FFF7C7FFB6
:106E50000CE00020FFF7D3FF0120FFF7C0FF05E0A3
:106E60000120FFF7CCFF0120FFF7B9FF10BD38B5B7
:106E70008AB00020FFF7B3FF0020FFF7C0FF142106
:106E8000002205AC2000FAF7DFFF04200590012066
:106E900006900020079001200890C14C05A9200011
:106EA000FEF714FB142100226D462800FAF7CCFFF0
:106EB0000220009001200190002002900120039008
:106EC00069462000FEF702FB0020FFF798FF002034
:106ED000FFF785FFB34C2000FFF734FF0020A060D0
:106EE0000020206000206060002020730020A0733C
:106EF000002060730020E073002020742000FFF762
:106F000027FFA94D0523A94A2100280003F06DFBA6
:106F1000A74AA849280003F079FB012000F013F8E4
:106F20000FF2E511280003F085FB01200BB030BD06
:106F300010B59D4C200003F091FB002802D02000EA
:106F400003F0ABFB10BDF8B5040001252000C0B272
:106F5000002803D0022830D00AD338E0924803F04A
:106F6000A8FB0020FFF73BFF0020FFF748FF30E0C1
:106F70008C4E3000FFF7E6FE8B4F380003F092FB9B
:106F80000FF2AD11380003F046FB0FF25D2138001F
:106F900003F041FB0FF2C511380003F03CFB1F204A
:106FA000B0600020B0733000FFF7D2FE0020FFF782
:106FB00016FF0020FFF723FF0BE07B4E300003F0AD
:106FC00078FB0FF24511300003F034FB01E00020A4
:106FD00005002800C0B2002805D0FFF72BFE764838
:106FE0000470FFF72BFE2800C0B2F2BD38B50500D3
:106FF0006C4C2000FFF7A6FE217B2800C0B290EA6F
:10700000010F05D0684803F048FB25730020A073EA
:107010002000FFF79DFE31BD38B50500614C200012
:10702000FFF790FEE17B2800C0B290EA010F05D087
:107030005D4803F032FBE5730020A0732000FFF7EA
:1070400087FE31BD38B50500564C2000FFF77AFEAB
:10705000617B2800C0B290EA010F03D0524803F0D0
:107060001CFB65732000FFF773FE31BD38B50500CA
:107070004C4C2000FFF766FE217C2800C0B290EA4D
:10708000010F03D0484803F008FB25742000FFF7E8
:107090005FFE31BD38B58AB0424C2000FFF752FE8A
:1070A000414803F0FFFA2000FFF752FE0020FFF7EF
:1070B00096FE0020FFF7A3FE1421002205AC20005D
:1070C000FAF7C2FE042005900320069000200790E6
:1070D00000200890324C05A92000FEF7F7F9142192
:1070E00000226D462800FAF7AFFE02200090032030
:1070F0000190002002900020039069462000FEF7D6
:10710000E5F901200BB030BD70B506003400002059
:10711000FFF765FE0020FFF772FE234D280003F005
:10712000C1FA0FF29901280003F075FA002070BD32
:1071300038B504002500A87BFFF751FEA87B002886
:1071400001D1012000E00020C0B2FFF758FE00206E
:10715000286032206860012032BD000038B504008C
:107160002500A868002802D0A868401EA860A8686A
:1071700000280AD00C4803F090FAA87B002801D11F
:10718000012000E00020A87302E00220FFF7DBFEF0
:10719000002032BD333B0020FC3A00203C91010826
:1071A00000000240B83A002094360020A43A0020A3
:1071B000516D0008456D0008323B002038B50500D0
:1071C0002C00207C002806D10120FFF718FE0020AB
:1071D000FFF705FE05E00020FFF711FE0120FFF795
:1071E000FEFD002032BD000001000A001368506857
:1071F000834204D21068401C1060002000E001208F
:10720000704705FF80B5DFF8D40B0068D0F8C400E4
:107210008047DFF8CC0B0068D0F8B800804701BD8C
:1072200080B50120DFF8B41B0968D1F8D010884779
:1072300002BD80B50020DFF8A41B0968D1F8D0108A
:10724000884702BD80B5DFF8940B0068D0F8D40001
:10725000804702BD70B505000E0000210020DFF858
:107260007C2B1268D2F8D82090470400002C0DD057
:1072700033002A000A2114F1400000F031F9411CCA
:107280008E4203D300212954401C00E0002070BD31
:1072900010B403000020002B13D0022911D3DFF813
:1072A0003C2B12681468022909D32278002A06D0E0
:1072B00022781A70641C5B1C401C491EF3E70022F4
:1072C0001A7010BC70472DE9F84304000D00002C23
:1072D00001D0002D01D1002018E0DFF8008BD8F894
:1072E0000000806803F0F8F90600B5420BD33700C0
:1072F000D8F80000D0F80890A0463A004946404629
:10730000FAF7E2FD01E0002006003000BDE8F2835C
:1073100001000020704701000800C0B20C2803DA09
:107320000800C0B2002801D1002000E00020704712
:107330002DE9F84195B0DFF8A45AFF212868A0F89C
:10734000141100202968C1F8180100212868C0F82C
:107350001C11002128688160DFF87C4B286844609C
:1073600010275FF000082600424639003000FAF787
:107370006BFDDFF8680B0068B0F8F460300080B295
:1073800000F0FF0003902F200290300080B2C0F385
:10739000032001902E20009033009BB21B0B9BB268
:1073A000DFF8D82B0F212000FEF781FC04A8296804
:1073B000D1F8CC108847002865D0BDF8100000F047
:1073C000ACF80400002C25D0BDF81010286881838B
:1073D000616828688160BDF810102868A0F8141151
:1073E0002868C0F81841E1682868C0F81C11A06836
:1073F00000280FD0A068818828680182A068C18811
:1074000028684182A068008929688882A068C168CC
:1074100028688161DFF8687B092138002A68126BCF
:1074200090472868C7602868D0F810018047002876
:1074300029D16B46DFF8F00BD0E90021C3E9002128
:107440000020082806D26946095C05AA024491700A
:10745000401CF6E70120ADF8140040F69470ADF83A
:107460001E0003F055F907003C2205A9380003F07F
:1074700056F98046CDF850804022002105A82B689F
:10748000D3F80431984716B0BDE8F08138B5040050
:107490000D002900C9B22000C0B2DFF840291268EF
:1074A000D2F8E42090470100002901D1002000E03B
:1074B000012032BD10B5040000210020DFF81C2996
:1074C0001268D2F8D82090470100002906D0002C7D
:1074D00004D0B1F84A002080012000E0002010BD57
:1074E000F0B404000D000026002901D08E4206D21F
:1074F000A05D002801D1350001E0761CF4E70026EC
:1075000000279F4201D2AF4201D3380003E0E05D83
:10751000D0557F1CF5E7F0BC704710B40100002285
:10752000DFF8F40B03689A420DD2DFF8F00B130179
:10753000C45C0B00A4B29BB29C4202D11201104465
:1075400011E0521CECE7002203689A420AD2DFF8ED
:10755000CC3B14011C5DFF2C02D11001184402E049
:10756000521CF1E7002010BC70472DE9FC4F85B09C
:1075700083468A469046109C119D2E005846C0B204
:1075800004280FDA5046C0B20C280BDA4046C0B2CD
:10759000162807DA5046C0B2002803D0002D01D0CB
:1075A000002C05D1002E01D00120F061002065E003
:1075B000DFF828984146C9B25046C0B2D9F8002039
:1075C000526C9047002803D10120F061002055E063
:1075D0004146C9B25046C0B2D9F80020D2F8E420E2
:1075E000904704900498002803D10120F061002006
:1075F00044E0346086F820B086F821A086F8228026
:10760000B460002070600698F060002200215846A7
:10761000C0B2D9F80030D3F8DC3098470700002F0B
:1076200003D0D7F86200002803D10220F0610020C7
:1076300024E0D7F86200029016F11C00019003A824
:107640000090029B4246D2B25146C9B25846C0B2DF
:10765000D9F800C0DCF8ECC0E0470100002901D1F6
:1076600000200BE0BDF80E007083BDF80C003083E5
:107670003161029870610020F061029807B0BDE8A6
:10768000F08FF8B506000C003500002D01D0002C5D
:1076900002D15FF0FF3075E095F82000042817DA7A
:1076A00095F821000C2813DA95F8220016280FDA35
:1076B00095F8210000280BD02868002808D06869B8
:1076C000002805D02869002802D0E868002804D1E5
:1076D0000120E8615FF0FF3054E06969A8688142E9
:1076E00001D26869A86069686869814201D36869E4
:1076F00068606A696968A86841188A4203D2696942
:107700006868091AA960A868002803D069686869D0
:10771000814205D1002020600020E861002031E096
:1077200000272968A868814204D22868A86001203F
:10773000070007E06968A86841186869814201D2BA
:10774000022007000420E861281DDFF89016096870
:10775000D1F8F01088470100002904D100202060F2
:107760007FF001000EE06868081868606B696A685D
:10777000A8688218934203D26A696868121AAA60DC
:1077800021603800F2BD10B5040000220021200065
:10779000C0B2DFF848361B68D3F8DC3098470100E8
:1077A000002901D1002001E0D1F8620010BD38B5F8
:1077B00005000C00002200212800C0B2DFF81C36B2
:1077C0001B68D3F8DC3098470100002901D0002C59
:1077D00001D1002003E0D1F862002080012032BDF9
:1077E0002DE9F04180460C0015001E00002200210A
:1077F0004046C0B2DFF8E4351B68D3F8DC30984768
:107800000700002F05D0002C03D0002D01D0002E42
:1078100001D1002008E02B0022000C213800FFF7E6
:107820005FFE010031600120BDE8F0812DE9F041EB
:1078300080460C0015001E00002200214046C0B208
:10784000DFF898351B68D3F8DC3098470700002F25
:1078500005D0002C03D0002D01D0002E01D1002036
:1078600009E02B0022000A2117F10C00FFF738FE77
:10787000010031600120BDE8F08138B505000C0041
:10788000002200212800C0B2DFF850351B68D3F871
:10789000DC3098470100002901D1002012E0002CC3
:1078A0000FD0B1F9C600012803D1012020700120BA
:1078B00008E0B1F9C600022803D10220207001209F
:1078C00000E0002032BD2DE9F04180460C0015009B
:1078D000002200214046C0B2DFF800351B68D3F813
:1078E000DC3098478446BCF1000F01D100205EE0F7
:1078F000002C08D1BCF9C600012801D1012056E0B6
:10790000BCF9C80053E0BCF9C800854203D3BCF9F8
:10791000C60002280DD0002D03D0BCF9C6000128F6
:1079200007D0BCF9C600012805D0BCF9C600022862
:1079300001D000203BE0BCF9C600012803D1DCF8EF
:107940006200208206E0122000FB05F06044B0F8DF
:10795000CA0020820020002100260027BCF9C62092
:10796000012A04D1DCF85220DCF8563008E012225B
:1079700002FB05F20CEB020EDEF8CC20DEF8D03074
:10798000BCF9C600012804D1DCF85A00DCF85E100E
:1079900008E0122000FB05F00CEB000EDEF8D4002E
:1079A000DEF8D810C4E90023C4E902010120BDE8D3
:1079B000F0812DE9F84380460C0015001E003700C9
:1079C0004046C0B2042805DA002C03D0002E01D0B6
:1079D000002D02D15FF0FF303DE0BC6287F83080BF
:1079E000DFF8FC9317F131014046C0B2D9F800200E
:1079F000126E9047002802D17FF001002BE097F82B
:107A00003100012811D0022812D100220021404665
:107A1000C0B2D9F800305B6E98473884388C0028A3
:107A200002D17FF0010016E005E00120388402E079
:107A30007FF001000FE07D620020F8850020B8850E
:107A40000020388300200021C7E902010020002126
:107A5000C7E904010020BDE8F2832DE9F84F834611
:107A60008A465E46BBF1000F06D0BAF1000F03D084
:107A7000DAF80000002802D15FF0FF30CBE0308C54
:107A800000280DD096F83100002809D096F8300073
:107A9000042805DAB06A002802D0706A002802D1F2
:107AA0005FF0FF30B7E0002400250027F18D308C17
:107AB000814280F0AD802800C0B2002840F0A8804C
:107AC0002800C0B2002840F08880B6F918000028CD
:107AD00052D196F83100012810D0022832D1F28D0F
:107AE00016F1080196F83000BD4B1B685B6E984795
:107AF000012802D07FF001008DE026E0DFF8E0826F
:107B000016F1180196F83000D8F80020526D904711
:107B1000002813D016F1080196F83000D8F800209C
:107B2000126F9047002809D016F1100196F8300026
:107B3000D8F80020526F9047002802D17FF0010052
:107B400069E002E07FF0010065E0D6E90401D6E9D2
:107B50000223FBF7C9FA80468946B6F91800401E91
:107B6000FBF7F2F902000B0040464946FAF7C0FE67
:107B7000C6E900010020B085B6F91800002819D028
:107B8000B08DB6F91810884227DAB08D02F05EFE8B
:107B9000D6E90023FAF79EFDD6E90223FBF7E6F9C2
:107BA000B26A02EBC402C2E90001641C706A84423A
:107BB00007D302E07FF001002DE001200500012045
:107BC0000700DAF80000844203D3012005000220F8
:107BD0000700B08D401CB08572E7B08DB6F9181063
:107BE00088420DDBF08D318C491E884204DBF08D1C
:107BF000401CF08501200500002030830020B08566
:107C00002800C0B2002803D1F08D401CF0854DE75C
:107C1000CAF800403800BDE8F28F2DE9F0410700B6
:107C20000C0015001E00B0463800C0B2042805DA6A
:107C3000002C03D0002E01D0002D02D15FF0FF30C8
:107C400015E0C8F8044088F81070C8F8005000200B
:107C5000A8F80800DFF81C0A40698047A8F80A0065
:107C6000002088F80C00002088F80D000020BDE8F6
:107C7000F0812DE9F84304000D002600002C04D00B
:107C8000002D02D02868002802D15FF0FF3051E0BB
:107C9000307C042805DA7068002802D0306800289B
:107CA00002D15FF0FF3045E000275FF000085FF091
:107CB00000094046C0B200283AD17089002825D07A
:107CC00031897089814206D301208046002070816D
:107CD000002030812CE016F10C013089C0B2DFF8B1
:107CE000942992699047002802D17FF0010021E099
:107CF000317B706800F81710706800EB4701707BEB
:107D000048707F1C3068874207D302E07FF0010093
:107D100010E001208046012081462868874203D375
:107D200001208046022081463089401C3081C0E716
:107D30002F604846BDE8F2832DE9F84381460C00E8
:107D4000002200214846C0B2DFF82C391B68D3F866
:107D5000DC3098470500002D01D0002C01D1002017
:107D600039E0B5F9C600012809D100260027D5F869
:107D70005220D5F85630C4E9002301202BE0B5F994
:107D8000C600022826D1B5F9C800012822DB002050
:107D90000021D5F8CC20D5F8D0305FF00008B5F937
:107DA000C800804512D200260027122000FB08F0F0
:107DB00005EB000CDCF8CC00DCF8D01002F054FD30
:107DC00001D202000B0018F10108E8E7C4E9002322
:107DD000012000E00020BDE8F28300002C07002015
:107DE000280700202DE9F14F8B46002200219DF845
:107DF0000000DFF884381B68D3F8DC3098470600B1
:107E0000002E02D0BBF1000F01D1002044E0B6F9F2
:107E1000C600012809D100220023D6F85A40D6F81E
:107E20005E50CBE90045012036E0B6F9C6000228D5
:107E300031D1B6F9C80001282DDB002000215FF008
:107E4000120AB6F9C8200AFB02F23244D2F8C24044
:107E5000D2F8C6500027B6F9C800874217D25FF0A3
:107E600000085FF00009B6F9C800401EC01B0AFBFD
:107E700000F03044D0F8D420D0F8D83020002900C9
:107E800002F0F2FC01D214001D007F1CE3E7CBE9F5
:107E90000045012000E00020BDE8F28FF8B50500A4
:107EA0000C00002200212800C0B2DFF8CC371B688C
:107EB000D3F8DC3098470100002901D0002C01D113
:107EC000002008E000220023D1F86660D1F86A7033
:107ED000C4E900670120F2BDDC050020E8080020AD
:107EE0002DE9F84F83460C0015001E0000220021EA
:107EF0000020DFF884371B68D3F8DC309847070090
:107F0000002F05D0002C03D0002D01D0002E01D170
:107F1000002030E000215FF000085846C0B2002881
:107F200005D0022809D005D3032809D00BE0B7F803
:107F30006E900AE0B7F8709007E0B7F8729004E02E
:107F4000B7F8749001E0002015E0484680B20D2893
:107F500002D3DFF828A705E0DFF82427484680B2DF
:107F600052F820A02B00220000215046FFF7B8FA5B
:107F7000010031600120BDE8F28F0000B49E0108CD
:107F8000FC0500202DE9F0478046894614001D00BD
:107F9000089E002200214046C0B2DFF8DC361B6894
:107FA000D3F8DC3098470700002F05D0002C03D011
:107FB000002D01D0002E01D1002033E05FF0000A37
:107FC0004846C0B2002805D0022815D00BD303289C
:107FD0001BD023E02B002200142117F17600FFF7BD
:107FE0007FFA01001CE02B002200142117F18A0007
:107FF000FFF776FA010013E02B002200142117F19D
:108000009E00FFF76DFA01000AE02B002200142108
:1080100017F1B200FFF764FA010001E0002001E06F
:1080200031600120BDE8F087F8A301082DE9F04197
:1080300080460C0015001E00002200214046C0B200
:10804000DFF834361B68D3F8DC3098470700002F80
:1080500005D0002C03D0002D01D0002E01D100202E
:1080600009E02B002200142117F13E00FFF738FA37
:10807000010031600120BDE8F0812DE9F04180462A
:108080000C0015001E00002200214046C0B2DFF89F
:10809000E8351B68D3F8DC3098470700002F05D07F
:1080A000002C03D0002D01D0002E01D1002009E0CA
:1080B0002B002200142117F11600FFF711FA01001E
:1080C00031600120BDE8F0812DE9F04180460C00CF
:1080D00015001E00002200214046C0B2DFF898358E
:1080E0001B68D3F8DC3098470700002F05D0002C20
:1080F00003D0002D01D0002E01D1002009E02B007B
:108100002200142117F12A00FFF7EAF9010031607B
:108110000120BDE8F081000074A7010890830108E8
:10812000D0B5040000210020DFF84C251268D2F8F9
:10813000E02090470100002901D0002C01D100204F
:1081400008E000220023D1F81660D1F81A70C4E9C3
:1081500000670120D0BDD0B5040000210020DFF869
:1081600018251268D2F8E02090470100002901D0BC
:10817000002C01D1002008E000220023D1F81E606D
:10818000D1F82270C4E900670120D0BD80B500217C
:108190000020DFF8E4241268D2F8E02090470100C4
:1081A000002901D1002001E0D1F8260002BD10B560
:1081B000040000210020DFF8C0241268D2F8E0207B
:1081C00090470100002901D0002C01D1002003E0DC
:1081D000D1F826002080012010BD2DE9F8430500CC
:1081E0000E0017009846DDF820904C46002C02D176
:1081F0005FF0FF300BE0002084F82300009443463A
:108200003A003100C9B22800C0B200F01EF8BDE843
:10821000F2832DE9F84305000E0017009846DDF8BB
:1082200020904C46002C02D15FF0FF300BE0012083
:1082300084F82300009443463A003100C9B2280074
:10824000C0B200F002F8BDE8F2832DE9FE4F83468C
:108250008A4617001C000C9D002D09D140F679328A
:10826000DFF82014DFF82004F9F782FDAFF3008077
:108270005846C0B20C2809DA5046C0B2162805DAB2
:108280005846C0B2002801D0002C03D10120E8617B
:1082900000206FE0DFF8E0835146C9B25846C0B213
:1082A000D8F80020526C9047002803D10120E861E3
:1082B00000205FE02C60002085F8200085F821B0C8
:1082C00085F822A0AC6000206860EF6000210020EB
:1082D000D8F80020D2F8E02090470600002E03D006
:1082E000D6F82600002803D10220E861002041E0F2
:1082F000D6F826900020029095F8230000280FD190
:1083000015F11C00009001AB4A465146C9B25846CF
:10831000C0B2D8F800C0DCF8F4C0E04701000EE0BD
:1083200015F11C00009001AB4A465146C9B25846AF
:10833000C0B2D8F800C0DCF8F8C0E047010000295E
:1083400001D1002016E095F82300002806D1BDF8E1
:1083500006006883BDF80400288305E0BDF8060028
:108360006883BDF8040028832961C5F814900020B3
:10837000E8614846BDE8FE8F70B506000C00350088
:10838000002D05D0002C03D095F82300002802D042
:108390005FF0FF3003E02100280000F015F870BD09
:1083A00070B506000C003500002D05D0002C03D060
:1083B00095F82300002802D15FF0FF3003E0210090
:1083C000280000F001F870BDF8B504000D00002C85
:1083D00007D140F63342AB49AB48F9F7C9FCAFF3DC
:1083E0000080002D07D140F63442A649A748F9F78E
:1083F000BFFCAFF3008094F82000002817D194F858
:1084000021000C2813DA94F8220016280FDA94F8C9
:10841000210000280BD02068002808D060690028BF
:1084200005D02069002802D0E068002804D101208E
:10843000E0615FF0FF3060E06069A168884201D2CE
:108440006069A06061686069814201D360696060B1
:1084500062696168A06841188A4203D261696068F4
:10846000091AA160A068002803D060686169884289
:1084700005D1002028600020E06100203DE00026BA
:108480002068A168884204D22068A060012006000C
:1084900007E06168A06841186069814201D202204A
:1084A00006000420E061002794F82300002807D18B
:1084B000201D71490968D1F8FC108847010006E0C9
:1084C000201D6D490968D1F8001188470100002975
:1084D00004D1002028607FF001000EE060680818D9
:1084E000606063696268A0688218934203D262691F
:1084F0006068121AA26029603000F2BD38B590B0F1
:108500000400002C35D05C4D2868D0F80C01804761
:1085100040282ED14022002168462B68D3F808312C
:108520009847002825D0002020709DF8020055288B
:108530001DD19DF80300532819D19DF8040042284D
:1085400015D19DF80500542811D19DF806004D283D
:108550000DD19DF80700432809D19DF80800212876
:1085600005D19DF80900002801D1012020700120CB
:1085700000E0002011B030BDF8B590B00500280033
:10858000C0B2002803D02800C0B201285CD13A4C08
:108590002068D0F80C018047402855D140220021A6
:1085A00068462368D3F80831984700284CD0280043
:1085B000C0B2012818D155208DF8020053208DF843
:1085C000030042208DF8040054208DF805004D2052
:1085D0008DF8060043208DF8070021208DF8080053
:1085E00000208DF8090017E056208DF80200452084
:1085F0008DF803004E208DF8040044208DF805000E
:108600004F208DF8060052208DF8070021208DF8AC
:10861000080000208DF8090002F07AF806003C22DC
:108620006946300002F07BF807000F9740220021D6
:1086300068462368D3F804319847002801D0012008
:1086400000E00020C0B200E0002011B0F0BD010049
:10865000080080B2012802D0022804D008E00648B1
:108660000068806905E0044800688069801C00E0BB
:1086700000207047F49601082C07002010A4010880
:10868000A88F0108C089010800A40108609C0108A6
:1086900010B50400200080B2FFF7D9FF008810BD9C
:1086A00038B505000C00280080B2FFF7D0FF0100AC
:1086B000002901D1002001E00C80012032BD000022
:1086C00038B504002000C0B2012811D0164D002298
:1086D00016492800FDF722F815492800FDF74AF849
:1086E0001449280002F0AFFC2800FDF74EF810E016
:1086F0000D4D00220D492800FDF710F80E49280005
:10870000FDF738F80D49280002F09DFC2800FDF720
:108710003CF831BD10B5044C2000FDF73DF82000B9
:10872000FDF714F810BD0000543200205C08002052
:10873000009401084490010888930108789001088A
:1087400080687047C06870470200002A05D0002981
:1087500003D090690860012000E00020704702000B
:10876000002A02D09161012000E0002070474FF400
:108770008050704710B5FEF75DFADFF830030478DB
:10878000FEF75CFA2000C0B210BD80B5FFF7F2FF23
:1087900002BD80B5FEF74EFA0021C4480170FEF715
:1087A0004DFA01BD10B50024FEF744FABF49087820
:1087B000002802D1012004000C70FEF73FFA2000CF
:1087C000C0B210BD0020704700207047704770B5E0
:1087D00004000D0016006078022806D0032817D088
:1087E000062828D0072828D02FE0FFF7C3FF00284D
:1087F00001D000202AE0002300220021200000F008
:1088000052F8002801D0012000E00020C0B21DE095
:10881000FFF7B0FF002801D0002017E0002300225E
:108820000021200000F077F8002801D0012000E0AE
:108830000020C0B20AE0012008E061880029012977
:1088400003D8200000F0E7F800E0002070BDF8B584
:1088500004000D0016001F006078032806D13B00BD
:1088600032002900200000F056F800E00020F2BDA0
:10887000F8B504000D0016001F006078022802D031
:10888000062807D00DE03B0032002900200000F050
:108890000AF807E03B0032002900200000F089F8C8
:1088A00000E00020F2BD2DE9F84305000C001600A1
:1088B0001F00B5F8048018EB0608688818EB00481C
:1088C000002C0AD139004046794AD26890470028E6
:1088D00001D0012000E000201BE0200002F005FD97
:1088E000874201D2B94603E0200002F0FEFC814637
:1088F0002000FFF725FF4A46010040466C4B9B686D
:108900009847002804D04946200002F09DFC00E072
:108910000020BDE8F2832DE9F04706000C001500A9
:108920001F00B6F8048018EB0508708818EB0048A3
:10893000002C11D1FFF71BFFF188884201D20020E3
:1089400035E0390040465A4A12699047002801D064
:10895000012000E000202AE0FFF724FF002825D0B6
:10896000200002F033FC874201D2B94603E0200028
:1089700002F02CFC8146002D16D1200002F026FCCE
:10898000B84211D1DFF82CA100222100504602F09C
:10899000BDFC4948C0F8008021005046FFF7DFFECB
:1089A000504602F013FC02E0FFF7F3FE0020BDE8A2
:1089B000F0872DE9F84380460C0015001E002000CA
:1089C00002F093FC864201D2370003E0200002F05F
:1089D0008CFC070002210022E9464846F9F734FAE8
:1089E000FFF7C8FE002803D0A5208DF8000002E0A4
:1089F00000208DF80000022D08D2032E06D232008E
:108A0000684600EB0501200002F04EFB200002F05A
:108A1000DDFBBDE8F28338B504000025608800283E
:108A200002D0012807D00CE024480068D0F8B80034
:108A30008047050005E021480068D0F8BC00804769
:108A400005002800C0B232BDF8B5FFF793FE00283C
:108A50002AD01A4C2068D0F8BC008047154D280059
:108A6000FFF770FE0600280002F0B0FB07003A0096
:108A70003100114800680E4B5B6898470020009059
:108A800069462800FFF760FE002807D00022290071
:108A9000009802F03BFC009802F0DFFAFFF779FE45
:108AA0002068D0F8B8008047F1BD0000383B0020B6
:108AB00060050020703A0020103B002028070020AD
:108AC00001480068704700BF083B00202DE9F843CB
:108AD000050000242878C00740F1AA80DFF8000BC9
:108AE000016811F00C01082907D0016811F00C0190
:108AF0000C2922D10068C0031FD54FF4804002002A
:108B0000B2FA82F1C9B2490951F00101C9B2012991
:108B100003D1DFF8C81A0A6802E0DFF8D41A0A683D
:108B2000B0FA80F111F01F01CA40D10740F18080F6
:108B3000686800287CD10120BAE36868012806D162
:108B4000DFF8981A086850F48030086025E06868FB
:108B500000280AD1DFF8840A016831F4803101600D
:108B6000016831F48021016017E0686805280AD1A6
:108B7000DFF8680A016851F480210160016851F44E
:108B80008031016009E0DFF8540A016831F4803176
:108B90000160016831F4802101606868002823D0F9
:108BA000FFF78EFF04004FF480400200B2FA82F11A
:108BB000C9B2490951F00101C9B2012903D1DFF855
:108BC0001C1A0A6802E0DFF8281A0A68B0FA80F175
:108BD00011F01F01CA40D1072AD4FFF771FF001B13
:108BE0006528E0D3032063E3FFF76AFF04004FF436
:108BF00080400200B2FA82F1C9B2490951F0010184
:108C0000C9B2012903D1DFF8D4190A6802E0DFF8FC
:108C1000E0190A68B0FA80F111F01F01CA40D107CB
:108C200006D5FFF74DFF001B6528E0D303203FE387
:108C30002878800740F1AD80DFF8A409016811F0C1
:108C40000C01042907D0016811F00C010C2930D166
:108C50000068C0032DD45FF080400200B2FA82F1B8
:108C6000C9B2490951F00101C9B2012903D1DFF8A4
:108C70006C190A6802E0DFF878190A68B0FA80F126
:108C800011F01F01CA40D10704D5E868012801D0BE
:108C900001200DE3DFF84C0903685FF47801B1FAB5
:108CA00081F233F4F8532E6916FA02F2134303608B
:108CB0006FE0E86800283DD05FF00046B6FA86F223
:108CC0000120D2B2DFF8B81911EB82010860FFF77A
:108CD000F7FE04005FF080400200B2FA82F1C9B2F0
:108CE000490951F00101C9B2012903D1DFF8EC189B
:108CF0000A6802E0DFF8F8180A68B0FA80F111F0AB
:108D00001F01CA40D10706D4FFF7DAFE001B032873
:108D1000E0D30320CCE2DFF8CC6832685FF478005F
:108D2000B0FA80F132F4F8522B6913FA01F10A43D8
:108D300032602EE05FF00046B6FA86F20020D2B232
:108D4000DFF83C1911EB82010860FFF7B9FE04005F
:108D50005FF080400200B2FA82F1C9B2490951F0D5
:108D60000101C9B2012903D1DFF870180A6802E0D5
:108D7000DFF87C180A68B0FA80F111F01F01CA40D0
:108D8000D10706D5FFF79CFE001B0328E0D3032084
:108D90008EE22878C00640F1F780DFF8446830683A
:108DA00010F00C0F7BD15FF480000100B1FA81F26A
:108DB000D2B2520952F00102D2B2012A03D1DFF835
:108DC0001C180A6802E0DFF828180A68B0FA80F177
:108DD00011F01F01CA40D10704D5A869002801D1AC
:108DE000012065E2DFF8FC77396811F46041286AF8
:108DF000814218D2286A00F0FDFB002801D0012032
:108E000056E2396831F46041286A014339603A68B2
:108E1000FF20B0FA80F122F07F42EB6913FA01F1F2
:108E20000A433A6018E0396831F46041286A014326
:108E3000396038684FF0FF08B8FA88F220F07F40B8
:108E4000E96911FA02F210433860286A00F0D2FB97
:108E5000002801D001202BE25FF4E027B7FA87F069
:108E600032685FF07066B6FA86F10123D5F820C04B
:108E70003CFA00FC1CF1010C13FA0CF34FF4004017
:108E80004343DFF8000812F0F002CA40805CC340A0
:108E9000DFF858070360002001F074FB74E0A86954
:108EA000002842D05FF40006B6FA86F00121C0B275
:108EB000DFF8CC2712EB80021160FFF701FE0400FF
:108EC0005FF480010A00B2FA82F0C0B2400950F0AB
:108ED0000100C0B2012803D1DFF80007006802E0FA
:108EE000DFF80C070068B1FA81F212F01F02D040DF
:108EF000C00706D4FFF7E4FD001B0328E0D30320DE
:108F0000D6E1DFF8E0160A6832F46042286A0243CC
:108F10000A600A68FF26B6FA86F022F07F42EB6903
:108F200013FA00F002430A602EE05FF40006B6FA7E
:108F300086F00022C0B2DFF8481711EB80010A600A
:108F4000FFF7BEFD04005FF480010A00B2FA82F070
:108F5000C0B2400950F00100C0B2012803D1DFF8CF
:108F60007C06006802E0DFF888060068B1FA81F24A
:108F700012F01F02D040C00706D5FFF7A1FD001B6D
:108F80000328E0D3032093E1287800074AD56869D5
:108F9000002823D05FF00046B6FA86F00122C0B266
:108FA000DFF8E41611EB80010A60FFF789FD040089
:108FB0005FF080421000B0FA80F1DFF834160968E3
:108FC000B2FA82F313F01F03D940C9072AD4FFF77E
:108FD00077FD001B0328EBD3032069E15FF0004617
:108FE000B6FA86F00022C0B2DFF89C1611EB8001C1
:108FF0000A60FFF765FD04005FF080421000B0FAE0
:1090000080F1DFF8EC150968B2FA82F313F01F0360
:10901000D940C90706D5FFF753FD001B0328EBD342
:10902000032045E12878400740F19C800026DFF8C6
:109030005C763868C0000AD4386850F080503860D8
:10904000386810F080500090009801200600DFF88A
:109050004086D8F80000C00513D4D8F8000050F4BA
:109060008070C8F80000FFF72BFD0400D8F800005E
:10907000C00506D4FFF724FD001B6528F6D30320A6
:1090800016E1A868012806D1DFF86415086850F4D5
:109090008070086025E0A86800280AD1DFF8500534
:1090A000016831F480710160016831F48061016010
:1090B00017E0A86805280AD1DFF83405016851F4E3
:1090C00080610160016851F48071016009E0DFF89E
:1090D0002005016831F480710160016831F480611C
:1090E0000160A86800281AD0FFF7EAFC04005FF4CA
:1090F00080021000B0FA80F1DFF8F4140968B2FAC7
:1091000082F313F01F03D940C90723D4FFF7D8FC1B
:10911000001B41F289318842E9D30320C8E0FFF700
:10912000CFFC04005FF480021000B0FA80F1DFF899
:10913000C0140968B2FA82F313F01F03D940C907BB
:1091400008D5FFF7BDFC001B41F289318842E9D305
:109150000320ADE03000C0B2012803D1386830F000
:1091600080503860686A002800F0A180DFF87084C1
:10917000D8F8000010F00C000C2800F09680686A07
:10918000022865D15FF08009B9FA89F1DFF8F0644F
:109190000020C9B216EB81010860FFF791FC0700BF
:1091A0004021B1FA81F0C0B2400950F00100C0B2D4
:1091B000012803D1DFF82404006802E0DFF830045E
:1091C00000684021B1FA81F212F01F02D040C007BE
:1091D00006D5FFF775FCC01B0328E1D3032067E029
:1091E000D8F8001031F47D01A86A0143E86A014310
:1091F000286B0143C8F800105FF08008B8FA88F0C7
:109200000121C0B216EB80063160FFF759FC040063
:109210004021B1FA81F0C0B2400950F00100C0B263
:10922000012803D1DFF8B403006802E0DFF8C003CF
:1092300000684021B1FA81F212F01F02D040C0074D
:1092400035D4FFF73DFC001B0328E1D303202FE0BA
:109250008026B6FA86F00022C0B2DFF8241411EBA3
:1092600080010A60FFF72CFC04004021B1FA81F074
:10927000C0B2400950F00100C0B2012803D1DFF8AC
:109280005C03006802E0DFF8680300684021B1FA7F
:1092900081F212F01F02D040C00708D5FFF710FC82
:1092A000001B0328E1D3032002E0012000E000209E
:1092B000BDE8F2832DE9F04104000D000026DFF83F
:1092C000D473386810F00100A84211D2012D03D1E7
:1092D000386850F00400386038684008400028437F
:1092E0003860386810F00100A84201D0012016E172
:1092F0002078800707D5DFF8E822116831F0F00107
:10930000A068014311602078C00740F1C680606802
:1093100002281BD14FF480400200B2FA82F1C9B298
:10932000490951F00101C9B2012903D1DFF8AC129A
:109330000A6802E0DFF8B8120A68B0FA80F111F0AA
:109340001F01CA40D10757D40120E8E06068032814
:1093500019D14021B1FA81F0C0B2400950F00100AA
:10936000C0B2012802D19D48026802E0DFF8800205
:1093700002684020B0FA80F111F01F01CA40D10705
:109380003AD40120CBE0606801281AD15FF0804018
:109390000100B1FA81F2D2B2520952F00102D2B206
:1093A000012A02D18D490A6802E0DFF844120A68F6
:1093B000B0FA80F111F01F01CA40D1071CD401207E
:1093C000ADE05FF480000100B1FA81F2D2B252093F
:1093D00052F00102D2B2012A02D180490A6802E0A9
:1093E000DFF80C120A68B0FA80F111F01F01CA40D0
:1093F000D10701D4012092E0DFF8E481D8F8001011
:109400008908890060680143C8F80010FFF758FB1D
:109410000600606802280ED1D8F8000010F00C0099
:1094200008283AD0FFF74CFB801B41F28931884273
:10943000F2D3032073E0606803280ED1D8F800004F
:1094400010F00C000C2828D0FFF73AFB801B41F2EB
:1094500089318842F2D3032061E0606801280ED18F
:10946000D8F8000010F00C00042816D0FFF728FBF5
:10947000801B41F289318842F2D303204FE0D8F8B3
:10948000000010F00C0F08D0FFF71AFB801B41F210
:1094900089318842F3D3032041E0386810F001009D
:1094A000854211D2012D03D1386850F00400386094
:1094B00038684008400028433860386810F00100E0
:1094C000A84201D001202AE02078400706D5444A6E
:1094D000116831F4E061E068014311602078000711
:1094E00007D53F4A106830F46050216950EAC10046
:1094F000106000F016F83A490B685FF07067B7FA31
:1095000087F1DFF8802113F0F003CB40D15CC84035
:10951000DFF884110860002001F034F80020BDE875
:10952000F0812DE9F0415FF0000C002100220023C2
:10953000002400262A48056815F00C07042F04D0E3
:10954000082F04D00C2F04D02DE0274840E02648F7
:109550003EE04FF47057B7FA87F8DFF844C115F4CE
:10956000701E3EFA08FE1CF80EC061464FF4407CA7
:10957000BCFA8CF815F4400E3EFA08FE1EF1010EFE
:1095800072460068C00306D5174800FB01F0B0FB27
:10959000F2F0030005E0144800FB01F0B0FBF2F02C
:1095A0000300180014E03F48D0F800C05FF4E02743
:1095B000B7FA87F01CF4604C3CFA00FC64465FF09C
:1095C000010C601C1CFA00FC4FF4004000FB0CF086
:1095D000BDE8F08130480068704700000038024064
:1095E00008380240043802400024F400E00700205C
:1095F0003438024018B401000022002327480068D4
:1096000010F0F00F23D121480468E40005D520486C
:10961000006810F4C050020011E0046854F0805457
:109620000460046814F080540094009C184C246872
:1096300014F4C0542200046834F080540460B2F57D
:10964000C05F04D1B1F5404F01D101200300012BCF
:1096500004D1104C206850F0040020600D4C2068AC
:109660004008400018432060206810F00100984234
:1096700001D0012000E0002012BC70470000000073
:1096800000004742D49F0108800647422438024028
:1096900000700040003C0240E00700200838024013
:1096A000D0A20108043802400249086830F00200E4
:1096B0000860704710ED00E040F0200070472DE991
:1096C000F14FB0B0924604910DF142013A9A2B91BC
:1096D00099464A7000200AE01AF8011B0498309A53
:1096E00090470028049000F043860D98401C0D9090
:1096F0009AF8000050B12528EED1002200210792EF
:10970000089109920A910B920C9104E00D9800F0D7
:1097100031BE41F001011AF8010F2028F9D02328A9
:109720000CD02B2804D02D2805D0302809D00BE0F0
:1097300041F00201EFE741F00401ECE741F00801DC
:10974000E9E741F01001E6E72A280FD1D9F8002017
:1097500052F8040BC9F8002000280F9003D54042AE
:109760000F9041F004010AF1010A14E00F92DFF8B2
:109770000C0C0AE00F9C844205DA04EB840302EB34
:109780004302303A0F920AF1010A9AF80020A2F13E
:1097900030030A2BEED39AF800202E2A03D04FF084
:1097A000FF300E9029E01AF8010F2A2809D1D9F8C4
:1097B000002052F8040BC9F800200E900AF1010AAB
:1097C0001BE02D280CBF0AF1010A002000220E9296
:1097D000DFF8A85B0BE040B90E9BAB4205DA03EB68
:1097E000830402EB4402303A0E920AF1010A9AF81D
:1097F0000020A2F130030A2BEDD3ADF840100FF694
:1098000080309AF8001001F01BFE08B11AF8010B25
:109810008DF842009DF84200682805D19AF80010A2
:1098200068290CD1622006E06C2804BF9AF8001069
:109830006C2904D171208DF842000AF1010A12AAA4
:1098400006921AF801BBBBF125002CD01C3800F0A1
:109850009781001F022840F29381133800F0BA84E8
:10986000093800F08D81801E00F04F85401E00F009
:10987000FC84401E022840F28381001F00F0F58422
:10988000401F00F0F280401E00F0A484401E00F053
:10989000DA80C01E0ED0801E00F09C84C01E00F036
:1098A000998400F03DBD0122252107928DF84810D2
:1098B00000F042BDD9F8000050F8044BC9F8000090
:1098C000002C059440F0AB802B994878002800F0DC
:1098D000A1804FF0FF340FF6B02001F0BDFD241A37
:1098E00040F0468500F028BD01236A4602A93046B3
:1098F00000F00CFE002840F03B85641EF4D1309649
:10990000079C12AE74B1309F16F8011B0498B8473B
:109910000028049000F02C850D98401C641E0D90CA
:10992000F2D130970A9C3021002C8DF800100CDD0C
:10993000309E01236A4602A9304600F0E7FD002868
:1099400040F01685641EF4D13096059E089C74B1D3
:10995000309F16F8011B0498B8470028049000F0C7
:1099600007850D98401C641E0D90F2D130970B9C1A
:109970003021002C8DF800100CDD309E01236A464A
:1099800002A9304600F0C2FD002840F0F184641EB8
:10999000F4D1309605980899099C461874B1309F07
:1099A00016F8011B0498B8470028049000F0E084E2
:1099B0000D98401C641E0D90F2D130970C9C302104
:1099C000002C8DF800100CDD309E01236A4602A9A0
:1099D000304600F09BFD002840F0CA84641EF4D19C
:1099E00030969DF8400041077FF582AE2020002D83
:1099F0008DF800007FF77CAE309C01236A4602A9F7
:109A0000204600F083FD002840F0B2846D1EF4D1A2
:109A100030946DE60FF65430059000F08DBC0E9D2D
:109A2000002D04D5204600F057FE044608E02A46E3
:109A300000212046F9F7B6FD002814BF041B2C4670
:109A4000089400F079BCD9F8001051F8040BC9F85B
:109A5000001020F00002002121F0FF33CDE90223A5
:109A600012AC0594782100F04CBC2B99487820B1B9
:109A70004FF0FF340FF6C4202FE79DF84200622814
:109A800060D0682817D06A283FD06C2806D071288B
:109A900047D074282CD07A281DD062E0D9F8001065
:109AA00051F8040BC9F80010002866D14FF0FF34BC
:109AB0000FF6A02011E7D9F8001051F8040BC9F8EF
:109AC000001020B94FF0FF340FF6882005E70D99FC
:109AD000018000F031BCD9F8001051F8040BC9F82E
:109AE0000010002849D14FF0FF340FF66820F4E64B
:109AF000D9F8001051F8040BC9F8001000283CD127
:109B00004FF0FF340FF64C20E7E6D9F8001051F87B
:109B1000040BC9F8001080B94FF0FF340FF6342061
:109B2000DBE6D9F8001051F8040BC9F8001020B991
:109B30004FF0FF340FF61C20CFE60D9AD317C0E983
:109B40000023F9E3D9F8001051F8040BC9F800100C
:109B500020B94FF0FF340FF6FC10BEE60D990170EE
:109B6000EAE3D9F8001051F8040BC9F8001020B945
:109B70004FF0FF340FF6DC10AFE60D990160DBE328
:109B80009DF842004C2807BFD9F80010CA1DD9F82B
:109B90000000C21D22F00702C9F80020D2E900012E
:109BA0000832C9F80020CDE90201C80F02D0079899
:109BB0002D210AE0BDF84010880702D507982B2117
:109BC00003E0C80705D50798202112AA1154401CAC
:109BD000079012A807994BF0200300EB010CDDE978
:109BE0000201CDE92C01612BCDF814C021AC0BD0C2
:109BF0000E98002848BF062105D404BF4BF0200072
:109C0000672801D101210E91DDE902677B0043EA5B
:109C1000D6735A15DB174FF0FF30834208BF8242DC
:109C200010D13F0347EA16573603002F08BF002E16
:109C300008D0ABF1610503211A2D089118D30FF656
:109C4000341110E0DDE902014A00521512F1010F52
:109C500011D108030FD1ABF1610503211A2D089131
:109C60001FD30FF6181103226046F8F72DF963E3AE
:109C70000FF6FC01F7E7DDE902016A46F8F700FE9E
:109C8000CDE902014BF02000612811D10598302266
:109C90000270811C0591BBF1610F0CBF7821582126
:109CA00002E00FF6D401DEE741700798801C0790B0
:109CB000DDE9020120F0000231F0004308BF002A74
:109CC00002D10026002542E14BF02008B8F1610FD7
:109CD00040F093800E98002847BF21210191401C3D
:109CE0000190019EDDE92C01761C00220023DDE9B4
:109CF000024500F0B9FD38BF85F0004500988DF8A9
:109D00008420001F002E00900DF1850732DD2046D3
:109D1000294600220023F8F73BFC2BD21C22F8F73F
:109D20000BFF04460D4601F0B7FBF61F002E8046E0
:109D300009DDF9F709F902460B4620462946F9F7ED
:109D4000D3F904460D46F81D0721B8F1000F0CDDCC
:109D5000491E5EBF08F00F0200F8012D4FEA2818D7
:109D6000F3D502E0002200F8012D491EFAD5C71DE7
:109D7000002ECCDC0DF185003F1A01980DF1850411
:109D80003E468742C8BF0646002E2FD4BE4206DAA2
:109D90000DF18500815D0829A8BF0F2000DA0020A1
:109DA000324621A98D1800E0761E15F80139521EA1
:109DB0008342F9D00F2804D10DF18501885C401C45
:109DC0008854002A04D50098001D21AC761C009010
:109DD000701E0BD421180B783033DAB23A2AA4BFA4
:109DE0005B443A3B401E01F80139F4D50E99002935
:109DF00040F1AC80701E0E90A8E00099DFF8FC26C0
:109E000047F29750414391FBF2F20092DDE92C4575
:109E1000C2F10702002A25F0004504DD204629464C
:109E200000F049FB0BE052420020DFF8D41600F0AE
:109E300042FB02460B4620462946F8F759FD0446E8
:109E40000D46B8F1660F06BF009E0A3606260E982C
:109E50003618142EC8BF142630208DF884000DF15A
:109E60008507002E34DD2046294601F031FB0146EE
:109E70000A4607F1080C04200A27B2FBF7FE0EEB96
:109E80008E03A2EB430230320CF8012C0A22BEFBF7
:109E9000F2F202EB8203AEEB43033033401E0CF8C8
:109EA000023DE9D1083E002E0CF10807D9DD084635
:109EB00000F0CCFC02460B4620462946F9F714F97F
:109EC0000022DFF84036F8F705FC04460D46CAE7E5
:109ED0000DF185003F1A0DF1850404E00098401E45
:109EE0007F1E0090641C20783028F7D0B8F1660FF0
:109EF00002D1009E761C04E0B8F1650F0CBF01266C
:109F000000260E983618B742B8BF7E1E002E1DD40C
:109F1000BE4204DAA05D3428C8BF392000DC3020FE
:109F20003246611E8D1800E0761E15F80179521E2A
:109F30008742F9D0392802D1A05C401CA054002AE5
:109F400004D50098401C0C46761C0090009DF8F744
:109F50004BF9406A0778DDF8388030B2002802DC1F
:109F600001260FF21C644BF02000662808BF6D1C10
:109F700016D0672845D128B210F1040F47DB4045C1
:109F800045DA9DF840106D1C080703D430B24045F7
:109F9000D8BF804628B2B8EB000848BF4FF0000891
:109FA0000FFA85FBBBF1000F00F3B3800898411C4A
:109FB0000891302205990A54B8F1000F03DC9DF88E
:109FC0004010080704D50898411C089105990F54C2
:109FD00018EB0B0FB8BFC8F100052DB2684245441D
:109FE00032B20B909542B8BF2E46059B089836B208
:109FF0000996324621461844F7F766FFAD1B0C95CB
:10A00000D1E0BBF1610F17D14FF0700B19E030B206
:10A01000404504DA9DF840100A0758BF8046B8F161
:10A02000010848BF4FF00008BBF1670F14BF4FF0A5
:10A03000450B4FF0650B04E0BBF1410F08BF4FF03B
:10A04000500B0898411C0891B8F1000F059914F8BD
:10A05000012B0A5403DC9DF8401008071AD5089814
:10A06000411C0891B8F1000F05990F5412DD761EBE
:10A0700030B28045B8BF46460598089B32B22146AB
:10A080001844F7F721FF089836B230180890A8EB6B
:10A0900006000B9005980899014428B2002881F821
:10A0A00000B003D42B204870891C04E02D224A7094
:10A0B0000546891C6D4200202CAA0AE02B460A2581
:10A0C00093FBF5F505EB8504A3EB440302F8013B94
:10A0D000401C2DB2002DF1DC012806DC4BF02002E3
:10A0E000652A04BF302201F8012B00282CAB08D1CF
:10A0F000302001F8010B06E0401E1A5C303201F8F6
:10A10000012B0028F8DC059A08981044091A0991D7
:10A1100049E031B228B281421CDA059B089832B27C
:10A1200021461844F7F7D0FE089936B27118089105
:10A13000ABEB0600B8F1000F0B9003DC9DF840007C
:10A14000020704D5059847540999491C0991CDF88F
:10A15000308028E0059B08982AB221461844F7F77A
:10A16000B3FE0898761B5844B8F1000F089003DC42
:10A170009DF840100A0703D5411C089105990F541A
:10A1800030B28045B8BF46460598089B32B204EB12
:10A190000B011844F7F798FE089836B2301808906B
:10A1A000A8EB06000B909DF8400000F0140010286A
:10A1B00040F0C280079A08980B99821809988A186B
:10A1C00082180C980F998018884280F2B580081A7E
:10A1D0000A90B1E09DF84200622808D068280ED0AD
:10A1E0006A2814D06C281FD0712810D01CE0D9F830
:10A1F000001051F8040BC9F80010C0B21AE0D9F8E9
:10A20000001051F8040BC9F8001080B212E0D9F820
:10A210000000C21D22F00702C9F80020D2E90001A7
:10A220000832C9F8002006E0D9F8001051F8040BF4
:10A23000C9F800100021CDE902019DF84000020795
:10A240005AD5DDE90201002908BF002854D04BF09F
:10A250002002782A50D1079912A830234354491C70
:10A260004A1C079200F801B046E09DF842006228BF
:10A2700008D068280ED06A2814D06C281FD0712806
:10A2800010D01CE0D9F8001051F8040BC9F80010E8
:10A2900040B21AE0D9F8001051F8040BC9F80010C8
:10A2A00000B212E0D9F80000C21D22F00702C9F87E
:10A2B0000020D2E900010832C9F8002006E0D9F8F0
:10A2C000001051F8040BC9F80010C117CDE90201C4
:10A2D000002902D507982D220AE0BDF84000810729
:10A2E00002D507982B2203E0C00705D50798202246
:10A2F00012A90A54401C079012A80799014405911D
:10A30000594602A800F04EF816E001200790D9F84F
:10A31000001051F8040BC9F800108DF848000BE04C
:10A3200001222521BBF1000F07928DF8481003D0C0
:10A33000022007908DF849B00F9D07980A992D1AB1
:10A3400008986D1A0B992D1A09986D1A0C992D1AE7
:10A350009DF840006D1A41073FF5D2AA2020002D3C
:10A360008DF800007FF7CCAA309E2C46FFF7BCBAD0
:10A370004FF0FF3031B0BDE8F08F0000CBCCCC0CFB
:10A38000686A6C747A4C00007072696E74665F73F0
:10A390003A2062616420257320617267756D656E75
:10A3A000740000002DE9FE4C06468B46376958467E
:10A3B0006F2808BF082205D0FFF77EF9782814BF60
:10A3C0000A221022D6E900013C2504468A46BBF148
:10A3D000640F18BFBBF1690F04D1002902D5644294
:10A3E0006AEB4A0ABAF1000F08BF002C0CD1306B9F
:10A3F00050B9082A3BD196F83810080737D53021D4
:10A400003B2587F83B1032E08DF800B0934620469C
:10A4100051465A460023F9F7FBF83032D0B26D1E90
:10A420003A2801950DDA7A55204651465A460023BE
:10A43000F9F7EEF804465FEA010A08BF002C05D1DF
:10A4400008E09DF800001218513AECE7F16878191D
:10A450008142DCD3BBF1080F09D196F8380001071F
:10A4600005D5785D302802D06D1E30207855C5F1B5
:10A470003C02306BB26179198242F16007DA318FA8
:10A48000821A4FF6EF7001403262318710E00028E7
:10A490000ED596F8380000F01400102808D1736B20
:10A4A0007069316A1B1A5B1A9B1A002BC8BF336292
:10A4B00003B0BDE8F08C2DE9D04306460F461446A4
:10A4C0004FF00008DFF8409012E0E00707D5424661
:10A4D0004B4630463946F8F7FDF806460F464046EB
:10A4E000494642464B46F8F7F5F8641080468946DF
:10A4F000002CEAD130463946BDE8D083A086010061
:10A500000000F03F84D7974100002440F8B505468D
:10A510000E4617461C4600205CB117F8011BB068B8
:10A52000A847B06030B1F06A401CF0620020641EA1
:10A53000F3D1F2BD4FF0FF30F2BD00007072696ED2
:10A5400074665F733A20256E20646973616C6C6F6A
:10A55000776564007072696E74663A206261642087
:10A56000256E20617267756D656E740000000000D5
:10A570006E616E004E414E00696E6600494E4600A7
:10A580003000000010B50400074801684FF47A70ED
:10A59000B1FBF0F0FAF780FF002221005FF0FF30FE
:10A5A000FAF753FF002010BDE007002081B00B49EF
:10A5B000086850F001000860086810F00100009081
:10A5C00000980749086850F080500860086810F04B
:10A5D00080500090009801B0704700BF20380240C2
:10A5E0002438024001000120704710B4040000200C
:10A5F0006060002020602161E260A3600248606129
:10A60000A061012010BC7047E5A500080300596156
:10A610009A6101207047020053689068834207D214
:10A620005068431C5360D36843F82010012000E0B9
:10A630000020704770B504000D00002620006169FD
:10A640008847002807D029002000FFF7E4FF060014
:10A650002000A16988473000C0B270BD10B5040069
:10A660006068002817D021686068814213D2206991
:10A67000E268216852F821108847002802D020683B
:10A68000401C206020686168884201D3012000E0FE
:10A690000020C0B200E0012010BD010000200860D1
:10A6A0000120704701000020486000200860012060
:10A6B000704738B5040000252000616988470028EC
:10A6C00006D02000FFF7EEFF05002000A1698847B3
:10A6D0002800C0B232BD00FF00F10103810704D0A1
:10A6E00010F8011B820781B1FAD10268A2F1013191
:10A6F000914311F0803104BF50F8042FF6E709BAF6
:10A70000B1FA81F100EBD100401CC01A7047FF0084
:10A7100080B500220021002000F001F802BD10B435
:10A720000300002901D100208BE05FF0FF3043409F
:10A73000082A4AD344480C785C4004F0FF0450F8DF
:10A74000244094EA1324491C0B78634003F0FF0370
:10A7500050F8233093EA14234C1C2178594001F01F
:10A76000FF0150F8211091EA1321641C23784B401B
:10A7700003F0FF0350F8233093EA1123641C21787F
:10A78000594001F0FF0150F8211091EA1321641C97
:10A7900023784B4003F0FF0350F8233093EA112352
:10A7A000641C2178594001F0FF0150F8211091EA12
:10A7B0001321641C23784B4003F0FF0350F823302F
:10A7C00093EA1123611C083AB2E7042A26D31E48F3
:10A7D0000C785C4004F0FF0450F8244094EA132401
:10A7E000491C0B78634003F0FF0350F8233093EAD1
:10A7F00014234C1C2178594001F0FF0150F821101E
:10A8000091EA1321641C23784B4003F0FF0350F8B6
:10A81000233093EA1123611C121FD6E7002A0CD0C3
:10A82000094C0878584000F0FF0054F8200090EAE6
:10A830001323491C521E002AF2D15FF0FF3043401F
:10A84000180010BC70470000E436010850B1B0FA9F
:10A8500080F18840C91CC1F58461090501EBD02154
:10A86000400570470146704741EA030C50EA4C0C22
:10A8700052EA0C0C4FF4001C09D307D01CEB410F1B
:10A880009CBF1CEB430F8B4208BF824270471CEBFE
:10A89000430FFBD8994208BF9042704710B504009F
:10A8A000002301220121200000F0B9FD10BD10B5E8
:10A8B000040001220121200000F072FD012201218B
:10A8C000200000F082FD10BD10B50400002201211F
:10A8D000200000F07AFD00220121200000F060FD40
:10A8E00010BD2DE9F54F87B00D00079810F5827661
:10A8F00002270798D0F81802002800F00C812800E1
:10A9000000F02BFD002800F006810798D0F818020F
:10A9100004900498C068002800F0FD80F168B068D9
:10A92000814202D2F068039001E0B0680390B468FD
:10A930000398241A0399280000F086FC280000F0F0
:10A94000D4FCF1688C4201D2210000E0F168884219
:10A9500002D3002C40F0DD80280000F037FC804658
:10A96000D6F80490B9EB0409B9EB080918EB040315
:10A970004A462900079810F50270DDF810C0DCF88F
:10A980000CC0E0470290280000F0E7FC8DF80500BD
:10A99000002C04D09DF80500002800F0B780029834
:10A9A000002800F0AD80C2469DF80500002800F0A8
:10A9B0009880280000F00AFC002800F08080280021
:10A9C00000F05EFC824600208DF80400280000F0B4
:10A9D0008CFCF1688C4201D2210000E0F1688842D1
:10A9E00002D30020070002E001208DF804009DF84A
:10A9F0000400002801D1002C77D10298002858D0FB
:10AA0000280000F0E3FB80469DF80400002801D0F8
:10AA1000200000E0002010EB08000590D6F804B0FC
:10AA20000598BBEB000B059B5A462900079810F5CB
:10AA30000270DDF810C0DCF80CC0E0470290002C7A
:10AA400004D0280000F089FC00282FD09DF80400D5
:10AA5000002819D0280000F048FCF1688C4201D28F
:10AA6000210000E0F16888420ED3280000F008FCC5
:10AA700018EB0A000090280000F0A8FB0099081AC3
:10AA800082460020070014E0280000F0F9FB18EBD4
:10AA90000A000090280000F099FB0099081A8246ED
:10AAA000280000F093FB0028A7D102E00220070055
:10AAB000A3E70298002818D10220070015E028001B
:10AAC00000F013FCF1688C4201D2210000E0F16833
:10AAD000884203D2280000F0D3FB82460020070002
:10AAE00003E0002C01D1002007003800C0B200288C
:10AAF00011D1089800280ED00898C0F800A00AE0EC
:10AB0000280000F0AAFA0220070004E00220070053
:10AB100001E0032007003800C0B209B0BDE8F08FA3
:10AB20002DE9FE4F06000F00140016F114085FF027
:10AB30000209D6F81802002800F09380380000F0CF
:10AB40000CFC002800F08D80D6F8180200900098C8
:10AB50000069002800F085805FF0000AD8F808003E
:10AB6000002811D1D8F80450D8F80C10B5FBF1F03A
:10AB700001FB1055002D02D1D8F80C00050029006A
:10AB8000380000F049FB0FE0D8F80C10D8F80800A6
:10AB9000814202D2D8F80CA001E0D8F808A0D8F879
:10ABA0000C10380000F038FBD8F80800002805D158
:10ABB000380000F052FA0020814652E0380000F0E0
:10ABC00005FB0500554502D30320814649E0002DD1
:10ABD00006D0380000F054FB002C07D0206005E0C0
:10ABE000380000F04DFB002C00D02060D8F804B0F5
:10ABF000D8F80800BBEB000B15EB0B0BD8F80830AE
:10AC00005A46390016F50270DDF800C0DCF810C0B5
:10AC1000E0470190380000F0A0FB00281FD0019809
:10AC2000002819D0D8F80810D8F80C00814209D3B0
:10AC3000380000F0CBFAD8F80C10884211D300206D
:10AC400081460EE0380000F0C1FAD8F808108842BA
:10AC500007D10020814604E00220814601E0022065
:10AC600081464846C0B2BDE8FE8F2DE9F84F050089
:10AC70000E0017005FF00008D5F818020090F08869
:10AC8000002858D03078000644D5380000F065FB25
:10AC900000283CD0380000F0E0F9F38800223900A9
:10ACA0003000009C2469A0470400380000F055FBE8
:10ACB000002829D015F1140BDBF80C10F088814224
:10ACC00004D2DBF80C90B9F1010901E05FF0000952
:10ACD000380000F07BFA8246002C12D0D14509D210
:10ACE000F188380000F081FAF288F9682800FBF753
:10ACF00083FE22E0524692B2F9682800FBF77CFE00
:10AD00001BE00220804618E00220804615E0022069
:10AD1000804612E0380000F020FB002808D0380000
:10AD200000F09BF9F288B9682800FBF7C2FE04E046
:10AD30000220804601E0022080464046C0B2BDE8C5
:10AD4000F28F2DE9F04781460C0015001E0020000F
:10AD5000C0B210F07F000001484410F11407D9F888
:10AD600018823000C0B2002815D1D8F82C00002875
:10AD700001D1022034E0280000F06FF92800FFF72D
:10AD800096FD29002000C0B2D8F82C20904700285A
:10AD900001D1022024E0280000F018FA8246F96868
:10ADA000504680B2814201D2F8688246514689B24B
:10ADB000F868814202D12800FFF779FD2300DBB259
:10ADC000524692B2E9684846FBF72BFE002801D0B4
:10ADD000022005E0514689B2280000F01DFA00204B
:10ADE000BDE8F087F8B504000D002800C0B210F0EF
:10ADF0007F000001204410F11406D4F818720020DE
:10AE00008DF800002B00DBB2002269462000FBF722
:10AE100008FE002801D0022000E00020F2BD2DE94C
:10AE2000F84304000D0016002800C0B210F07F00A7
:10AE30000001204410F11407D4F81882300000F00B
:10AE4000C5F9F968884215D2300000F04EFAF96869
:10AE5000884202D2300000F013FA31002800C0B25C
:10AE6000D8F82C209047002804D1300000F0F5F8E5
:10AE700002203FE0300000F0A9F98146F968484619
:10AE800080B2814205D2F86881463000FFF70FFD9D
:10AE90001EE0494689B2F868814203D13000FFF7CD
:10AEA00006FD15E0484680B2002803D03000FFF7C9
:10AEB0000BFD0DE0484680B2002809D13000FFF7B5
:10AEC000EDFC002801D1002014E03000FFF7FCFC6D
:10AED0002B00DBB24A4692B2F1682000FBF7D5FDA9
:10AEE000002806D1494689B2300000F095F90020CB
:10AEF00000E00220BDE8F2832DE9F84F83468A4640
:10AF000015001E005046C0B210F07F0000015844EA
:10AF100010F58277DBF818827C68B868241A300054
:10AF2000C0B2002803D02800FFF7C1FC02E02800CF
:10AF3000FFF7CAFCD8F8280000284AD0002C0DD111
:10AF4000280000F08AF829005046C0B2D8F828201E
:10AF50009047002801D000203FE03AE0210028007F
:10AF600000F072F9002834D029005046C0B2D8F859
:10AF70002820904700282CD03000C0B2002807D0ED
:10AF8000280000F023F9002823D1280000F065F8FC
:10AF9000280000F0AAF98146280000F0A6F9F96817
:10AFA000884216D3280000F06BF9494689B2F86848
:10AFB0001FFA89F9B9EB0109B1FBF0F100FB019926
:10AFC0005346DBB24A4692B2A9685846FBF7BEFD2B
:10AFD00003E0280000F041F80220BDE8F28F2DE9DF
:10AFE000F84304000D001600D4F81872300000F089
:10AFF00034F8300000F079F980462800C0B210F033
:10B000007F000001204410F58279414689B2D9F8C9
:10B010000C00814214D3414689B2D9F80C001FFAC2
:10B0200088F8B8EB0108B1FBF0F100FB01882B00B8
:10B03000DBB2424692B2B1682000FBF751FD00E05E
:10B040000220BDE8F28303000220002903D0C3F8E8
:10B05000181200221000C0B27047002807D04168C3
:10B0600081604168C160026941690A4002617047BC
:10B070002DE9F04106000C0015001F00DDF81880D6
:10B08000002C01D0002D01D100200BE07460356050
:10B09000C6F8188000203061002070613000FFF792
:10B0A000DCFF0120BDE8F0812DE9F04704000D0030
:10B0B0001600002C1ED0002D1CD0002E1AD0606867
:10B0C000002817D02068002814D0A76860683F1AAD
:10B0D0002168F01981420DD3B046A946D4F808A0E2
:10B0E000424649465046F6F7EFFEA0683044A0605D
:10B0F000300000E00020BDE8F0872DE9F0470500B2
:10B100000E001400002D23D0002E21D0002C1FD0C3
:10B11000686800281CD02868002819D0AF686868C3
:10B120003F1A2968E019814202D22868C01B040036
:10B13000002C0DD0A046B146D5F808A0424649469D
:10B140005046F6F7C1FEA8682044A860200000E041
:10B150000020BDE8F0872DE9F84F04000D0016002F
:10B160009846002C2FD0606800282CD0206800283A
:10B1700029D0A768E0683F1A002D22D0002E20D0E9
:10B18000002F20D0BE420DD2B346D4F80C90AA4670
:10B190005A4649465046F6F797FEE0683044E0606C
:10B1A000300011E0BB46D4F80C90AA465A464946F6
:10B1B0005046F6F789FE6068E0606068A06038007D
:10B1C00002E0002000E00020BDE8F28F010000292D
:10B1D00009D04868002806D00868002803D088688D
:10B1E000CA68801A00E0002070470200002A11D0CF
:10B1F000506800280ED0106800280BD09368D068E3
:10B200001B1A994204D2D06808189060080002E026
:10B21000180000E0002070470200002A12D0002928
:10B2200010D0506800280DD0106800280AD093680C
:10B23000D0681B1A8B4200D21900D0680818D06061
:10B24000080000E00020704710B40200002A14D06B
:10B25000002912D0506800280FD0106800280CD0A8
:10B26000136894685068241A1B1B8B4200D2190083
:10B27000906808189060080000E0002010BC70473B
:10B280002DE9F0410400002C1FD0606800281CD07C
:10B290002068002819D0A568E0682D1A002D0CD070
:10B2A0002E00E768D4F8048032003900404600F0F0
:10B2B00021F960682818A06001E06068A060E0687B
:10B2C0006168401A6168E16000E00020BDE8F0813B
:10B2D0000100002907D04868002804D00868002829
:10B2E00001D0086800E000207047010000290BD061
:10B2F0004868002808D00868002805D088684A688F
:10B30000801A0968081A00E000207047F8B50400A8
:10B310000D001600002C1ED0002D1CD068680028DF
:10B3200019D02868002816D0A769200029001C22FF
:10B33000F6F7DAFD002068600020A8600020E860D1
:10B340000020286029696869014029613000C0B285
:10B35000002800D1A7610020F2BD010000291DD006
:10B36000486800281AD00868002817D08868002884
:10B3700014D0C868002811D04A6808688218886804
:10B3800082420BD34A6808688218C868824205D393
:10B390008A68C868824201DB012000E00020704713
:10B3A00030B40300002B0DD01C69586984438C43D2
:10B3B00012EA010004431D69586905402C431C61D1
:10B3C000012000E0002030BC704710B40300002BC7
:10B3D00007D05C698C4312EA010004435C610120E0
:10B3E00000E0002010BC704770B406690E4011EAFE
:10B3F00002041D00EDB2002D08D16640B1430029C2
:10B4000001D0012000E00020C0B206E094EA060F5F
:10B4100001D1012000E00020C0B270BC7047F8B537
:10B4200004000F0015001E00002C07D03300DBB213
:10B430002A0039002000FFF7D7FF00E00020F2BD0E
:10B44000C9B202788A421AB11CBF10F8012FF9E77D
:10B4500018BF00207047010280B500B906A0054959
:10B460000B681BB122220021984701E0F6F792FEFB
:10B47000222002BD243B0020636F6E7374726169E9
:10B480006E742068616E646C65723A20626164203B
:10B490006D65737361676500C1F30A5340F21E4224
:10B4A000D31A0CDDCA0283F3070342EA505242F07A
:10B4B0000042DA4002EBE17282EAE17070476FEA23
:10B4C000E17203F2E13008B182F0004070470304FA
:10B4D000400D40F21E4C40EAC120BCEB115C40F034
:10B4E000004003D48CF30701C84070476FEAE17055
:10B4F0007047040181423ABF53189842F6F7E4BC02
:10B500008018990707D0521E24BF13F8011D00F8B8
:10B51000011DF6D8704781071BD1103A07D330B40C
:10B5200033E93210103A20E93210F9D230BC10322F
:10B53000121F24BF53F8041D40F8041DF8D838BF6B
:10B54000121D521E24BF13F8011D00F8011DF8D86A
:10B550007047121FF3D3C10709D153F8041D121FFE
:10B5600020F8041D4FEA31414180F6D2E7E753F855
:10B57000041D121F00F8041D4FEA3121A0F801102C
:10B580004FEA3141C170F2D2D9E7020380687047B7
:10B59000C068704710B5040000230122012120007B
:10B5A000FFF73DFF10BD10B504000022012120006F
:10B5B000FFF70BFF002201212000FFF7F1FE10BD75
:10B5C000F8B50400002060700020A07000202070FA
:10B5D0000020E07008270025261D2A0039003000D1
:10B5E000F6F732FCF1BDF8B50400002060730020CE
:10B5F000A073002020730020E0730827002514F1B9
:10B6000010062A0039003000F6F71EFCF1BDF8B52F
:10B6100007000224002517F118062A002100300037
:10B62000F6F712FCF1BD10B5040014F11500606CC2
:10B63000FFF7AEFF20660C2214F10C01606CFFF7DF
:10B6400033FD002803D100202066002000E0012007
:10B6500010BD10B50400002C07D15622DFF84C1A9B
:10B66000A8A0F6F785FBAFF30080206E002815D068
:10B67000A16B206E416094F84000002806D0206E37
:10B68000017A51F00101206E017205E0206E017A0D
:10B6900011F0FE01206E0172012000E0002010BDBB
:10B6A00010B50400A06DFFF773FF6066022214F16D
:10B6B0001801A06DFFF7F8FC002803D10020606698
:10B6C000002003E0206D801C2065012010BD10B516
:10B6D0000400002C07D18722DFF8D01989A0F6F7E3
:10B6E00047FBAFF30080606E002813D094F856003B
:10B6F00050F08000207694F85500607694F856104B
:10B7000051F08001606E017094F85510606E4170C8
:10B71000012000E0002010BD2DE9F04104000D00E3
:10B720001600DFF88C7940F281182000FFF7D0FD79
:10B73000404510D32000FFF7CBFD404508D3A6229B
:10B74000DFF86819DFF86C09F6F712FBAFF3008039
:10B750007FF008004DE03800FFF732FF3800FFF7B8
:10B7600042FF3800FFF753FF00203877002087F8AA
:10B7700028000020386200207862FC62002087F8F0
:10B780003000002087F83100002087F834000020C6
:10B7900087F840000020B8630020F8637D64002033
:10B7A00087F84800002087F84900002087F84C00FF
:10B7B000002087F8540000203865002087F85600E4
:10B7C000002087F85500BE65002087F85C00DFF890
:10B7D0009C0A00688047002806D0DFF8941A5FF0C2
:10B7E000FF300860086804E0DFF8841A0020086071
:10B7F0000868BDE8F08118B589B006ACDFF8740AB6
:10B8000090E80E0084E80E0006A800F0A4FE03AC49
:10B81000DFF8640A90E80E0084E80E0003A800F048
:10B820009AFE6C46DFF8540A90E80E0084E80E0099
:10B83000684600F090FEDFF8340AC0698047DFF800
:10B84000301A0020086008680AB010BD38B504003E
:10B85000DFF85C582078052812D02078052808D019
:10B86000EA22DFF84818DFF8180AF6F781FAAFF392
:10B870000080DFF8FC197FF009000860086840E0EC
:10B880002079002802D1287F002827D0207900289D
:10B8900003D1E1796878814220D1687885F8310058
:10B8A00000202877002085F830002079002802D079
:10B8B000002085F831002800FFF782FEA0790028DB
:10B8C00003D1E86AFFF7C9FB02E0E86AFFF7D8FC9A
:10B8D000DFF89C1900200860086812E0E17995F80B
:10B8E0003100814208D1002085F83100DFF880194D
:10B8F00000200860086804E0DFF87419022008607E
:10B90000086832BD6374780038B50500DFF8A047D9
:10B910002878042813D02878042809D04FF491728D
:10B92000DFF88817DFF8900AF6F722FAAFF3008005
:10B93000DFF83C197FF009000860086850E02879BA
:10B94000002803D194F83400002836D02879002844
:10B9500003D1E979607B81422FD1607B84F8490073
:10B96000002084F83400002084F84800002020667D
:10B970002879002802D0002084F849002000FFF731
:10B9800032FEA879002809D04FF49B72DFF81C170B
:10B99000DFF8280AF6F7ECF9AFF30080606CFFF7E8
:10B9A0005CFB6879002802D0606CFFF7FCFDDFF8D3
:10B9B000C01800200860086812E0E97994F849008E
:10B9C000814208D1002084F84900DFF8A418002043
:10B9D0000860086804E0DFF898180220086008682A
:10B9E00032BD38B50400DFF8C8562078062813D0D9
:10B9F0002078062809D040F26112DFF8B016DFF88F
:10BA0000080BF6F7B5F9AFF30080DFF864187FF0A4
:10BA10000900086008683FE02079002803D195F804
:10BA20004C00002833D02079002804D1E17995F822
:10BA3000560081422BD1002085F84C00002085F86B
:10BA40005C00002085F8540000202865002085F85F
:10BA50005500002085F85600002068662800FFF792
:10BA6000D6FDA079002809D04FF4BA72DFF83C1651
:10BA7000DFF84809F6F77CF9AFF30080A86DFFF70F
:10BA8000ECFADFF8EC1700200860086804E0DFF843
:10BA9000E01702200860086832BD10B40200DFF829
:10BAA00010360800C0B2002803D193F84C000028DB
:10BAB0001AD00800C0B2002805D1140093F856002F
:10BAC000E4B2844210D1002083F84C00002083F8B7
:10BAD0005C00012083F8540013F11800DFF8904750
:10BAE00000202060206804E0DFF884470220206006
:10BAF000206810BC704770B504000D0000262800B7
:10BB0000FFF764FB0C2802D27FF001006BE00023FA
:10BB10000C2221002800FFF71EFB0C2802D07FF02A
:10BB2000020060E06178A0784140FF2902D160788E
:10BB3000002802D17FF0030055E021780800C0B250
:10BB4000012808D002281CD07E2841D07F2842D06E
:10BB5000802843D045E06068002802D17FF00300D0
:10BB60000EE06068206201202077012084F8300018
:10BB700000206062207A10F0010084F82800002084
:10BB800031E06068002802D17FF003001FE0207AD6
:10BB9000800702D57FF0060019E06068A0630120ED
:10BBA00084F83400012084F848000020E06300207D
:10BBB00084F8400060786073A078A073022020733E
:10BBC0000020E073A06B20610120207500200AE0B6
:10BBD0007FF0050007E07FF0050004E07FF005003E
:10BBE00001E07FF00400DFF888160860086870BD87
:10BBF00070B504000D000026A06DFFF776FB02284B
:10BC000002D27FF0010013E084F85650002084F83F
:10BC10005500012084F84C00012084F85C000020CD
:10BC200084F85400002020652000FFF7F0FC00207D
:10BC3000DFF83C160860086870BD0100DFF870246A
:10BC4000002906D1DFF828367FF00900186018684F
:10BC500014E0107F002802D05078087009E092F8B4
:10BC60003100002803D092F83100087001E0002074
:10BC70000870DFF8FC350020186018687047010074
:10BC8000DFF82C24002906D1DFF8E4357FF0090025
:10BC90001860186815E092F83400002802D0507B34
:10BCA000087009E092F84900002803D092F8490092
:10BCB000087001E000200870DFF8B435002018603B
:10BCC000186870470100DFF8E823002906D1DFF883
:10BCD000A0355FF0FF301860186806E0506A086011
:10BCE000DFF88C3500201860186870470100DFF815
:10BCF000C023002906D1DFF878355FF0FF301860E7
:10BD0000186806E0D06B0860DFF864350020186022
:10BD1000186870470100087F002805D1DFF850251A
:10BD200002201060106804E0DFF844250120106054
:10BD300010687047010091F83400002805D1DFF841
:10BD4000302502201060106804E0DFF8242501206F
:10BD5000106010687047010091F84C00002805D170
:10BD6000DFF80C2502201060106804E0DFF80025E1
:10BD70000120106010687047FEB505000024DFF850
:10BD800030630027287802287AD13000FFF7C2FFFD
:10BD9000022874D169683000FFF7ADFE040030005E
:10BDA000FFF7C8FF01286AD1012007003000FFF724
:10BDB0003AFC002803D15FF0FF3004005FE0706CB4
:10BDC000FFF7F1FB716C300000F05CFA0400002C0E
:10BDD00055D4002C45D0022C16D006D3042C31D0DB
:10BDE00021D3062C3DD03CD33EE0012C08D140F2BB
:10BDF0006532AE49DFF81407F5F7BAFFAFF30080FC
:10BE00005FF0FF3004003AE0022C08D140F26B32C0
:10BE1000A649DFF8FC06F5F7ABFFAFF300805FF053
:10BE2000FF3004002BE0032C08D140F271329F490F
:10BE3000DFF8E006F5F79CFFAFF300805FF0FF301E
:10BE400004001CE0042C08D140F277329749DFF857
:10BE5000C806F5F78DFFAFF300805FF0FF300400F8
:10BE60000DE0052004000AE0002C08D040F28732E3
:10BE70008E49DFF8A806F5F77BFFAFF300800AE0F4
:10BE80007FF00900040040F29132884986A0F5F75E
:10BE90006FFFAFF30080002C0BD43000FFF73AFFA8
:10BEA000012806D1012007006968300000F004F97C
:10BEB00004003800C0B2002803D1002C01D10220B8
:10BEC0000400DFF8AC030460002C14D5220069687C
:10BED000300000F03DFBEC46DFF8440690E80E0031
:10BEE0008CE80E006846FFF7B1FC14F1080F02D091
:10BEF0005FF0FF3004002000FEBDF8B5040000270D
:10BF00006B4D207801280CD12800FFF713FF012882
:10BF100005D16168280000F0B5F9060000E00226AE
:10BF200009E07FF009064FF47A7260495EA0F5F7E8
:10BF30001FFFAFF30080DFF838030660002E04D542
:10BF400032006168280000F004FB3000F2BDFEB54D
:10BF500005000224564E2878002802D003280CD071
:10BF60007DE06868002802D07FF0090099E0297A16
:10BF70003000FFF73DFE04007CE03000FFF7EBFEF1
:10BF800001286BD13000FFF78BFB002803D15FF055
:10BF9000FF30040062E06968300000F011FA04002C
:10BFA000002C5BD4002C45D0022C16D006D3042CD8
:10BFB00031D021D3062C3DD042D344E0012C08D10E
:10BFC00040F249423949DFF84405F5F7D1FEAFF3B5
:10BFD00000805FF0FF30040040E0022C08D140F206
:10BFE0004F423249DFF82805F5F7C2FEAFF3008073
:10BFF0005FF0FF30040031E0032C08D140F25542DD
:10C000002A49DFF81005F5F7B3FEAFF300805FF0C3
:10C01000FF30040022E0042C08D140F25B422349A7
:10C02000DFF8F404F5F7A4FEAFF300805FF0FF3013
:10C03000040013E0002196F85600FFF72EFD0400DF
:10C04000052004000AE0002C08D040F27142174994
:10C05000DFF8C804F5F78CFEAFF300800AE07FF04C
:10C060000900040040F27A4210490FA0F5F780FE63
:10C07000AFF300807E480460002C11D5220069686F
:10C08000300000F067FA6F46DFF8980490E80E0081
:10C0900087E80E006846FFF7A4FC5FF0FF3004005D
:10C0A0002000FEBD0000000030000000908201086A
:10C0B000A0390020949701082DE9F84F8AB08246F4
:10C0C00088464046FFF782F80400DAF82070DAF874
:10C0D00024003F1ADAF82050D5F1040515F00305C5
:10C0E0004046FFF757FA814600269AF830008DF84F
:10C0F00000004846C0B200280AD0E819844205D2A0
:10C10000002004005FF0FF3006000DE03C000BE073
:10C1100015EB070B1BF10C0B4046FFF7D9F88345D5
:10C1200002D35FF0FF300600002E6ED19DF80000B4
:10C13000002802D04D48806880474046FFF728FA23
:10C140009DF800304A46D2B22100DFF820C1DCF869
:10C150000CC0E047002808D001280FD07FF0010173
:10C16000884206D0B0F1FF3F16D10021404801605F
:10C1700012E05FF0FF313E4801600DE04846C0B27A
:10C18000002804D05FF0FF313948016004E000204E
:10C190000400042136480160002C0CD021004046E8
:10C1A000FFF73AF83F1B002F05D1002D03D02900DF
:10C1B0004046FFF731F84846C0B2002821D0DFF8EA
:10C1C000B0B0DBF80000002812D44046FEF7FEFFB6
:10C1D00000280DD004ABDFF8500390E8061083E888
:10C1E000061004A8FFF732FB0320CBF8000008E09C
:10C1F00001ABCE4890E8061083E8061001A8FFF7CF
:10C2000025FB00208AF830002BE000213000174A7F
:10C2100092699047002805D07FF00101401A01285B
:10C2200004D908E000201249086010E05FF0FF30F8
:10C230000F4908600BE040F23552BD49B1A0F5F757
:10C2400097FDAFF300805FF0FF31094801600DF109
:10C250001C0CB84890E80E008CE80E0007A8FFF709
:10C26000F5FA034800680BB0BDE8F08F3497010879
:10C27000203B00208808002094080020A00800200F
:10C2800078940108F8B588B006000D002800FFF783
:10C290002CF804000020019014F00300241AB16B64
:10C2A000F06B0019814203D2B16BF06B091A0C00DC
:10C2B000002C18D1A04F002038602800FEF786FF20
:10C2C00000280DD105AB9D4890E8061083E80610C4
:10C2D000707B8DF81B0005A8FFF716FB0620386061
:10C2E000002001905CE001208DF800002800FFF79D
:10C2F0004DF96B4601AA2100914F3F69B8470028CC
:10C300001ED001283DD07FF00101884234D0B0F129
:10C31000FF3F45D10020019002AB8A4890E886009B
:10C3200083E88600707B8DF80F0002A8FFF7ECFA17
:10C330002800FFF738F97FF002007F4908602FE0FE
:10C340009DF8000086F84000019800280BD0F16BA2
:10C3500001984118F1630198001D96F83C1011F006
:10C360000301401A0190F06BB0633000FFF771F9E0
:10C3700000207149086013E05FF0FF306E490860EB
:10C380000EE0F16B01984118F163002086F840003F
:10C39000F06BB0633000FFF75CF90521664801607F
:10C3A00001992800FEF750FF002086F848006248F7
:10C3B000006809B0F0BD0000A0940108589601087B
:10C3C000F0B587B006000D002800FEF78EFF0400D0
:10C3D00000200090002C1AD1574F00203860280010
:10C3E000FEF7F4FE00280FD104ABDFF85CC19CE837
:10C3F000070083E8070096F856008DF8170004A898
:10C40000FFF7EFFA06203860002000904EE0280089
:10C41000FFF7BCF816F155036A462100484F7F69C3
:10C42000B84700281FD0012833D07FF0010188428F
:10C430002AD0B0F1FF3F39D10020009001AF43482E
:10C4400090E80E0087E80E0096F856008DF80B0075
:10C4500001A8FFF7C6FA2800FFF7A5F87FF0020150
:10C460003548016022E0012086F854000098002839
:10C4700003D0316D0098411831653000FFF727F97E
:10C4800000212D48016011E05FF0FF312A48016072
:10C490000CE0316D009841183165002086F8540099
:10C4A0003000FFF714F905212348016000992800A6
:10C4B000FEF7CAFE002086F85C001F48006807B03F
:10C4C000F0BD10B504002079002810D00020E071E4
:10C4D00001206071012020710020A0712000FFF771
:10C4E00013FA2000FFF7B2F92000FFF77AFA144898
:10C4F00040688047002801D1002001E05FF0FF3054
:10C5000010BD000030000000189201087C96010860
:10C51000C8940108B4970108A0960108D4970108AF
:10C52000AC080020B8080020C4080020D008002073
:10C5300090820108DC080020203B00209CA3010819
:10C5400034970108A8A30108B4A30108C0A30108F7
:10C5500070477047704710B50400207800280BD052
:10C56000022811D00CD3042816D011D306281BD0D2
:10C5700016D307281CD01FE02000FFF7E8FC1DE0C1
:10C580002000FFF7BAFC19E02000FFF7F5FB15E0EB
:10C590002000FFF7DCFC11E02000FFF7B5F90DE00B
:10C5A0002000FFF753F909E02000FFF71AFA05E031
:10C5B0002000FFF786FF01E07FF0090010BD0405B1
:10C5C00010B402000023002A03D1002010240C60C4
:10C5D00009E01F2A03D12E2010240C6003E012F181
:10C5E0000F0001240C6010BC70470100112907DB0B
:10C5F0001A2905DA012011F00F01491E88400BE0CD
:10C600000800102802D0202802D004E0002003E017
:10C610004FF4007000E00020704780B50A20DFF87A
:10C620008C1BD1F89C108847002801D0002001E025
:10C630007FF0050002BD10B50400200080B2DFF8D5
:10C640006C1BD1F89C108847002801D0002001E025
:10C650007FF0050010BD3EB50024DFF8505B684652
:10C66000E96888479DF800008DF805009DF80000F6
:10C6700010F00100002802D07FF00C00BFE09DF810
:10C680000000C0B2C009C0B2002802D07FF00C0088
:10C69000B5E00020E96E884702909DF80A00402826
:10C6A0000CD09DF80000C0F34000C0B2002805D0B7
:10C6B0009DF8000010F0FD008DF800009DF80000CE
:10C6C000C0F38010C0B2002805D09DF8000010F023
:10C6D000BF008DF800009DF805109DF8000090EA5D
:10C6E000010F08D0686880476846A96988470DF13E
:10C6F0000500E96888479DF805009DF8001091EA5B
:10C70000000F02D07FF00C0079E00DF102002969E2
:10C7100088479DF802008DF804009DF80200C0F3E0
:10C720008000C0B2002805D19DF8020050F004003E
:10C730008DF802009DF80200C0F34110C0B203283A
:10C7400005D09DF8020050F060008DF802009DF8C1
:10C7500004109DF8020090EA010F08D06868804735
:10C760000DF10200E969884701A8296988479DF809
:10C7700004109DF8020090EA010F02D07FF00C0037
:10C780003DE00DF10100A96888479DF801008DF892
:10C7900003009DF80100C0B2C009C0B2002805D056
:10C7A0009DF8010010F07F008DF801009DF8010058
:10C7B000C0F38200C0B2002805D09DF8010010F03F
:10C7C000E3008DF801009DF803009DF8011091EA47
:10C7D000000F09D0686880470DF10100696988473A
:10C7E0000DF10300A96888479DF803109DF801002A
:10C7F00090EA010F02D07FF00C0000E020003EBD67
:10C80000F8B504002000C0B2002804D0DFF89C096D
:10C81000806F804732E0DFF89459E86F8047070067
:10C82000002F02D55FF0FF3000E00020002801D08B
:10C83000380023E0FFF70FFF0600002E02D55FF05F
:10C84000FF3000E00020002801D0300016E000207A
:10C8500000F034FA0700002F02D55FF0FF3000E04F
:10C860000020002801D0380008E00A20D5F89C10EC
:10C870008847002801D1380000E00020F2BDF8B55B
:10C8800004000D00DFF82469D6F880008047070017
:10C89000002F02D55FF0FF3000E00020002809D013
:10C8A0002800C0B2002803D0D6F89400804701E0E9
:10C8B000380009E02000C0B2002803D0706D804726
:10C8C000002001E07FF00600F2BD70B586B00600E2
:10C8D0000C001500002C04D0002D02D02888002860
:10C8E00002D17FF006003FE13000C0B200281DD029
:10C8F000022800F08E8019D3042817D0C0F0898058
:10C90000062813D012D3082800F00681C0F0D28088
:10C910000A2800F01A81C0F00B810C2800F0AF80CB
:10C92000C0F0ED800E2867D059D31BE10020DFF85E
:10C930007C18C96E884700903000C0B2002808D02B
:10C94000012813D004282FD005283AD006281AD061
:10C9500044E02888022802D27FF0090004E1BDF8F3
:10C9600000002080022028800020FDE02888022886
:10C9700002D27FF00900F7E0BDF80200208002201B
:10C9800028800020F0E02888042802D27FF00900E7
:10C99000EAE09DF8030010F03F00FFF726FE20605C
:10C9A000042028800020DFE02888042802D27FF0BD
:10C9B0000900D9E05FF4F0102060042028800020F6
:10C9C000D2E02888042802D27FF00900CCE05FF48E
:10C9D00000102060042028800020C5E0C2E02888E4
:10C9E000042802D27FF00900BEE05FF4003020602E
:10C9F000042028800020B7E02888042802D27FF095
:10CA00000900B1E05FF400102060042028800020BD
:10CA1000AAE03000C0B2022819D003282CD12888FF
:10CA2000002802D17FF009009EE00020CDF805002B
:10CA300000208DF804006846DFF87017C96E88473B
:10CA40009DF8040020700120288000208CE02888B8
:10CA5000002802D17FF0090086E0CDF80540288843
:10CA60008DF804006846DFF84417C96E88479DF8C2
:10CA700004002880002077E07FF0090074E0288817
:10CA8000002814D0DFF82407D0F898008047002849
:10CA900002D45FF0FF3000E00020002801D0012028
:10CAA00000E0002020700120288000205CE07FF062
:10CAB000090059E0288800281ED003A800F005F9D5
:10CAC0000100002902D45FF0FF3000E000200028C0
:10CAD00010D00498002807D00398002804D0012023
:10CAE00028800120207003E0012028800020207091
:10CAF000002039E0080037E07FF0090034E02888A2
:10CB0000032806D24FF48050208002202880002085
:10CB10002AE07FF0090027E02888022805D320209A
:10CB200020800220288000201EE07FF009001BE00A
:10CB30002888032806D24FF4007020800220288025
:10CB4000002011E07FF009000EE02888032806D2BB
:10CB50004FF40070208002202880002004E07FF045
:10CB6000090001E07FF0060006B070BD7CB504004E
:10CB70000D007FF00506FFF750FDB04201D13000F7
:10CB800094E0002C08D12800C0B2012801D1002077
:10CB90008CE000F00DFB89E0207AC0B24008C0B202
:10CBA000002802D07F280DD01EE001A90020DFF868
:10CBB000FC25D2F8882090470090009800F0B1FA48
:10CBC000002114E02800C0B2002802D07FF0060047
:10CBD0006CE0207A10F00100002802D07FF00600FF
:10CBE00064E000F0E5FA61E07FF006005EE02029F5
:10CBF00029D20800C008225C11F00700D2B2C2405E
:10CC0000D0071ED52800C0B200280DD1009A080018
:10CC1000C008125C012311F0070083409A43009B77
:10CC20000800C0081A540CE0009A0800C008125C02
:10CC3000012311F0070083401A43009B0800C0083D
:10CC40001A54491CD3E7009800F02DFA009800F020
:10CC500068FA00211E2928D20800C008205C11F0C3
:10CC60000702C0B2D040C0071DD52800C0B20028BE
:10CC70000CD1009A0800C008125C11F00700D2B273
:10CC8000C240D0070FD57FF007000FE0009A0800E0
:10CC9000C008125C11F00700D2B2C240D00702D423
:10CCA0007FF0070002E0491CD4E7002076BD10B5F4
:10CCB000040001212000FFF759FF10BD10B504004A
:10CCC00000212000FFF752FF10BD7CB504007FF06B
:10CCD00006057FF00506FFF7A0FCB04201D1300049
:10CCE00044E001A90020DFF8C424D2F8882090474E
:10CCF0000090009800F015FA4BF6EF60002C03D07E
:10CD0000217A11F0FE0121720022202A2ED2009BEE
:10CD10001100C9085B5C12F00701DBB2CB40D907F8
:10CD200015D54DF6ED610800002C0FD0217A51F099
:10CD3000010121721100C908635C012512F007018D
:10CD40008D402B431100C90863540DE00EE0002C08
:10CD50000AD01100C908635C012512F007018D405B
:10CD6000AB431100C9086354521CCEE776BD2DE9D0
:10CD7000F84306000F001400002C02D17FF00600DB
:10CD800096E03000C0B2002805D0022811D010D3A0
:10CD9000032866D088E0B7F5003F02D27FF0060096
:10CDA00086E0E119DFF8F004814202D37FF006004B
:10CDB0007EE0002200213000C0B200280ED1E01930
:10CDC000000501D0012500E00025E019000BB0EBC3
:10CDD00017302D18B8465FEA18380EE0202F02D21F
:10CDE0007FF0060064E0E31940F20120834202D3A1
:10CDF0007FF006005CE02500B846002D30D0DFF85B
:10CE0000AC93D9F80400804718F00F0F15D1102DFE
:10CE100013D34046000980B2D9F8681088474FF410
:10CE2000FA60FFF708FC10F1060F02D17FF01F0037
:10CE30003EE018F11008103DDFE7404680B2D9F817
:10CE4000641088474FF4C870FFF7F5FB10F1060F28
:10CE500002D17FF01F002BE018F101086D1ECCE716
:10CE600025E0032F02D27FF0060021E0E0192128FF
:10CE700002D37FF006001BE0002C14D0DFF82C5307
:10CE800068688047380080B2A96E88474FF4FA601E
:10CE9000FFF7D1FB10F1060F02D17FF01F0007E072
:10CEA0007F1C641EE8E702E07FF0060000E000203F
:10CEB000BDE8F2832DE9FC4F85B082460D001600D7
:10CEC000BAF5003F02D27FF00600ABE0002E01D0A1
:10CED000002D02D17FF00600A4E016EB0A01DFF876
:10CEE000B803814202D37FF006009BE000208DF85A
:10CEF00000009DF81800002802D0012804D004E0AA
:10CF000001208DF8000003E002E07FF0060089E0D8
:10CF100057463F0B16EB0A00000501D0012400E044
:10CF2000002416EB0A00000BB0EB1A3024185FEA5D
:10CF30000A585FEA1858D8F58058DFF8709202A9AD
:10CF40000320D9F8882090470190464500D2B0468A
:10CF50005FEA0A5001D1022C18D2029A92B20199CA
:10CF60005FEA0A50000DBAEB0000D9F85C30984730
:10CF7000CDF81080039501995FEA0A50000D01EB8E
:10CF8000000B049A03995846F4F79EFFD9F8040061
:10CF90008047380080B2D9F8641088474FF4C870D1
:10CFA000D9F89C108847002802D55FF0FF3000E0D8
:10CFB0000020002802D07FF01F0033E0390001A8D4
:10CFC00000F02BF9002802D55FF0FF3000E00020D0
:10CFD000002802D07FF01F0024E09DF80000002808
:10CFE00010D0424692B201995046D9F85C30984729
:10CFF00042462900019800F053F9002802D07FF042
:10D0000008000FE07F1C18EB0A0A4544B6EB08063F
:10D010005FEA0A50000DD0F580508046641E002C57
:10D0200093D1002007B0BDE8F08FF8B506000C00E2
:10D030001500B6F5003F02D27FF006001DE0002C7F
:10D0400001D0002D02D17FF0060016E0A919924808
:10D05000814202D37FF006000FE07FF00507FFF763
:10D06000DCFAB84201D1380007E02A0092B2210070
:10D0700030004E4BDB6D98470020F2BD80B54B4829
:10D08000406D8047002002BD10B5484CA06D804720
:10D090000A20D4F89C108847002801D0002001E025
:10D0A0007FF0050010BD2DE9F8430400002C02D1EB
:10D0B0007FF0060033E00025202D2FD200200090C5
:10D0C00069462800FFF77CFA0600370000988019AF
:10D0D000874221D22800C00814F8008015F007000C
:10D0E0005FFA88F838FA00F818F00108DFF8BC9009
:10D0F000D9F8040080474146C9B23800D9F84C201D
:10D1000090477FF005090320FFF795FA484501D1C4
:10D11000484604E07F1CD9E76D1CCDE70020BDE840
:10D12000F2832DE9FC410400002C02D17FF00600BF
:10D1300039E00025202D35D20020009069462800D6
:10D14000FFF73EFA06000027B04600988019804598
:10D150000BD240461549096D8847002802D00120AE
:10D16000070002E018F10108EFE73800C0B200281C
:10D170000BD02800C008215C012215F00700824076
:10D1800011432800C00821540AE02800C008215C8F
:10D19000012215F00700824091432800C008215465
:10D1A0006D1CC7E70020BDE8F6810000E0790108AA
:10D1B0003EB53A4C60688047A06C80477FF005051B
:10D1C0000320FFF738FAA84201D1280024E001A982
:10D1D0000020D4F88820904700900098002802D0C2
:10D1E0000198052802D27FF0090015E00098FFF7AA
:10D1F00098FF002120290ED2009A0800C008125C76
:10D2000011F00700D2B2C240D00702D57FF007006C
:10D2100002E0491CEEE700203EBD2DE9F843040082
:10D220000D0026684FF4805707FB05F7DFF86C8088
:10D23000D8F898008047002802D55FF0FF3000E062
:10D240000020002802D07FF01F0023E05FF00009DB
:10D25000606881451DD2D8F804008047390030004D
:10D26000D8F8602090470320D8F89C108847002801
:10D2700002D55FF0FF3000E00020002802D07FF0F0
:10D280001F0007E017F5807719F5807916F580768D
:10D29000DEE70020BDE8F28301002000E07901080C
:10D2A0000300002013F0030F09D0521E22BF13F811
:10D2B000010B11F801CBB0EB0C00F3D0704711F06B
:10D2C000030F14D1121F22BF53F8040B51F804CBE3
:10D2D0006045F7D0121D0AD200BA9CFA8CFCB0EB64
:10D2E0000C0038BF6FF0000088BF01207047521E4D
:10D2F00022BF13F8010B11F801CBB0EB0C00F6D0F4
:10D30000521C08BF10467047F8B5040020688569B4
:10D31000206846692068476894F83E00102803D0CA
:10D3200094F83E0040284ED116F0011F05D0B805F4
:10D3300003D5200000F03BFA12E0DFF8840A064231
:10D3400005D0B80503D5200000F078FA08E0DFF832
:10D35000740A064204D0B80502D5200000F075FA20
:10D36000206D002819D1DFF8600A054215D0DFF8DA
:10D370005C0A064208D0780506D56A48064203D101
:10D38000200000F064F861E0664806425ED0B8050F
:10D390005CD5200000F0C8F858E0DFF8340A0642F7
:10D3A00008D0780506D55F48064203D1200000F07A
:10D3B0000FF94BE05B48064248D0B80546D520003F
:10D3C00000F075F942E0DFF8FC09064205D0B80527
:10D3D00003D5200000F0A8FB38E0DFF8F80906428A
:10D3E00005D0B80503D5200000F0B8FB2EE0DFF82B
:10D3F000D809054215D0DFF8D409064208D07805CF
:10D4000006D54848064203D1200000F025FB1DE068
:10D41000444806421AD0B80518D5200000F041FB58
:10D4200014E0DFF8AC09064208D0780506D53D487F
:10D43000064203D1200000F043FB07E039480642D2
:10D4400004D0B80502D5200000F05FFBF1BD10B597
:10D450000400208D002843D194F83D0021283FD1BD
:10D46000E06A042819D0E06A082816D0E16ADFF8DB
:10D47000E405814211D02068416831F4E061206800
:10D48000416011202063002084F83E00202084F8B1
:10D490003D00200000F0D9FC41E02068416831F4F3
:10D4A000E061206841602068006850F400702168E5
:10D4B000086000202063202084F83D0094F83E009E
:10D4C000402806D1002084F83E00200000F0BEFC79
:10D4D00025E0002084F83E00200000F0B6FC1EE0AD
:10D4E00094F83D00212807D094F83E00402816D13A
:10D4F00094F83D00222812D1608D002806D12068C2
:10D50000416831F480612068416008E0616A481C2C
:10D510006062097820680161608D401E608500208E
:10D5200010BD00000400010010B5040094F83D0097
:10D5300021284BD1608D002809D0616A481C6062A7
:10D54000097820680161608D401E60853EE0E06AD8
:10D55000042819D0E06A082816D0E16ADFF8F4043C
:10D56000814211D02068416831F4E0612068416057
:10D5700011202063002084F83E00202084F83D0024
:10D58000200000F062FC21E02068416831F4E06195
:10D59000206841602068016851F4007120680160D2
:10D5A00000202063202084F83D0094F83E004028AD
:10D5B00006D1002084F83E00200000F047FC05E082
:10D5C000002084F83E00200000F03FFC002010BD49
:10D5D00010B5040094F83D00222866D1608D04281F
:10D5E00009D3606A411C6162216809690170608D1C
:10D5F000401E608559E0608D022802D0608D0328AE
:10D600001CD1E06A02280CD02068016831F48061E6
:10D61000206801602068016851F4006120680160A1
:10D6200005E02068016851F480612068016020688D
:10D63000416831F480612068416036E0E06A022888
:10D6400006D02068006830F480602168086005E03A
:10D650002068016851F48061206801602068416899
:10D6600031F4E06120684160606A411C61622168B8
:10D6700009690170608D401E6085202084F83D009E
:10D6800094F83E00402808D100202063002084F850
:10D690003E00200000F0DBFB07E0122020630020AA
:10D6A00084F83E00200000F0D3FB002010BD10B530
:10D6B0000400608D03281AD1E06A042807D0E06ACC
:10D6C000082804D0E16ADFF88C03814205D1206884
:10D6D000016831F4806120680160606A411C616208
:10D6E000216809690170608D401E60855DE0608D74
:10D6F000022851D1E06A042817D0E06A082814D023
:10D70000E06AD449884210D0E06A022806D0206836
:10D71000006830F48060216808600CE020680168CF
:10D7200051F480612068016005E02068016851F4CF
:10D73000007120680160606A411C616221680969AA
:10D740000170608D401E6085606A411C61622168C5
:10D7500009690170608D401E60852068416831F460
:10D76000407120684160202084F83D0094F83E001C
:10D77000402808D100202063002084F83E002000CB
:10D7800000F065FB11E012202063002084F83E00C9
:10D79000200000F05DFB08E0606A411C61622168C6
:10D7A00009690170608D401E6085002010BD010078
:10D7B00091F83E0040280FD1086D002805D14A6C31
:10D7C00012F0FE020868026136E04A6C52F0010273
:10D7D000D2B2086802612FE00869B0F5804F10D11D
:10D7E00091F83D00212805D14A6C12F0FE0208682C
:10D7F000026121E04A6C52F00102D2B20868026173
:10D800001AE0086D00280AD14A6C92B2D20912F0CF
:10D81000060252F0F002D2B2086802610CE0086D14
:10D82000012809D14A6C92B2D20912F0060252F0D4
:10D83000F102D2B2086802610020704701004A6C10
:10D84000D2B2086802610020704781B0010091F8EF
:10D850003D00222840F0F180086D00280DD191F89C
:10D860003E00402809D100200090086840690090DF
:10D870000868806900900098E8E0086D002816D1DB
:10D880000869B0F5404F12D1002000900868406947
:10D89000009008688069009000980868026852F457
:10D8A000807208680260086D401C0865CEE0488DF3
:10D8B00000280FD100200090086840690090086897
:10D8C0008069009000980868026852F40072086845
:10D8D0000260AFE0488D012866D1CA6A5D48824285
:10D8E00029D10868026832F480620868026008681A
:10D8F000406800050FD50868026832F48062086845
:10D900000260002000900868406900900868806903
:10D91000009000988EE00020009008684069009018
:10D9200008688069009000980868026852F40072E4
:10D93000086802607EE0C86A04281FD0C86A082808
:10D940001CD0086B122819D0C86A022806D00868B3
:10D95000006830F480600A68106005E008680268BA
:10D9600052F48062086802600020009008684069F4
:10D97000009008688069009000985BE00868026881
:10D9800032F48062086802600020009008684069F4
:10D99000009008688069009000980868026852F456
:10D9A00000720868026045E0488D022829D1C86AE3
:10D9B00002280CD00868026832F4806208680260AD
:10D9C0000868026852F400620868026005E00868AE
:10D9D000006850F480600A681060086840680005BC
:10D9E00005D50868426852F48052086842600020F9
:10D9F000009008684069009008688069009000986D
:10DA000018E00868026852F48062086802600868DA
:10DA10004068000505D50868426852F480520868DD
:10DA200042600020009008684069009008688069A2
:10DA3000009000980020086508E000200090086829
:10DA4000406900900868806900900098002001B04B
:10DA5000704700000000FFFF10B50400608D002833
:10DA60001DD0616A481C6062097820680161608D80
:10DA7000401E6085608D002811D194F83D00292852
:10DA80000DD12068416831F4806120684160212017
:10DA90002063282084F83D00200000F0DAF90020FF
:10DAA00010BD0100488D002808D04A6A501C486209
:10DAB000127808680261488D401E48850020704732
:10DAC00010B50400608D00281DD0606A411C6162A1
:10DAD000216809690170608D401E6085608D002895
:10DAE00011D194F83D002A280DD12068416831F405
:10DAF00080612068416022202063282084F83D0056
:10DB0000200000F0A7F9002010BD0100488D00287A
:10DB100008D0486A421C4A620A6812690270488D3D
:10DB2000401E48850020704770B504000025002085
:10DB300021688969490701D401210D00216889699B
:10DB4000090601D4E66800E0A669320092B2290015
:10DB5000C9B2200000F07FF9002070BD1CB50400A0
:10DB60002068416831F4E061206841600020009045
:10DB70002068406900902068016851F00101206828
:10DB8000016000982068016831F4806120680160BC
:10DB900020684068000510D594F83D00222803D085
:10DBA00094F83D002A2804D1A06B00684068608585
:10DBB00003E0606B006840686085608D00281DD0C0
:10DBC00020684069400708D5606A411C616221688D
:10DBD00009690170608D401E6085206840694006BB
:10DBE00008D5606A411C6162216809690170608D15
:10DBF000401E6085206C50F004002064206C0028DA
:10DC000003D0200000F030F82CE094F83D002828E4
:10DC100007D094F83D002A2803D094F83D00292825
:10DC20000ED1DFF8B401E06200202063202084F8E8
:10DC30003D00002084F83E00200000F00DF911E0C6
:10DC4000206B222803D094F83D0022280AD100201E
:10DC50002063202084F83D00002084F83E0020004E
:10DC600000F0F8F8002016BD38B5040094F83D50D7
:10DC7000292D01D02A2D05D100202063282084F8E9
:10DC80003D000FE094F83D00602806D02068406811
:10DC9000000502D4202084F83D00002020630020ED
:10DCA00084F83E002068016831F40061206801605A
:10DCB00020684068000542D52068416831F4006161
:10DCC00020684160606B90F82100012816D00FF2A7
:10DCD0000D11606B4163606B00F0C0F8002858D0F4
:10DCE000206800684008400021680860202084F80F
:10DCF0003D00606B616B496B88474AE00FF2DD01C4
:10DD0000A06B4163A06B00F0A9F8002841D0206807
:10DD10004069400605D5606A411C61622168096955
:10DD200001702068016849084900206801602020CE
:10DD300084F83D00A06BA16B496B884729E094F8FB
:10DD40003D00602818D1202084F83D000020206488
:10DD500020684069400605D5606A411C61622168FF
:10DD6000096901702068016849084900206801605C
:10DD7000200000F09FF80CE020684069400605D5BF
:10DD8000606A411C6162216809690170200000F02D
:10DD900092F894F83D00282810D1206C40070DD54A
:10DDA000DFF83400E06200202063202084F83D008A
:10DDB000002084F83E00200000F04EF831BD000045
:10DDC00008000100020001000400020080000100C0
:10DDD00040000100100001000000FFFF38B5040002
:10DDE000656A2868016831F4806128680160002054
:10DDF00068850021686B41630021A86B416395F839
:10DE00003D00602811D1202085F83D00002085F8D4
:10DE10003E000020286428680168490849002868F5
:10DE20000160280000F046F80EE0202085F83D0053
:10DE3000002085F83E0028680168490849002868E4
:10DE40000160280000F037F831BD70477047704717
:10DE500070477047704770477047070138B5040036
:10DE6000002594F82100022804D00420A06301209A
:10DE700005001CE02068016831F00E012068016097
:10DE80002068016849084900206801600121206C70
:10DE90008140E06B4160012084F82100002084F87B
:10DEA0002000606B002802D02000616B88472800AA
:10DEB000C0B232BD7047704710B504002100C9B22E
:10DEC0000020DFF808255269904710BD80B500207A
:10DED0008DF8000069460020DFF8F0249269904731
:10DEE000002802D09DF8000000E0002002BD70B5BF
:10DEF00004000D00002C01D0802D01D2002013E081
:10DF0000DFF8C804006A066880222100300001F0B2
:10DF1000E5F8002802D45FF0FF3000E00020002880
:10DF200001D0200000E0002070BD2DE9F84304007E
:10DF30000E005FF00008002C0FD101208046DFF8B2
:10DF400034060078012802D1DFF8845432E0DFF88B
:10DF5000800404004FF480600600002C01D0802E65
:10DF600001D2002027E04046C0B2002803D00021A3
:10DF7000DFF80006017031002000FFF7B8FF050050
:10DF8000002D01D1002016E0FCF7C2FB81467C2267
:10DF900029004846FCF7C3FB0700E86F874201D021
:10DFA000002008E04046C0B2002803D00121DFF87D
:10DFB000C40501702800BDE8F2830300DFF81004F7
:10DFC000704770B504000D00002C01D0802D01D2E7
:10DFD000002014E0DFF8A005006A06680023802214
:10DFE0002100300001F094F8002802D45FF0FF30E7
:10DFF00000E00020002801D0200000E0002070BDDB
:10E000002DE9F14F82B0DFF8C8434FF48066002C51
:10E0100001D0802E01D2002042E00021DFF8E0068E
:10E02000017031002000FFF762FF0500002D1FD1B5
:10E0300025000A2001903020009015F14007009A39
:10E0400001993800F3F700FF5FF0400B0027A84666
:10E050003A0059464046F3F7F7FE5FF030085FF0AC
:10E06000000915F14C0A4A4641465046F3F7ECFECA
:10E070009DF80800A5F84A00FCF74AFB80467C2280
:10E0800029004046FCF74BFB0700EF6731002000FA
:10E09000FFF797FF0100002901D1002000E00120D7
:10E0A000BDE8FE8F2DE9F14F82B0C94C4FF4806678
:10E0B000002C01D0802E01D2002049E00021DFF8A1
:10E0C0004006017031002000FFF711FF0500002D10
:10E0D0001FD125000A2001903020009015F1400743
:10E0E000009A01993800F3F7AFFE5FF0400B00276C
:10E0F000A8463A0059464046F3F7A6FE5FF03008BE
:10E100005FF0000915F14C0A4A4641465046F3F7C4
:10E110009BFE0A270298009015F140083A000099EA
:10E120004046F3F7D1FEFCF7F3FA81467C22290042
:10E130004846FCF7F4FA8046C5F87C8031002000A0
:10E14000FFF73FFF0100002901D1002000E001207E
:10E15000BDE8FE8F0200002A01D0502901D2002024
:10E1600009E0DFF860070068D0F81C01002801D141
:10E17000002000E0002070472DE9F84304000E0065
:10E180005FF00008002C0DD101208046DFF87005FB
:10E190000078032801D18E4D31E08D4804004FF402
:10E1A00080600600002C01D0502E01D2002027E014
:10E1B0004046C0B2002803D00021DFF844050170BA
:10E1C00031002000FFF7C6FF0500002D01D100201F
:10E1D00016E0FCF79DFA81464C2229004846FCF7E0
:10E1E0009EFA0700E86C874201D0002008E0404614
:10E1F000C0B2002803D00321DFF804050170280015
:10E20000BDE8F28302000020704738B504000D001D
:10E210002900C9B22000C0B2DFF8A8261268D2F8DF
:10E22000E420904732BD10B40400002010BC7047B9
:10E230002DE9FE4F0400002C0BD06068002808D0A8
:10E24000A068002805D02069002802D0E0680028D6
:10E2500005D1002C01D00120A0610020B3E0D4F84A
:10E260000C9019F104095FF00608206808FB00997A
:10E270000020C049087000256068854280F0A080B9
:10E28000AA266068401BB04202D26068401B0600AC
:10E290004F4F08FB06F23900484600F01FFF0028E8
:10E2A00002D45FF0FF3000E00020002803D10420FA
:10E2B000A061002087E001970027B7427CD2019936
:10E2C00008FB07F0095A019A08FB07F01044807810
:10E2D00051EA0041080206D581F0FF1191F47F4117
:10E2E000491C4942FFE7A0687A19120110440090C6
:10E2F0000800F4F729FE82468B46B4F91600B4F9FB
:10E300001410401AF4F720FE0022DFF8BC35F4F7B1
:10E31000EFFA5FF06042DFF8B435F4F7E9FA5246FD
:10E320005B46F4F7D7F982468B46B4F91600B4F988
:10E3300014100818F4F708FE0022DFF89435F4F7FB
:10E34000D7FA52465B46F4F711FE009AC2E9000183
:10E350000021019808FB07F21044B0F80300019A6D
:10E3600008FB07F31A44527950EA0240020206D52C
:10E3700080F0FF1090F47F40401C4042FFE7A1680E
:10E380007A19120101EB020AF4F7DEFD5FF0404258
:10E39000DFF84035F4F7ACFADFF83C25DFF83C3520
:10E3A000F4F798F9DFF83825DFF83835F4F792F903
:10E3B000CAE902017F1C80E7751908FB06995BE733
:10E3C0000020A0616068BDE8FE8F000060050020AD
:10E3D000542E002010B40400002010BC704710B46C
:10E3E0000400002010BC70472DE9F04F87B0814633
:10E3F000B9F1000F0FD0D9F8040000280BD0D9F8DC
:10E400000800002807D0D9F81000002803D0D9F858
:10E410000C00002807D1B9F1000F02D00120C9F883
:10E4200018000020A2E0D9F80C00001DD9F8001057
:10E4300010EB4100059000214E4801700020039030
:10E440000399D9F80400814280F08B804FF400706A
:10E450000490D9F804100398091A0498814204D250
:10E46000D9F804100398091A0491DFF87C44049841
:10E4700042002100059800F031FE002802D45FF030
:10E48000FF3000E00020002804D10420C9F8180063
:10E4900000206BE006945FF000080498804556D297
:10E4A000B9F91600F4F750FD0022DFF81C34F4F738
:10E4B0001FFA06000F00B9F91400F4F745FD002219
:10E4C000DFF80434F4F714FA04000D0032003B00C6
:10E4D00020002900F4F74AFD00225FF08043F4F7A2
:10E4E00007FA82468B46D9F80800039918EB010118
:10E4F000090100EB010200200021C2E90201D9F864
:10E500000800039918EB01010901084400900698DE
:10E5100030F91800F4F718FDCDE901013000390099
:10E5200022002B00F4F7E0FDDDE90123F4F7D2F837
:10E530000022DFF8B833F4F7DBF952465B46F4F714
:10E5400015FD009AC2E9000118F10108A5E7039939
:10E550000498411803910598049910EB4100059027
:10E560006EE70020C9F81800D9F8040007B0BDE82C
:10E57000F08F0000363B0020600500202DE9F04FB1
:10E5800087B08146B9F1000F0FD0D9F804000028F8
:10E590000BD0D9F80800002807D0D9F810000028BF
:10E5A00003D0D9F80C00002807D1B9F1000F02D030
:10E5B0000120C9F8180000209EE0D9F80C00001DC9
:10E5C000D9F8001010EB4100059000214C48017073
:10E5D000002003900399D9F80400814280F08780DD
:10E5E0004FF400700490D9F804100398091A0498A5
:10E5F000814204D2D9F804100398091A0491BA4C44
:10E60000049842002100059800F068FD002802D41B
:10E610005FF0FF3000E00020002804D10420C9F89A
:10E620001800002068E006945FF000080498804518
:10E6300053D2B9F91600F4F787FC0022A24BF4F785
:10E6400057F906000F00B9F91400F4F77DFC002219
:10E650009D4BF4F74DF904000D0032003B00200003
:10E660002900F4F783FC00225FF08043F4F740F9BF
:10E6700082468B46D9F80800039918EB010109017D
:10E6800000EB010200200021C2E90001D9F80800D6
:10E69000039918EB0101090108440090069830F92C
:10E6A0001800F4F751FCCDE90101300039002200D7
:10E6B0002B00F4F719FDDDE90123F4F70BF8002234
:10E6C0008A4BF4F715F952465B46F4F74FFC009A73
:10E6D000C2E9020118F10108A8E70399049841185A
:10E6E00003910598049910EB4100059072E7002012
:10E6F000C9F81800D9F8040007B0BDE8F08F000091
:10E70000363B00202DE9F04104000F0015006D4953
:10E710000868D0F81C610868D0F81C01002847D0B0
:10E720003069002844D0002C42D0306987423FD263
:10E73000002D3DD00868D0F81C01C068C019002821
:10E740000DD40868D0F81C01C068C01920F0004042
:10E750006749096AD1F8008018EB000819E00868D9
:10E76000D0F81C01C068C019002810D5604A08689C
:10E77000D0F81C01C168C91921F00041106A006875
:10E780004118506AD0F8008018EB010801E05FF0F2
:10E7900000082A002100404600F0A0FC002802D416
:10E7A0005FF0FF3000E00020002801D0280000E0EA
:10E7B0000020BDE8F08143480168D1F81C110068D1
:10E7C000D0F81C01002801D0086900E00020704743
:10E7D00010B590B0FFF7EFFF402816D1402200217E
:10E7E0006846FFF78FFF00280DD0FBF791FF04006C
:10E7F0003C2269462000FBF792FF01000F988142FE
:10E8000001D0002002E0012000E0002010B010BD87
:10E810002DE9F04104000F0015002A490868D0F8DE
:10E820001C610868D0F81C01002848D03069002815
:10E8300045D0002C43D03069874240D2002D3ED0D5
:10E840000868D0F81C01C068C01900280DD40868F9
:10E85000D0F81C01C068C01920F000402449096AA2
:10E86000D1F8008018EB000819E00868D0F81C0106
:10E87000C068C019002810D51D4A0868D0F81C01CE
:10E88000C168C91921F00041106A00684118506A36
:10E89000D0F8008018EB010801E05FF000080023C9
:10E8A0002A002100404600F033FC002802D45FF02B
:10E8B000FF3000E00020002801D0280000E0002008
:10E8C000BDE8F0812C07002000005940FFFF6F4198
:10E8D00000006940FFFF5F41182D4454FB210940AF
:10E8E000F8C1631ADCA54C40542E0020E0FFEF4035
:10E8F00060050020030000207047030000207047DF
:10E900000200002070470200002070470200002033
:10E91000704702000020704710B504000021DFF8A6
:10E9200034080170DFF830281068002810D021006A
:10E93000C9B2012012681268126B9047002802D5F4
:10E940005FF0FF3000E00020002801D0002020E030
:10E95000DFF808084068804700F053F9DFF8000846
:10E96000DFF800184160DFF800188160DFF8FC175D
:10E97000C160DFF8FC170161DFF8F8174161DFF8CB
:10E98000F8178161DFF8F4170162DFF8F4174162CC
:10E99000012010BD38B50024002C13D1DFF8E45756
:10E9A000012055F8241089688847002802D45FF0B8
:10E9B000FF3000E00020002802D005EB840002E0D8
:10E9C000641CE9E7002032BDF8B5DFF88867002055
:10E9D000307000F0E1F8DFF8844720688047DFF806
:10E9E0007857FFF7D7FF28602868002805D100F086
:10E9F00008F960688047002096E028680068406B4E
:10EA0000006829680968496B4968884201D3002079
:10EA10008AE028680068406B8068002805D0286874
:10EA20000068406BC068002801D100207CE0DFF85E
:10EA300058175FF4602008605FF4801088602868D1
:10EA40000068406B0068486028680068406B026896
:10EA500008688218CA6008682A681268526BD3680E
:10EA6000B0FBF3F203FB1200002804D02868006812
:10EA7000406BC26800E0002288682B681B685B6BF3
:10EA8000DB68B0FBF3F703FB1700002804D028680D
:10EA90000068406BC76800E0002728680068406B8A
:10EAA000836828680068406BC0684343BA180868E8
:10EAB000821888688218934201D2002034E0DFF87F
:10EAC000A0060FF2ED4242600FF2355282600FF263
:10EAD0007D52C2600FF2BD5202610FF2812242618B
:10EAE0000FF2714282612A681268526B02624162BF
:10EAF00000202968096889688847002802D55FF0E6
:10EB0000FF3000E0002000280BD0012100202A68FF
:10EB10001268126B904700F074F86068804700201C
:10EB200002E001203070C0B2F2BDF0B4DFF8305620
:10EB300042682B6ADB68B2FBF3F34468026812197F
:10EB40002C6AE668B2FBF6F406FB1422002A01D018
:10EB5000012400E000244668026896192A6AD268F7
:10EB6000B6FBF2F2A4180025082D03D200224A5564
:10EB70006D1CF9E71D00A5420CD22A00D2088E5C5C
:10EB8000012715F0070297403E432A00D2088E5411
:10EB90006D1CF0E7F0BC704730B585B01421002241
:10EBA0006C462000F3F750F90420009000200190FB
:10EBB00000200290DFF8D45569462800F6F786FC5D
:10EBC00004212800F6F769FD0400042000900320CA
:10EBD00001900020029069462800F6F777FC220099
:10EBE000D2B204212800F6F763FD04200090112022
:10EBF00001900120029069462800F6F767FC05B0F5
:10EC000030BD18B585B0142100226C462000F3F702
:10EC10001BF9042000900320019000200290694617
:10EC2000DFF86805F6F752FC06B010BD2DE9FE438B
:10EC300081460F0014001D000026DFF81C85D8F85F
:10EC40000000002801D1002085E0002C00F0828027
:10EC50004846C0B2002802D001280AD013E0DFF8ED
:10EC6000300506003100DFF8F804406AFFF75DFF69
:10EC700009E0DFF81C0506003100DFF8E404406A13
:10EC80000830FFF752FF002E64D06846D8F8001015
:10EC9000096889698847002802D45FF0FF3000E0E6
:10ECA0000020002856D0009820600198606038004D
:10ECB000C0B2002802D05FF0FF3000E00020A0606A
:10ECC0003800C0B2002802D05FF0FF3000E0002022
:10ECD000E06021683068014021606168706801402F
:10ECE0006160A16830680140A160E168706801401E
:10ECF000E1602168A068814203D16168E0688142D7
:10ED000010D000206074002D0ED0287A10F0010081
:10ED10002872287A50F001002872306828607068E4
:10ED2000686001E0012060740020D8F800100968D4
:10ED3000896988474BF6EF61884207D04DF6ED614F
:10ED4000884207D101202074012004E000202074B3
:10ED5000012000E00020BDE8FE8300002DE9F8431B
:10ED600090B081460C00DFF8F0733868002801D1BC
:10ED70000020EBE04846C0B2002805D04846C0B2AB
:10ED8000012801D00020E1E000230BAA012100208E
:10ED9000FFF74CFF002800F0D880002306AA0121CD
:10EDA0000120FFF743FF002800F0CF809DF83D00D1
:10EDB000002805D09DF83C00002801D0012500E086
:10EDC00000259DF82900002805D09DF8280000287E
:10EDD00001D0012600E000264846C0B2002805D137
:10EDE00021002800C9B2C0B2814209D04846C0B251
:10EDF000012807D120003100C0B2C9B2884201D138
:10EE00000120A3E04846C0B2002802D12000C0B2D1
:10EE100001E02800C0B200280AD14846C0B201284B
:10EE200002D12000C0B201E03000C0B2002802D000
:10EE30005FF0010801E05FF000084046C0B2002822
:10EE400071D04846C0B2002802D12000C0B201E013
:10EE50002800C0B29DF83D10814222D09DF83D00AF
:10EE6000002801D1012500E0002503AB0BAA2900F1
:10EE7000C9B20020FFF7DAFE002801D1002065E0CA
:10EE80002900C9B203A83A6812685269904700285D
:10EE900002D55FF0FF3000E00020002801D0002004
:10EEA00054E04846C0B2012802D12000C0B201E0BF
:10EEB0003000C0B29DF82910814222D09DF829006F
:10EEC000002801D1012600E000266B4606AA310089
:10EED000C9B20120FFF7AAFE002801D1002035E0C9
:10EEE0003100C9B268463A681268526990470028F2
:10EEF00002D55FF0FF3000E00020002801D00020A4
:10EF000024E000203968096809688847002802D48D
:10EF10005FF0FF3000E00020002801D0012000E079
:10EF20000020C0B212E000203968096849688847AB
:10EF3000002802D45FF0FF3000E00020002801D05C
:10EF4000012000E00020C0B200E0002011B0BDE8C8
:10EF5000F083000030B585B005000C00002C16D001
:10EF600000236A4601212800C0B2FFF75FFE002897
:10EF70000DD09DF81000002805D09DF81100002844
:10EF800001D0012000E000202070012000E00020DE
:10EF900005B030BD80B5002204217C48F6F788FB1F
:10EFA00001BD80B5012204217848F6F781FB01BD3F
:10EFB000F8B504000D001600674F3868002801D12D
:10EFC00000201BE063480078002815D000233200A1
:10EFD000290038680068406B006820183F683F6867
:10EFE0003F6AB847002802D45FF0FF3000E00020FD
:10EFF000002801D0012000E00020C0B2F2BD0000D6
:10F0000070B504000D001600534B1868002801D19C
:10F0100000201AE04F480078002814D03200290060
:10F0200018680068406B006820181B681B685B6AE2
:10F030009847002802D45FF0FF3000E0002000284D
:10F0400001D0012000E00020C0B270BD10B4020069
:10F05000414B1868002801D1002019E018680068A9
:10F06000406B446818680068406B0068241A8C4242
:10F070000DD318680068406B446818680068406BDE
:10F080000068241A641AA24201D2012000E0002084
:10F0900010BC704710B402002F4B1868002801D133
:10F0A000002019E018680068406B44681868006820
:10F0B000406B0068241A8C420DD318680068406BBE
:10F0C000446818680068406B0068241A641AA242F9
:10F0D00001D2012000E0002010BC704770B5040090
:10F0E0000D0016001C4B1868002802D17FF00C00A0
:10F0F0000DE018480078002807D0320029002000D1
:10F100001B681B685B6A984701E07FF00C0070BDCC
:10F11000F8B504000D0016001F00DFF83CC0DCF855
:10F120000000002802D17FF00C0011E009480078AF
:10F1300000280BD00023320029002000DCF800C09A
:10F14000DCF800C0DCF820C0E04701E07FF00C00F4
:10F15000F2BD0000303B0020F83A002098980108EA
:10F1600060050020F5E80008FBE8000801E9000858
:10F1700007E900080DE9000813E90008EC98010808
:10F18000549E010870A70108CC3A002000040240F8
:10F19000E43A00200100002000291CD03E291AD2A8
:10F1A000102905D24FF4805202FB01F2100012E048
:10F1B000102909D32E2907D25FF4803202FB01F215
:10F1C000B2F57022100006E04FF4805202FB01F20B
:10F1D00012F5E112100070472DE9F84305000E000A
:10F1E0000024002030602800C0B2002805D002288A
:10F1F0000DD007D303280FD014E005203060DFF8CE
:10F20000A809040005203060DFF8A00904000820E8
:10F210003060DFF8940904004FF480503060DFF86C
:10F2200088090400002C0BD03068002808D0D6F8DC
:10F2300000900027A0463A0049464046F2F704FEF7
:10F240002000BDE8F28380B5DFF86409C06880471C
:10F250000120F6F73EFE01BD80B50120F6F739FE2C
:10F26000DFF84C09806880470120F6F732FE01BDC7
:10F270007CB50400684600F04BF89DF8000010F0E3
:10F280000100002804D1002000F061F801203EE0D8
:10F29000200080B20A2810DA200080B200F090FC32
:10F2A000684600F054F89DF8000010F001000028B6
:10F2B00001D101202BE0002029E0F9F701FC050035
:10F2C0000026200080B2864215D2684600F034F84D
:10F2D0009DF8000010F00100002804D1002000F08B
:10F2E00036F8012013E0012000F06AFCF9F7E8FB92
:10F2F000401B0600E5E7684600F029F89DF800008D
:10F3000010F00100002801D1012000E0002076BDAE
:10F3100038B50400FFF797FFDFF898080521017062
:10F32000DFF88C5801212A699047002C03D0012175
:10F3300020006A69904731BD10B50400002C05D04B
:10F3400001212000DFF868285269904710BD10B5F0
:10F350000400002C05D001212000DFF85428526958
:10F360009047FFF779FF10BD80B5684600F0B5F80B
:10F370009DF8000010F00100002801D1002001E0FC
:10F380007FF0050002BD80B5002000F0CDF90090AF
:10F39000BDF80000FF2802D15FF0FF3008E00A202E
:10F3A000FFF766FF002802D17FF01F0000E0002079
:10F3B00002BD80B50A20FFF75BFF002802D17FF075
:10F3C0001F0000E0002002BD3EB500F0D5FB1E206E
:10F3D000F6F77FFD00F093F9072000F0F1FB7FF0D6
:10F3E00007050024022C12D2FFF7CDFF0500002DE7
:10F3F00002D55FF0FF3000E00020002807D0002C8D
:10F4000001D028003AE000F0BCFB641CEAE7002DC4
:10F4100002D55FF0FF3000E00020002801D0280076
:10F420002CE0002000F080F90090BDF80000FF28DB
:10F4300002D15FF0FF3021E001A800F078FB002846
:10F4400002D15FF0FF3019E09DF80000EF2802D0F4
:10F450007FF0010012E09DF8030010F03F00152836
:10F4600002D07FF0020009E09DF80200402801D0A0
:10F47000702801D1002001E07FF003003EBD80B57F
:10F48000FFF7A2FF0100002902D55FF0FF3000E086
:10F490000020002801D0080000E0002002BD80B557
:10F4A000FFF7D1FEDFF80C07062101700121DFF81C
:10F4B000002712699047FFF7CFFE01BD80B5FFF727
:10F4C000C2FEDFF8F006042101700121DFF8E0261A
:10F4D00012699047FFF7C0FE01BD38B50400FFF781
:10F4E000B2FEDFF8D00605210170DFF8C456012115
:10F4F0002A699047012120006A699047FFF7ACFE16
:10F5000031BD38B50400FFF79EFEDFF8A8063521AF
:10F510000170DFF89C5601212A69904701212000E3
:10F520006A699047FFF798FE31BD38B50400FFF7D0
:10F530008AFEDFF8800615210170DFF8745601217C
:10F540002A699047012120006A699047FFF784FEED
:10F5500031BD10B50400FFF776FEDFF85806012133
:10F560000170217841700221DFF84426126990472A
:10F57000FFF772FE0F20FFF77BFE10BD10B50400F1
:10F58000FFF761FEDFF82C06312101702178417010
:10F590000221DFF81C2612699047FFF75DFE0F205D
:10F5A000FFF766FE10BD10B50400FFF74CFEDFF854
:10F5B000040611210170217841700221DFF8F02545
:10F5C00012699047FFF748FE0F20FFF751FE10BD6C
:10F5D000F8B504000D001600FFF735FEDFF8D4057E
:10F5E000032101702100090C41702100090A81707A
:10F5F000C470DFF8BC7504213A699047310089B2C4
:10F6000028007A699047FFF727FEF1BD70B5040026
:10F610000D00FFF718FEDFF89C0502210170DFF8EE
:10F6200098150D402900090C41702900090A8170C4
:10F63000C570DFF87C650421326990474FF4807112
:10F64000200032699047FFF707FE0320FFF710FE06
:10F6500070BD10B50400FFF7F6FDDFF85805202156
:10F660000170220092B24FF480514A43121442704A
:10F67000220092B24FF480514A431212827000214C
:10F6800001FB04F1C1700421DFF8242512699047C1
:10F69000FFF7E2FD10BD10B50400FFF7D4FDDFF861
:10F6A0001405D8210170220092B25FF480314A43E0
:10F6B00012144270220092B25FF480314A43121257
:10F6C0008270002101FB04F1C1700421DFF8E02405
:10F6D00012699047FFF7C0FD10BD80B5FFF7B3FD7D
:10F6E000DFF8D004B92101700121DFF8C4241269C8
:10F6F0009047FFF7B1FD0320F6F7EBFB01BD80B5A6
:10F70000FFF7A1FD0420F6F7E4FBDFF8A804AB2126
:10F7100001700121DFF8982412699047FFF79CFDE2
:10F720000420F6F7D6FB01BD7CB504000020ADF83F
:10F73000020000208DF8020000208DF80300002058
:10F740008DF8000000208DF8010000200090FFF7E8
:10F750007AFDDFF860649F203070DFF85454012197
:10F7600030002A699047012168466A699047012163
:10F770000DF102006A69904701210DF103006A69E9
:10F780009047FFF769FD002C20D0207900281DD07C
:10F79000FFF759FD5A203070002070700020707003
:10F7A0000020F07000203071052130002A69904758
:10F7B00000262079864207D20121D4F80500304482
:10F7C0006A699047761CF4E7FFF746FD009876BD1E
:10F7D00080B5FFF738FDDFF8DC03982101700121C7
:10F7E000DFF8CC2312699047FFF736FD01BD80B5E5
:10F7F000FFF729FDDFF8BC037E2101700121DFF84E
:10F80000B02312699047FFF727FD01BD70B50400D2
:10F810000D00FFF718FD2800C0B2002804D03621E3
:10F82000DFF89003017003E03921DFF888030170ED
:10F83000DFF880632000FFF7ADFC000C7070200043
:10F84000FFF7A8FC000AB0702000FFF7A3FCF070DF
:10F8500004213000D64A12699047FFF7FDFC70BDC5
:10F860007CB50400FFF7EFFC00208DF80000D14EBE
:10F870003D2030702000FFF78DFC000C70702000E0
:10F88000FFF788FC000AB0702000FFF783FCF070DF
:10F89000C74D042130002A699047012168466A69F2
:10F8A0009047FFF7D9FC9DF8000010F0010076BDED
:10F8B00038B50400002C1DD0FFF7C5FCBD4842211F
:10F8C000017000214170817811F00F0151F0100199
:10F8D0008170817811F0F00181700021C170B44D08
:10F8E00004212A6990474FF4807120002A699047CB
:10F8F000FFF7B2FC31BD38B50400002C1DD0FFF776
:10F90000A2FCAC484221017000214170817811F0C5
:10F910000F0151F020018170817811F0F0018170A8
:10F920000021C170A24D04212A6990474FF48071D3
:10F9300020002A699047FFF78FFC31BD38B50400DD
:10F94000002C1DD0FFF77FFC9A4842210170002156
:10F950004170817811F00F0151F030018170817890
:10F9600011F0F00181700021C170914D04212A69CC
:10F9700090474FF4807120002A699047FFF76CFC94
:10F9800031BD80B5FFF75FFC8A484421017000213A
:10F990004170817811F00F0151F010018170817870
:10F9A00011F0F00181700021C1700421804A1269B8
:10F9B0009047FFF751FC01BD80B5FFF744FC7D483F
:10F9C0004421017000214170817811F00F0151F044
:10F9D00020018170817811F0F00181700021C170E7
:10F9E0000421734A12699047FFF736FC01BD80B5C8
:10F9F000FFF729FC6F484421017000214170817894
:10FA000011F00F0151F030018170817811F0F00197
:10FA100081700021C1700421654A12699047FFF787
:10FA20001BFC01BD38B50400002C1DD0FFF70BFCFA
:10FA300060484821017000214170817811F00F0168
:10FA400051F010018170817811F0F0018170002176
:10FA5000C170574D04212A6990474FF480712000EE
:10FA60006A699047FFF7F8FB31BD38B50400002CF8
:10FA70001DD0FFF7E8FB4F4848210170002141707D
:10FA8000817811F00F0151F020018170817811F01F
:10FA9000F00181700021C170454D04212A69904711
:10FAA0004FF4807120006A699047FFF7D5FB31BDA4
:10FAB00038B50400002C1DD0FFF7C5FB3D48482198
:10FAC000017000214170817811F00F0151F0300177
:10FAD0008170817811F0F00181700021C170344D86
:10FAE00004212A6990474FF4807120006A69904789
:10FAF000FFF7B2FB31BD38B50400002C16D0FFF77C
:10FB0000A2FB2C484B210170002141700021817023
:10FB10000021C17000210171254D05212A699047FE
:10FB2000082120006A699047FFF796FB31BD10B5A8
:10FB30000400002C17D02000FFF7DDFF0021002279
:10FB40000023082B09D2E05CFF2800D1521CE05CA6
:10FB5000002800D1491C5B1CF3E7082903D0082AC0
:10FB600001D0012000E0002010BD80B5FFF774FB3C
:10FB700012480068804701BD80B510484068804742
:10FB800001BD80B50D48406880471E20F6F7A1F9F9
:10FB9000FFF7EBFF0A20F6F79CF9FFF7EDFF1E20B9
:10FBA000F6F797F901BD00002C1A0020311A002049
:10FBB00098980108083A002000FFFF00D8A3010828
:10FBC00031B50025F8F77CFF0400F8F779FF001B3A
:10FBD00000998842F9D331BD4020704738B5FFF70E
:10FBE000FBFF182802D25FF0FF3026E0DFF8BC18D8
:10FBF000012000F0ADFCDFF8B818022000F0A8FCEE
:10FC0000DFF8B04800202071002060710020A07152
:10FC100000F036FF206001F053FA050001F048FAC9
:10FC2000040001F049FA2A002100FBF775FD0028C5
:10FC300002D05FF0FF3000E0002032BD80B501202F
:10FC400000F0B4FC022000F0B1FCFBF7D4FD002072
:10FC500002BD18B589B006ACDFF85C0890E80E006C
:10FC600084E80E0006A8FCF776FC03ACDFF84C082D
:10FC700090E80E0084E80E0003A8FCF76CFC6C46CC
:10FC8000DFF83C0890E80E0084E80E006846FCF7B8
:10FC900062FCDFF820080021017100214171002180
:10FCA00081710AB010BD2DE9F047A0B007000C002B
:10FCB0001500387810F06000C0B2002802D020286B
:10FCC0003CD018E27878012837D17888002834D1E0
:10FCD000B888012804D0812811D082281ED02CE0B9
:10FCE0001DAEDFF8E00790E80E0086E80E001DA8C4
:10FCF000FCF731FC012001F06AF90120FCE11AAEA9
:10FD0000DFF8C40790E80E0086E80E001AA8FCF79A
:10FD100022FC812001F08AF90120EDE117AEDFF825
:10FD2000AC0790E80E0086E80E0017A8FCF713FC5D
:10FD3000822001F07BF90120DEE1DCE1DFF874676D
:10FD40003079002807D07878012802D07878052803
:10FD500001D1002030717079002807D0787803280D
:10FD600002D07878052801D100207071B079002880
:10FD700004D07878062801D00020B0717878012866
:10FD800016D002284CD003286ED0042800F0A7809B
:10FD9000052800F0DA80062800F02181072800F00D
:10FDA0003C81402800F05B81802800F07181A2E155
:10FDB000B888012801D000209EE15FF002085FF0C2
:10FDC000000916F1070A4A4641465046F2F73CF848
:10FDD00016F10800FBF731FF0DF1200CDFF8F006FB
:10FDE00090E80E008CE80E0078888DF8270008A8AF
:10FDF000FCF7B1FB002801D1012000E00020C0B2D7
:10FE0000002807D0012001F0B6F801203071012050
:10FE1000F07103E0002030718120F07101206BE16E
:10FE2000B888012801D0002066E15FF008085FF083
:10FE3000000916F1070A4A4641465046F2F704F80F
:10FE4000307900280CD0002000906846FBF73AFF7C
:10FE50000098C6F80B000120F0710020307101E01D
:10FE60008220F071012047E1B888812801D000206C
:10FE700042E15FF002085FF0000916F1070A4A4606
:10FE800041465046F1F7E0FF16F10800FBF7F7FE98
:10FE90000DF1140CDFF83C0690E80E008CE80E0023
:10FEA00078888DF81B0005A8FCF755FB002801D1C8
:10FEB000012000E00020C0B200280AD0812001F01B
:10FEC000B5F8812000F03DFB012070710120F07138
:10FED00003E0002070718120F07101200CE1B888EE
:10FEE000812801D0002007E15FF008085FF00009D9
:10FEF00016F1070A4A4641465046F1F7A5FF7079C8
:10FF000000281ED00020019001A8FBF7EFFE002181
:10FF1000812001F0D9F8002809D10198C6F80B001A
:10FF2000002030720120F071002070710BE0002081
:10FF3000C6F80B00012030720220F07101207071B0
:10FF400001E08220F0710120D6E0B888002801D0BD
:10FF50000020D1E05FF001085FF0000916F1070A08
:10FF60004A4641465046F1F76FFF012001F003F881
:10FF70000DF1500CDFF8600590E80E008CE80E00E3
:10FF800014A8FCF7E8FA812001F050F811ABDFF873
:10FF90004C0590E8061083E8061011A8FCF7DBFA80
:10FFA000822001F043F80DF1380CDFF8340590E8B9
:10FFB0000E008CE80E000EA8FCF7CDFA0DF12C0C0B
:10FFC000DFF8200590E80E008CE80E000BA8FCF787
:10FFD000C2FA0120F0710120B07101208CE0B888D4
:10FFE000002801D0002087E05FF002085FF00009E0
:10FFF00016F1070A4A4641465046F1F725FFB07907
:020000040801F1
:10000000002806D0002030720120F0710020B0716D
:1000100001E08220F07101206EE0B888002801D054
:10002000002069E05FF018085FF0000916F1070A88
:100030004A4641465046F1F707FF0120F0714FF460
:100040008070A6F809000421F17200213173A6F82E
:100050001300042070750C20B07501204CE0B888A6
:10006000002801D0002047E05FF001085FF00009A0
:1000700016F1070A4A4641465046F1F7E5FE0120CF
:10008000F0710120DFF8601489688847012033E0AF
:10009000B888002801D000202EE0B878000604D4EB
:1000A000B87810F07F00022801DA002024E05FF029
:1000B00003085FF0000916F1070A4A464146504618
:1000C000F1F7C2FE0120F071B87810F07F003072B5
:1000D00000207072812000F0A9FF02AB00220020F6
:1000E000002183E80700307A8DF8100002A8FCF7A1
:1000F00032FA012000E0002020B0BDE8F08710B403
:100100000400002010BC70472DE9F04105000E00EE
:1001100014001F005FF00008002C01D000207BE0DD
:10012000287810F06000202875D16878012810D058
:1001300002281AD003280CD0042822D005282CD05D
:10014000062836D0072840D040284AD0802854D0EE
:1001500061E0022F08D10222DFF890133000FAF795
:10016000CCFF10EB0800804655E0082F08D108228C
:10017000DFF878133000FAF7C0FF10EB0800804674
:1001800049E0082F08D10822DFF860133000FAF7A1
:10019000B4FF10EB080080463DE0012F08D101229A
:1001A000DFF848133000FAF7A8FF10EB080080468C
:1001B00031E0022F08D10222DFF830133000FAF7C5
:1001C0009CFF10EB0800804625E0182F08D118226C
:1001D000DFF818133000FAF790FF10EB08008046A4
:1001E00019E0012F08D10122DFF800133000FAF7DF
:1001F00084FF10EB080080460DE0032F0BD1032293
:10020000DFF8E8123000FAF778FF10EB08008046BC
:10021000822000F086F94046BDE8F081FEB5050079
:100220000E006F46DFF8C80290E80E0087E80E0067
:1002300001966846FCF78FF90400002C5AD4012C73
:1002400061DB2100012919D002292ED0032920D0F9
:1002500004291FD005293ED0062931D07FF009009E
:1002600081423CD114F10A0F07D14FF44A72A149DF
:10027000A148F1F77DFDAFF3008044E0012C07D1E8
:1002800040F22E329B499D48F1F772FDAFF300809A
:1002900039E0C6E7042C07D140F23A329549984834
:1002A000F1F766FDAFF300802DE0022C07D14FF48B
:1002B000507290499348F1F75BFDAFF3008022E064
:1002C000062C07D140F246328A498F48F1F750FD9B
:1002D000AFF3008017E0812000F02BF913E0002C31
:1002E00011D04FF4557283498848F1F741FDAFF3BF
:1002F000008008E014F1080F02D1812000F03BFEDD
:10030000012000F038FE002C01D4012000E0002084
:10031000C0B2FEBD7FB505000E006C467C4890E87B
:100320000E0084E80E0001966846FCF714F90400FC
:10033000002C50D4012C4CDB2100012919D00229BA
:1003400038D0032920D0042929D0052936D0062900
:1003500030D07FF00900814231D114F10A0F07D16A
:1003600040F2793263496448F1F702FDAFF300804F
:100370002FE0012C07D140F27F325E495F48F1F750
:10038000F7FCAFF3008024E0032C07D140F2853264
:1003900058496048F1F7ECFCAFF3008019E0042CF9
:1003A00007D140F28B3253495548F1F7E1FCAFF3E6
:1003B00000800EE0812000F039FE0AE009E0002C08
:1003C00007D040F29E324B495048F1F7D1FCAFF3D1
:1003D0000080012000E0002004B070BD0200012078
:1003E00070477FB505000E006C464B4890E80E0044
:1003F00084E80E0001966846FCF7ADF80400002C76
:1004000050D42100002940D0012919D0022938D028
:10041000032920D0042929D0052936D0062930D037
:100420007FF00900814231D114F10A0F07D14FF456
:100430006F7230493048F1F79BFCAFF300802FE03A
:10044000012C07D140F2C2322A492C48F1F790FC26
:10045000AFF3008024E0032C07D14FF472722549DA
:100460002C48F1F785FCAFF3008019E0042C07D18C
:1004700040F2CE321F492248F1F77AFCAFF30080F8
:100480000EE0822000F0D2FD0AE009E0002C07D047
:1004900040F2E23217491D48F1F76AFCAFF30080E1
:1004A000012000E0002004B070BD0000A09D010804
:1004B000B49D0108303A0020E4070020F007002036
:1004C000FC07002008080020140800202008002055
:1004D00060A301086CA301082C0800203808002044
:1004E00044080020500800203C910108373A0020C1
:1004F00078A30108E8820108E89201081096010833
:1005000034960108109301083893010854970108A4
:1005100084A301087497010890A301080200012038
:10052000704710B5040000212000C0B200F0ECFCC0
:1005300010BD10B5040001212000C0B200F0E4FCA1
:1005400010BD10B504002000C0B200F001FD10BDC8
:1005500070B506000C0016F07F063000C0B200280F
:1005600022D03000C0B208281EDA002C1CD0DFF8E0
:10057000F8543000C0B255F82000002814D120688B
:10058000002805D13000C0B245F8204001200CE021
:100590003000C0B221688847002805D03000C0B2C2
:1005A00045F82040012000E0002070BD38B505006E
:1005B00015F07F052800C0B2002821D02800C0B265
:1005C00008281DDADFF8A0442800C0B254F8200043
:1005D00000280ED02800C0B254F82000006900287E
:1005E00007D02800C0B22900C9B254F82110096907
:1005F000884700212800C0B244F82010012000E004
:10060000002032BD70B50021DFF860040160DFF822
:10061000604425680026042E0CD22868804701001B
:1006200049B2002901D040B205E0761C54F82600FA
:100630000500F0E7002070BD70B50021DFF834043C
:100640000160DFF8241408680022082A07D200237A
:1006500041F82230521C51F822301800F5E7DFF83B
:1006600018240A60DFF814542E680024002C0CD1E2
:1006700030688047010049B2002901D040B205E04E
:10068000641C55F824000600F0E7002070BD70B52A
:100690000021DFF8D8030160DFF8D4432568002685
:1006A000042E06D268688047761C54F826000500A0
:1006B000F6E7002070BD70B50021DFF8B8030160D7
:1006C000DFF8B8532E680024002C06D170688047EC
:1006D000641C55F824000600F6E7DFF88C03016877
:1006E0000022082A07D2002340F82230521C50F87A
:1006F00022301900F5E7002070BD70B5DFF87043B7
:1007000025680026042E06D268698047761C54F8B6
:1007100026000500F6E770BD70B5DFF860532E685F
:100720000024002C06D170698047641C55F8240011
:100730000600F6E770BD2DE9F84304000D00160031
:100740002800C0B200281ED0DFF82473D7F800803C
:100750005FF00009B9F1040F15D23200D2B22900BE
:10076000C9B22000D8F808309847002805D0DFF833
:10077000FC02C0F80090012009E019F1010957F8C6
:1007800029008046E6E70021B84801600020BDE866
:10079000F2832DE9F84305000E0017003000C0B2C7
:1007A000002819D0DFF8D482D8F800900024002C5B
:1007B00012D13A00D2B23100C9B22800D9F80830BB
:1007C0009847002803D0AB480460012008E0641C6F
:1007D00058F824008146EAE70021A648016000207D
:1007E000BDE8F283F8B504000D0016001F003B00C1
:1007F000320029002000DFF878C2DFF870E2DEF86E
:1008000000E05CF82EC0DCF80CC0E047F2BDF8B5A3
:1008100004000D0016001F003B00320029002000DC
:10082000DFF858C2DFF84CE2DEF800E05CF82EC0DA
:10083000DCF80CC0E047F2BDF8B504000D0016006E
:100840001F003B00320029002000DFF824C2DFF83F
:100850001CE2DEF800E05CF82EC0DCF810C0E047D7
:10086000F2BDF8B504000D0016001F003B00320079
:1008700029002000DFF804C2DFF8F8E1DEF800E02C
:100880005CF82EC0DCF810C0E047F2BD0300002A7F
:1008900008D01800C0B2012804D19078002801D1F6
:1008A000012000E0002070470300002A08D0180053
:1008B000C0B2012804D19078002801D1012000E0C5
:1008C00000207047002A06D00300DBB2012B02D1C2
:1008D0009378002BFFD07047002A06D00300DBB2CC
:1008E000012B02D19378002BFFD0704770B5050023
:1008F0000E0000242800C0B200281DD02800C0B27D
:1009000010F07F00082817DA57492800C0B210F00D
:100910007F0051F82040002C01D1012000E0002090
:10092000C0B2002808D1606800281CD0310028001F
:10093000C0B26268904717E02800C0B2002812D009
:1009400049480468002C01D1012000E00020C0B219
:10095000002808D16068002805D031002800C0B206
:100960006268904700E0002070BD70B505000E0081
:1009700000242800C0B200281DD02800C0B210F00A
:100980007F00082817DA38492800C0B210F07F002D
:1009900051F82040002C01D1012000E00020C0B21D
:1009A000002808D1A06800281CD031002800C0B25F
:1009B000A268904717E02800C0B2002812D02A4849
:1009C0000468002C01D1012000E00020C0B2002802
:1009D00008D1A068002805D031002800C0B2A26864
:1009E000904700E0002070BD70B505000E000024A7
:1009F0002800C0B200281DD02800C0B210F07F002F
:100A0000082817DA18492800C0B210F07F0051F802
:100A10002040002C01D1012000E00020C0B20028BD
:100A200008D1E06800281CD031002800C0B2E2687C
:100A3000904717E02800C0B2002812D00A48046886
:100A4000002C01D1012000E00020C0B2002808D114
:100A5000E068002805D031002800C0B2E268904765
:100A600000E0012070BD0000503A0020143B00203F
:100A700004A00108183B00208C9D0108F0A7010884
:100A8000DFF884160868002805D008680068D0F8E8
:100A90001002406A00E0002070472DE9FE4F04007C
:100AA0000D00002641F29000F4F706FCC4F8140291
:100AB000D4F81402002802D102200600BDE0D4F8C8
:100AC00014028346CBF80040DFF83C06C0F800B0C3
:100AD000D4F818724023022201212000F4F741FAD1
:100AE0004020C4F820014023022281212000F4F795
:100AF00038FA402020634023032282212000F4F7AB
:100B000030FA022020642000F4F706FC0094002351
:100B100040221BF190011BF10400FAF7A9FA00949E
:100B2000002340221BF1D0011BF12000FAF7A0FAAC
:100B3000009400234FF45C621BF588711BF13C00AC
:100B4000FAF796FA009400234FF4C0721BF56D611A
:100B50001BF15800FAF78CFA00940023402241F26E
:100B600050000BEB00011BF17400FAF781FA3868B2
:100B7000804700285FD11BF1580201212000FAF7BD
:100B80002EFA94F8FC01012804D17869002801D0DC
:100B90007869804794F8FC0103284ED1F869002851
:100BA0004BD00020ADF800005FF00008D4F8100230
:100BB000406AC06900280AD06946207CD4F8102217
:100BC000526AD269904780460020060001E0022068
:100BD00006003000C0B200282FD1CDF808805FF0A9
:100BE0000009BDF80000002824D0C2469AF8000091
:100BF00000281FD09AF80100042810D1CDF80480F5
:100C0000019A4946C9B22800C0B2FB69984719F158
:100C10000109C0B2002802D1022006000AE0BDF896
:100C200000109AF80000091AADF800109AF80000B8
:100C30008044D6E701E0022006003000C0B2BDE8E3
:100C4000FE8F2DE9FE4F81460C000025D9F81402D5
:100C500000287BD0D9F81802002877D0D9F818627C
:100C6000306A002850D099F8FD01032803D099F884
:100C7000FD01042848D199F8FC01032803D199F813
:100C8000FC01042840D00020ADF800000027D9F86E
:100C90001002406AC06900280BD0694699F810001C
:100CA000D9F81022526AD269904707000020050047
:100CB00001E0022005002800C0B2002824D10197DD
:100CC0005FF00008BDF8000000281DD0BA469AF871
:100CD0000000002818D09AF80100042809D1BB466A
:100CE0005A464146C9B22000C0B2336A984718F14B
:100CF0000108BDF800109AF80000091AADF80010BC
:100D00009AF800000744DDE799F8FC01012804D1B6
:100D10007069002801D070698047706880470021A1
:100D2000DFF8E4030160D9F81402F4F7D0FA0020E8
:100D3000C9F8140201214846F4F78DF9812148468B
:100D4000F4F789F982214846F4F785F92800C0B202
:100D5000BDE8FE8F70B504000D00D4F81402002821
:100D60001BD0D4F81802002817D0D4F81862280035
:100D7000C0B2002809D1B06800280ED0002200219E
:100D800014F50270B368984707E0306B002804D070
:100D900000212800C0B2326B9047002070BD2DE9C1
:100DA000F84380460C000025D8F81462D8F8187271
:100DB000B868002801D102206EE000220121200045
:100DC000BB689847002801D1022065E0207810F028
:100DD0006000C0B200282FD0202801D0402850D178
:100DE000E088002824D0207800060FD5CDF80080B8
:100DF0000023402216F19001301DFAF739F9321D17
:100E000021004046F9F731FF050014E0CDF80080DD
:100E10000023402216F1D00116F12000FAF728F93C
:100E200016F1200221004046F9F71FFF050002E0FD
:100E30004046F5F7B5FE24E060780A2802D00B287A
:100E40001ED01DE0786A002817D0B4F80490002066
:100E50008DF800006A464946C9B2D8F80400C0B20D
:100E60007B6A9847002805D0012269464046F5F77D
:100E7000C3FD04E00220050001E002200500FFE7B9
:100E8000FFE72800C0B2002804D000220021200083
:100E9000BB6898472800C0B2BDE8F28370B5060071
:100EA0000C00D6F81452220015F120013000F9F799
:100EB00018FD70BD70B506000C00D6F81452220063
:100EC000291D3000F9F72CFE70BD70B504000D002F
:100ED000D4F8146255F08000C0B2812802D0822874
:100EE00008D00FE016F13C022900C9B22000F9F742
:100EF00096FF08E016F174022900C9B22000F9F744
:100F00008EFF00E0022070BDF8B504000D007E48A1
:100F10000668376854F08000C0B2812802D0822869
:100F20000AD013E02B00DBB216F13C022100C9B25B
:100F30003800F9F706FF0AE02B00DBB216F1740265
:100F40002100C9B23800F9F7FCFE00E00220F2BD32
:100F500070B504006C4805682E6854F08001C9B271
:100F60008139012905D82100C9B23000F9F73AFFCB
:100F700000E0022070BD70B5060063480468256873
:100F80003000C0B201280ED0812802D0822814D0AF
:100F90001CE03100C9B22800F4F77EF814F13C00DF
:100FA000FAF75BF812E03100C9B22800F4F774F8E0
:100FB00014F15800FAF751F808E03100C9B22800DE
:100FC000F4F76AF814F17400FAF747F870BD70B5D9
:100FD00006004D48046825683000C0B201280ED0D4
:100FE000812802D0822817D01FE014F13C00FAF7C4
:100FF00034F83100C9B22800F4F76FF815E014F1A5
:1010000058023100C9B22800F9F7E9FF3100C9B22E
:101010002800F4F762F808E014F17400FAF71DF8FC
:101020003100C9B22800F4F758F870BD70B5060059
:101030003548046825683000C0B201280ED08128E8
:1010400002D0822814D01CE014F13C00FAF705F815
:101050003100C9B22800F4F761F812E014F1580029
:10106000F9F7FBFF3100C9B22800F4F757F808E0A0
:1010700014F17400F9F7F1FF3100C9B22800F4F758
:101080004DF870BDF8B504000F001500D4F81462D7
:101090003800C0B2012809D12B00DBB216F158028A
:1010A0003900C9B22000F9F727FF00E00220F2BDA5
:1010B000154800683C307047134800685830704746
:1010C00011480068743070472DE9F04105000C00AC
:1010D0000D48066837685FF000082900C9B238007B
:1010E000F5F776FD010011F1010F01D1012000E0BB
:1010F0000020C0B2002801D0002003E0002C00D066
:1011000021600120BDE8F0811C3B002010B50400E7
:10111000002C01D1012011E02068016831F040016C
:1011200020680160200000F0AAFC0020606500201B
:1011300084F85100002084F85000002010BDF8B55C
:1011400007000C0015001E0097F85100012840F020
:10115000DB80002C03D0280080B2002801D10120C0
:10116000D3E097F85000012801D10220CDE0012002
:1011700087F85000122087F85100002078653C6302
:10118000BD86FD860020F8640020B8640020B863A6
:101190000020B8870020F887B86AB0F5005F0BD14F
:1011A0003868016831F400513868016038680168B6
:1011B00051F4005138680160B868B0F5004F05D1AE
:1011C0003868016851F48041386801603868006807
:1011D000400605D43868016851F040013868016064
:1011E000F868002830D17868002802D0F88E0128ED
:1011F00008D1386B411C396301783868C160F88EBA
:10120000401EF886F88E002813D0330000220221F9
:10121000380000F0BAFB002801D0032075E0386BDD
:10122000411C396301783868C160F88E401EF88629
:10123000E8E7B86AB0F5005F38D13868016851F462
:1012400080513868016031E07868002802D0F88E5B
:10125000012809D1386B01883868C160386B801C5F
:101260003863F88E401EF886F88E002814D03300BC
:1012700000220221380000F088FB002801D0032062
:1012800043E0386B00883968C860386B801C38636D
:10129000F88E401EF886E7E7B86AB0F5005F05D122
:1012A0003868016851F480513868016033000022C9
:1012B0000221380000F069FB002805D0786D50F05D
:1012C00020007865032020E03300012280213800CF
:1012D00000F05BFB002805D0786D50F020007865A9
:1012E000032012E0B868002806D13868C068009072
:1012F0003868806800900098012087F8510000202D
:1013000087F85000002000E00220F2BDFEB5070083
:101310000C0015001E000020ADF8040097F85100E5
:10132000012840F00E81002C03D0280080B2002854
:1013300001D1012006E197F85000012801D10220D7
:1013400000E1012087F85000222087F8510000209A
:101350007865BC63BD87FD870020B8640020F86411
:10136000002038630020B8860020F886B868B0F501
:10137000004F05D13868016831F480413868016058
:10138000B86AB0F5005F0BD13868016831F40051DC
:10139000386801603868016851F4005138680160AC
:1013A0007868B0F5827F0ED1B86800280BD1002094
:1013B00087F8500000962B009BB2220021003800D5
:1013C00000F0C1F8BEE038680068400605D438680F
:1013D000016851F0400138680160F868002821D1A7
:1013E000F88F022813DB330000220121380000F0BF
:1013F000CCFA002801D00320A4E0B86B411CB963EB
:101400003968C9680170F88F401EF887E8E7B86A44
:10141000B0F5005F28D13868016851F48051386810
:10142000016021E0F88F022814DB33000022012143
:10143000380000F0AAFA002801D0032082E03868C2
:10144000C168B86B0180B86B801CB863F88F401E10
:10145000F887E7E7B86AB0F5005F05D1386801683A
:1014600051F48051386801603300002201213800B6
:1014700000F08BFA002801D0032063E0F868002810
:1014800006D1B86B411CB9633968C968017006E0C0
:101490003868C168B86B0180B86B801CB863F88F7E
:1014A000401EF887B86AB0F5005F13D13300002200
:1014B0000121380000F069FA002805D0786D50F05D
:1014C0000200786503203DE03868C068ADF804008C
:1014D000BDF804007868B0F5827F0DD1B868B0F52A
:1014E000004F03D0B868B0F5806F05D13868016847
:1014F00031F0400138680160012087F85100B86A76
:10150000B0F5005F18D138688068C00614D5786DD2
:1015100050F0020078653868016831F4005138688D
:1015200001603868016851F400513868016000209A
:1015300087F85000012005E0002087F850000020C7
:1015400000E00220FEBD2DE9FC4180460C001500A4
:101550001E00089F0020ADF8000098F851000128F7
:1015600004D098F85100222840F00C82002C05D0BD
:10157000002D03D0300080B2002801D1012002E20A
:1015800098F85000012801D10220FCE1012088F8E0
:10159000500098F85100012802D1322088F85100FB
:1015A0000020C8F85400C8F83850A8F83C60A8F8E3
:1015B0003E60C8F83040A8F83460A8F836600020D3
:1015C000C8F848000020C8F84C00D8F82800B0F54A
:1015D000005F0FD1D8F80000016831F40051D8F84D
:1015E00000000160D8F80000016851F40051D8F8FB
:1015F00000000160D8F800000068400607D4D8F861
:101600000000016851F04001D8F800000160D8F8EE
:101610000C00B0F5006F40F0B380D8F8040000284B
:1016200008D0D8F80400B0F5827F13D1B8F836009E
:1016300001280FD1D8F830000188D8F80000C16027
:10164000D8F83000801CC8F83000B8F83600401ECA
:10165000A8F83600B8F83600002827D1D8F82800B6
:10166000B0F5005F07D1D8F80000016851F480514F
:10167000D8F8000001603B0000220121404600F044
:1016800084F9002801D003207DE1D8F80000C1686A
:10169000D8F838000180D8F83800801CC8F8380025
:1016A000B8F83E00401EA8F83E000DE1B8F836003C
:1016B000002845D03B0000220221404600F065F999
:1016C000002801D003205EE1D8F830000188D8F866
:1016D0000000C160D8F83000801CC8F83000B8F8AD
:1016E0003600401EA8F83600B8F8360000280CD1A5
:1016F000D8F82800B0F5005F07D1D8F800000168DD
:1017000051F48051D8F8000001603B000022012113
:10171000404600F03AF9002801D0032033E1D8F820
:101720000000C168D8F838000180D8F83800801C63
:10173000C8F83800B8F83E00401EA8F83E00B5E7EB
:10174000D8F80400002840F0BF803B0000220121AF
:10175000404600F01AF9002801D0032013E1D8F820
:101760000000C168D8F838000180D8F83800801C23
:10177000C8F83800B8F83E00401EA8F83E00A3E0C4
:10178000D8F80400002808D0D8F80400B0F5827F0B
:1017900011D1B8F8360001280DD1D8F83010481C06
:1017A000C8F830000878D8F80010C860B8F83600DB
:1017B000401EA8F83600B8F83600002822D1D8F824
:1017C0002800B0F5005F07D1D8F80000016851F497
:1017D0008051D8F8000001603B0000220121404602
:1017E00000F0D3F8002801D00320CCE0D8F80000A6
:1017F000C168D8F838000170B8F83E00401EA8F85B
:101800003E0061E0B8F83600002841D03B000022DD
:101810000221404600F0B9F8002801D00320B2E0D0
:10182000D8F83010481CC8F830000978D8F8000003
:10183000C160B8F83600401EA8F83600B8F8360087
:1018400000280CD1D8F82800B0F5005F07D1D8F8EF
:101850000000016851F48051D8F8000001603B009D
:1018600000220121404600F090F8002801D003201A
:1018700089E0D8F83800411CC8F83810D8F80010B2
:10188000C9680170B8F83E00401EA8F83E00B9E7EC
:10189000D8F80400002817D13B000022012140465F
:1018A00000F073F8002801D003206CE0D8F838006D
:1018B000411CC8F83810D8F80010C9680170B8F891
:1018C0003E00401EA8F83E00D8F82800B0F5005FA2
:1018D00016D13B0000220121404600F056F80028B6
:1018E00007D0D8F8540050F00200C8F85400032084
:1018F00049E0D8F80000C068ADF80000BDF800006D
:101900003B0001228021404600F03FF8002807D02C
:10191000D8F8540050F02000C8F85400032032E0FA
:10192000012088F85100D8F82800B0F5005F24D1D4
:10193000D8F800008068C0061FD5D8F8540050F0D1
:101940000200C8F85400D8F82800B0F5005F0FD1A5
:10195000D8F80000016831F40051D8F800000160A7
:10196000D8F80000016851F40051D8F80000016077
:10197000002088F85000012005E0002088F8500081
:10198000002000E00220BDE8F6812DE9F8430500C3
:101990000E0017001C005FF00009F7F791F8804671
:1019A0003800C0B2002833D1286880683040B04287
:1019B00062D014F1010FF7D0002C05D0F7F780F8B2
:1019C000B0EB08008442EFD22868416831F0E001B2
:1019D000286841602868016831F04001286801608A
:1019E000A86AB0F5005F0BD12868016831F4005196
:1019F000286801602868016851F400512868016076
:101A0000012085F85100002085F85000032034E0C3
:101A1000286880683040B0422ED114F1010FF7D011
:101A2000002C05D0F7F74CF8B0EB08008442EFD259
:101A30002868406830F0E00029684860286801683C
:101A400031F0400128680160A86AB0F5005F0BD151
:101A50002868016831F4005128680160286801682D
:101A600051F4005128680160012085F851000020E0
:101A700085F85000032000E00020BDE8F2837047A5
:101A8000C0B20A2801D1012000E00020C0B2704796
:101A900070B506000C0015002A0012B221003000BB
:101AA00000F0A1FC002801D1002001E07FF003003C
:101AB00070BD70B504000D0016003000020012B2B7
:101AC00029002000FFF7E4FF002801D1012000E0F9
:101AD0000020C0B270BD01000800406870470100DE
:101AE0000800C0B2062805D2DFF86C08C9B200EBC6
:101AF000C10000E0002070472DE9F04104000D0016
:101B00002800C0B2062808D37122DFF85018DFF889
:101B10005008F0F72DF9AFF300802800C0B2062876
:101B200019D2DFF83468B04616F12807444501DBC6
:101B3000A74208DA7822DFF82418DFF82808F0F73F
:101B400017F9AFF30080444505DBA74203DBEDB294
:101B500006EBC50000E00020BDE8F0812DE9F34F61
:101B60008BB014001D00169E179FDFF8FC870B98A2
:101B7000C8F83C005FF0000A5FF07F0B0C9800286B
:101B80003CD0082100220DF124094846F0F75CF909
:101B90000B9BDFF8D827082109A8F4F788F809A8D3
:101BA000F8F79AFD0090009858450BD209A908EB68
:101BB0000A00403000F0B2FD0098BBEB000B00982B
:101BC00010EB0A0A0C98F8F787FD8146B9F1800FEF
:101BD00008D3A122DFF88417DFF89407F0F7C8F8DC
:101BE000AFF30080D94509D20C9908EB0A004030C8
:101BF00000F094FDBBEB090B19EB0A0A002C01D095
